:020000040800F2
:100000000002002029050008C5040008810400083A
:10001000D5040008E5040008F5040008000000000D
:10002000000000000000000000000000450400087F
:100030000505000800000000290400081505000857
:100040008901000889010008890100088901000868
:10005000890100088901000899160008991600080E
:1000600099160008991600089916000889010008D9
:100070008901000889010008890100088901000838
:100080008901000889010008890100088901000828
:1000900089010008890100088901000899160008F3
:1000A0008901000889010008890100088901000808
:1000B0003118000889010008890100088901000839
:1000C00089010008890100088901000889010008E8
:1000D0008901000889010008491200084F12000830
:1000E00099160008890100088901000889010008A3
:1000F00089010008890100088901000889010008B8
:1001000089010008890100083718000889010008E2
:100110008901000889010008890100088901000897
:100120008901000889010008890100088901000887
:100130008901000889010008890100088901000877
:100140008901000889010008890100088901000867
:100150008901000889010008890100088901000857
:100160008901000889010008890100088901000847
:1001700089010008890100088901000800000000C9
:10018000000000008901000800F0C4B900F004BBC1
:100190007047000070B50C46064600F061F9094B47
:1001A000094A1D682919914202D8084A914204D28D
:1001B0000C2333604FF0FF3500E0196000F058F970
:1001C000284670BD0002002000000220E0640020EC
:1001D0001946104600F0ECBA1946104600F0F0BA85
:1001E000132303604FF0FF307047132303604FF079
:1001F000FF307047132303604FF0FF307047022930
:100200004FF0000303608CBF002001207047000006
:10021000114B70B500241C60104B114D18682E68EE
:1002200000F09CF80F4B53F820301B68A3F1080234
:1002300096420FD026B13179092904BF0A213171C4
:10024000092103F8041C33F9021C074B2A601980AA
:10025000012070BD204670BDF8020020CC030020B4
:100260000003002008030020FC020020082930B50C
:10027000037919D9082B32D842791A4B53F82250F6
:1002800000F108042DB12D68856053F822502C60D0
:1002900000E0846043F82240134C4279012303FAC2
:1002A00002F22368134319E0082B18D945790D4B46
:1002B00053F825203AB11468A2420BBF00222468EB
:1002C00043F825201460427953F822303BB9064C9C
:1002D000012303FA02F2236823EA02032360017177
:1002E00030BD00BF08030020CC03002008B50A4B36
:1002F0001B681A79082A02D95B7983420AD900F06F
:10030000BAF818B1054B01221A6008BDBDE80840D3
:1003100000F082B808BD00BF00030020F8020020F2
:1003200008B500F09DF8094B094A1B88094D1BB21E
:10033000002442F82340084A286813682146013BFC
:100340001360FFF793FF2C6000F062F8FC020020BE
:100350004803002000030020040300200023C207FC
:1003600002D440080133FAE718467047134423F0DB
:10037000030310B54FF077321C1F43F8042C6207BB
:1003800042BF4FF0883243F8082CA3F108044FF025
:10039000807304E909000F4B44F80C3C002344F837
:1003A000103C032344F8143C2246022344F8183C32
:1003B000012344F81C3C42F8201D0B2342F8043D65
:1003C000013B032BFAD120466FF0020340F8443D75
:1003D00010BD00BF21030008064B0749074A1868F3
:1003E000884203D1934201D20433F8E70348C01A8C
:1003F000704700BF00000020FEE7FEE7000200207B
:10040000EFF30880704700000048704700000020AC
:1004100000F02AF801DFFEE7024A536843F08053F8
:100420005360704700ED00E0EFF3098020E9F00F22
:1004300040F804ED02490968086000F003F8000084
:1004400000030020FFF7E4FE04480068016801C9CA
:10045000B1E8F00F81F30988004700000003002095
:10046000EFF3108072B6704762B6EFF310807047FA
:1004700080F310887047EFF30580C0B2704700002A
:100480000D490E4A0E4B6846904203D8984201D956
:10049000002102E009468D460121042072460242F5
:1004A00002D1EFF3088001E0EFF309802DE9F00FAE
:1004B0006B4600F06FF800BF000200200000022031
:1004C0006005002008B50249042000F08DFB00BF44
:1004D000CC16010808B50249062000F085FB00BFD4
:1004E000D816010808B50249072000F07DFB00BFBF
:1004F000EB16010808B50249082000F075FB00BFA3
:10050000FD16010808B50249092000F06DFB00BF87
:100510001117010808B502490A2000F065FB00BF69
:10052000231701087047704708B5FFF7FBFF6A46BD
:10053000114B1249934202D243F8041BFAE7104AC6
:10054000104B11498B4204D252F8040F43F8040BAC
:10055000F8E70E4B0E4A0021934202D243F8041BE7
:10056000FAE7FFF7E0FF00F01FFB0FF09DF9BDE891
:10057000084000F073BB00BF00000020FEE7FEE76C
:100580009C52010800020020F8020020F80200201E
:10059000E06400202DE9F04F9A46494B8FB0934616
:1005A0009A6B03925A6B04929F6ADA6A05921A6BED
:1005B000DB6B0793434B06921A68434B9A420446FF
:1005C000884602D041480FF059FCB8F1000F05D021
:1005D0003F4800250FF052FC2E4626E094E80E001E
:1005E000E068D4F81C9008902069099060690A902E
:1005F00019F4007F3748A6690D930CBF04F120055C
:1006000004F124050C920B910FF038FC089B009329
:100610000BA90EC930480FF0A7FBCDF80090334668
:100620000A9A09992D480FF09FFB2D480FF026FCE0
:1006300039462C480FF098FB05992B480FF094FB96
:1006400006992A480FF090FB079929480FF08CFB78
:100650003A0403D5039927480FF086FB3B0603D5E0
:10066000049925480FF080FB24480FF007FC5946F9
:1006700023480FF079FBB8F1000F1BD121480FF090
:10068000FDFB314620480FF06FFB69461F4BC91A2E
:1006900003D549421E480FF067FB20468268C368B5
:1006A00001698C4641698E46AD46514691E8F00F8E
:1006B0004168006801BE1749052000F095FA00BFA7
:1006C00000ED00E000000020FEE7FEE73117010822
:1006D000471701087617010891170108CE1701087E
:1006E0000C1801081518010825180108351801080B
:1006F0004518010855180108651801087518010802
:100700007A1801088C180108BD180108580100204A
:10071000E51801081219010810B568B1012815D1B2
:10072000174A136823F003031360136843F400733C
:1007300043F0010313601BE0114B1A6842F00E02F4
:100740001A605A6842F480725A6011E00D4A1369C7
:1007500023F0040313610024FFF782FEBFF34F8FE1
:1007600030BFFFF785FE54B1BDE8104000F010BC6B
:10077000044A136943F0040313610124ECE710BD3C
:100780000070004000ED00E008B5FFF769FE0020B2
:10079000BDE80840FFF7C0BF034B044A4FF4E13106
:1007A000002000F0C7BC00BF04020020270E000894
:1007B0000A460146014800F041BB00BF0402002088
:1007C00010B50A460C460146002000F019FD2046EF
:1007D00010BD002000F0D6BF034B1968024611B9C6
:1007E000084600F0AFBF70471404002010B5094A56
:1007F00013685BB19C6881688C4202D21A461B6800
:10080000F7E703D15C6841688C42F7D90360106058
:1008100010BD00BF20040020F0B51F4E1F4D3368EF
:100820001F4C013333601F4B00201A6818602B687F
:10083000226019460746B64641B1DEF800C08E6810
:10084000664503D80F4601200968F5E700B1296025
:1008500007B9F0BD00213960E2B133B15168586881
:10086000814294BF1146194600E0114608461268BD
:100870001B680AB903600BE00BB9026008E0556819
:100880005E68B54294BF15461D4605602846EEE7F2
:100890002160F0BD2360F0BD18040020200400207A
:1008A0001C040020100400202DE9F0412E4F2F4C95
:1008B00001233B6023683BB9FFF7AEFFFFF789FFD9
:1008C0000130FBD0002502E0FFF783FF05464FF023
:1008D0000008236823B9FFF77CFF854214D91AE08A
:1008E0005E68FFF776FF854208D923685E68FFF7E8
:1008F00070FFA8422CD3B042F7D329E08642F4D946
:10090000361A132EE7D8F0E7236843B9FFF761FFE3
:10091000854206460BD9FFF77FFF0025D9E75E68C1
:10092000FFF757FF063E14308642D2D309E010F19C
:10093000140F04D3FFF74DFF8642FBD9EBE74FF0CE
:10094000FF3600233B603046BDE8F041FFF744BF6F
:1009500023681A682260C3F80480C3F80880DA6844
:1009600018699047B5E700BF140400201C0400205C
:10097000144B1A6882420AD112681A6012B1506888
:10098000063801E04FF0FF30FFF726BF13461A6824
:1009900022B19042FAD102681A6070470A4A13687D
:1009A0001BB1984203D01A46F9E7084A05E00368EC
:1009B000136070479842FAD01A461368002BF9D199
:1009C000704700BF1C0400201004002020040020F9
:1009D00008B500231846054A054900F0E5FE4FF02A
:1009E000FF30BDE80840FFF7F7BE00BFA9080008C8
:1009F00040420F0070B5084EFFF7EBFE3468054625
:100A0000FFF7E7FE8542F7D800222346141843F18A
:100A100000052046294670BD18040020F8B504469C
:100A20000D46FFF7D6FE002385420646236010D30D
:100A3000A5F10A0383420CD20A35FFF7CAFE8542AC
:100A4000FBD3FFF7C6FE8542FBD8E36820699847D1
:100A50003EE0FFF705FD63680746002B34D1A3682D
:100A6000002B31D11B4B65601A681B68B54238BF3B
:100A70000132A260A2689A4203D92046FFF7B6FE6F
:100A80001EE0B54202D9144B19460EE0134A136812
:100A900023B159688D4201D31A46F8E723601460E8
:100AA0000EE05068854203D313461A68002AF8D135
:100AB00022601C600B689C4202D1A81FFFF78CFECD
:100AC0003846FFF7D5FC03E02046FFF751FFC9E7A2
:100AD0000020F8BD180400201C0400201004002091
:100AE00038B50446FFF7BCFC6368054633B9A36814
:100AF00023B92846BDE83840FFF7BABC2046FFF7C7
:100B000037FFF6E7C36870B504460D46C3B1FFF77B
:100B1000E7FF092D0CD8FFF75CFE0646FFF759FEEC
:100B2000801B8542FAD8E3682069BDE87040184709
:100B3000FFF74FFE29182046BDE87040FFF76EBF53
:100B400070BD00002DE9F04704460E4690461AB9E4
:100B5000BDE8F047FFF7D6BFFFF782FC63680746A2
:100B6000E3B9A368D3B9DFF83CA0FFF732FEDAF8A7
:100B700000508146FFF72DFE8145F6D8304408EB42
:100B80000502864288BF01326060A2602046FFF7FE
:100B90002DFE3846BDE8F047FFF76ABC2046FFF758
:100BA000E7FEE0E71804002008B50121094800F03D
:100BB0009BFC0121084800F097FC0121074800F048
:100BC00093FC0121064800F08FFCBDE8084000F0CE
:100BD00021B900BF0D0C02400C0C02400E0C02406B
:100BE0000F0C02407047000008B50F4B1A680C4606
:100BF0009AB9012203281A6003D171460B480FF0FD
:100C0000B3F821460A480FF0AFF800F04FF9094851
:100C10000FF0AAF808480FF0A7F8FFF721FCFFF73C
:100C2000E1FFFFF7B1FD00BF2404002037190108E0
:100C30003B190108631901085719010808B501F0AB
:100C4000BDF803480FF090F800F0BCFE002008BD8E
:100C50006519010808B500F00BF9FCE71FB5FFF7AF
:100C6000FFFB0E4B0E481B68029300240D4B0093B4
:100C70000F220C234FF48071019400F055F80A4BB9
:100C80000A481B6802930A4B009307220C234FF477
:100C9000C061019400F048F8FFF7BAFB1802002089
:100CA00028040020550C00081C0200202805002004
:100CB0003D0C000808B5FFF7D3FB094B1B681A79F8
:100CC000082A07D95A79074B53F8221011B109683D
:100CD00043F82210FFF7CCFBBDE80840FFF79CBBB0
:100CE000000300200803002038B50B79082B03D936
:100CF00008490320FFF778FF4C7901F108020368E7
:100D00002BB113F8035CAC4201D31846F7E78B60B4
:100D1000026038BD25190108031F53F8042F9A42B9
:100D2000FBD0181A704700000F2A2DE9F74F05462F
:100D30008B4691469A462AD810F003031BBFC3F195
:100D40000403ED180B46CB1A303B23F003031AF0D3
:100D5000080F05EB030405D02A46A24203D2126015
:100D60000432FAE72D600193FFF77AFB2749019BD4
:100D70008046012251F8227016B25FB10132212A59
:100D8000F8D14046FFF774FB6FF08A003BE06FF04C
:100D9000150038E01D490C9841F822402A46E680AB
:100DA0000D99FFF7E3FA0E9B194AA3624FF0FF3348
:100DB000E3611368206001331AF0010F6562C4F823
:100DC0002CB084F805902771A760E7602761676100
:100DD000A7612762136004D001212046FFF746FA7D
:100DE0000DE00A212046FFF741FA1AF0040F06D160
:100DF0004046FFF73DFB4846FFF778FA02E04046E1
:100E0000FFF736FB304603B0BDE8F08F4803002003
:100E10000403002008B501F043FA00F0B9F8BDE87A
:100E2000084000F01CB838B50446043000F01BFD43
:100E30000546204601F034F8284638BDF8B504468A
:100E40000E461746051D3A463146284600F0F6FC88
:100E500020B90121204600F0F3FFF4E7F8BD08B502
:100E6000002000F01BFA0120BDE8084000F016BA8F
:100E7000F8B50D4B1E68C6F307221D4622B9F4B221
:100E8000003418BF012400E00224FFF7E9FA2B68C0
:100E90009E42074602D12046FFF73EFC3846BDE899
:100EA000F840FFF7E5BA00BF200200202DE9F04F1F
:100EB0002C4B2D4A1B882D492D482E4EDFF8CCB0E7
:100EC0008BB00DF1280906F1800A29F8043D0EF0D7
:100ED0004BFFFFF781FA0546FFF796FA0446FFF746
:100EE0008FFA2A46009023464FF4007122480EF0F4
:100EF0003BFF25EAE5754FF4007856F8044B14B330
:100F00002779E26A5BF82730606A0793904406927B
:100F1000FFF702FF069AB4F90610079B101A226821
:100F20000592626A04920390E26A029262790192E7
:100F3000082FD4BF4F4609F1010700970544A26A64
:100F40000E480EF011FFB245D7D10D4B02958DE83A
:100F500008010C4A0C4819460EF006FF0BB0BDE81C
:100F6000F08F00BFBD190108EC190108F219010842
:100F7000F71901084C0300203F1A0108891A0108DB
:100F8000C51A0108C71A0108CB1A0108C0190108BF
:100F900038B5FFF765FA1B4C0023E360054600F007
:100FA00037F84FF41443A360A268164B12F00C0FED
:100FB000FAD1154A40F20571116081221A601A684F
:100FC00042F480321A601A6812F4003F0D4AFAD0D7
:100FD0000E4B5360136843F0807313601168094B24
:100FE0008901FBD59A6842F002029A609A6802F081
:100FF0000C02082AFAD100F017F82846BDE838405C
:10100000FFF736BA00380240003C0240042A40078D
:10101000044B1A6842F001021A601A689207FCD564
:10102000704700BF00380240044B9A6812F00C0F62
:101030001EBF1A6822F001021A6070470038024091
:10104000034B044A00280CBF10461846704700BFE7
:1010500000BD010580DE800204281CD8DFE800F016
:1010600003080D1217000D4B1A6C1143196412E09E
:101070000A4A536C194351640DE0084A136B194333
:10108000116308E0054A536B1943516303E0034AB7
:10109000936B19439163BFF34F8F70470038024041
:1010A000042821D8DFE800F003090F151B000F4AC0
:1010B000136C23EA0101116470470C4A536C23EA54
:1010C000010151647047094A136B23EA010111635E
:1010D0007047064A536B23EA010151637047034A84
:1010E000936B23EA01019163704700BF003802400F
:1010F00038B514230C4A4343D4582568AA0608D5AA
:101100000A4B616803EBC002C9B253F83030506833
:1011100098472B0748BF6368054B1B681BB1BDE8A8
:101120003840FFF7C7BD38BD441B0108280B00201D
:10113000F802002001282DE9F04780460D461746A9
:1011400003D92B490320FFF74FFDDFF8B090294A60
:10115000142404FB009442F83070E66802EBC002ED
:1011600001215360304600F0BFF9304600F080FAAC
:101170003046617C00F054FA4E464FB1D4F80890E6
:101180000021484600F0B0F9217C484600F048FABA
:10119000142303FB08F806EB080999F812A0D9F804
:1011A00004105046FFF758FF56F808400023E3604C
:1011B000504623616361FFF743FFB0FBF5F080B257
:1011C000A06077B199F8133001215AB203F01F03E0
:1011D00001FA03F35209084941F8223042F22C0384
:1011E00001E042F20803E3600020BDE8F08700BFA1
:1011F00025190108280B002000E100E0441B01082C
:10120000012838B505D80E4C14230A4403FB0043CB
:1012100009E00C490320FFF7E7FC25682D06FCD503
:1012200011F8015B65608A4201D01C68F5E7142360
:101230005843034B1A5813685B06FCD538BD00BFF2
:10124000441B0108251901080020FFF751BF0120A8
:10125000FFF74EBFF8B5104C04EB4014012167684E
:10126000384600F041F9A6680021304600F03CF90C
:10127000E5680121284600F037F9247D38462146EB
:1012800000F0CEF92146304600F0CAF92146284642
:10129000BDE8F84000F0C4B9781B010801282DE929
:1012A000F041044603D910490320FFF79DFC0F4B82
:1012B000DFF83C80002543F820506401FFF7CAFFA7
:1012C00008EB04031E7F9F6930463946FFF7C4FED2
:1012D00058F8043039461D603046DD615D60BDE878
:1012E000F041FFF7DDBE00BF25190108380B0020D3
:1012F000781B0108012870B50C4621D84A1C22D061
:1013000021F0FF0313F5807F11D114F0FF041AD1EF
:101310000E4B03EB40152E69731C14D0012130468F
:1013200000F0E2F8297D304600F07AF906E001216C
:10133000204600F0D9F8204600F09AF9002070BD50
:101340004FF0FF3070BD6FF0010070BD781B0108D9
:10135000042B2DE9F84304460E461546984603D95A
:1013600017490320FFF740FC1648DFF8609067013B
:10137000012100EB840000F063FD09EB07031C7FF3
:1013800099692046FFF768FE0F4B59F8071004EBE8
:1013900084041C4416F5807F14F8082045EAC20531
:1013A00045F004050D6015BF0B684B6843F44073AE
:1013B00043F0040314BF0B604B600020BDE8F883CA
:1013C00025190108380B00206C1B0108781B010847
:1013D0000B4A430110B50446D018D3588169007FE9
:1013E00000221A605A6822F004025A60FFF758FE81
:1013F000044800EB8400BDE8104000F051BD00BF80
:10140000781B0108380B00202DE9F843089E099F3E
:10141000884691461D4623B91EB931490320FFF77E
:10142000E3FB304B400118F5807F1C58236843F0E4
:101430004003236005D0B8F1FF3F02D0404600F0E2
:1014400020F9A6B92F44AF4206D0A3689E07FCD569
:1014500015F8013B2373F6E7A3689807FCD5A3684A
:101460001906FCD4A368DA0720D5E368FAE70DB1C2
:10147000002319E030463744B84217D0A3689B07D1
:10148000FCD52573A368DE07FCD5237B00F8013B60
:10149000F2E7A2689007FCD5EA5C2273A268D10744
:1014A000FCD5227BF2540133BB42F2D1A3689A07E8
:1014B000FCD5A3681B06FCD4B9F1000F0ED1B8F11E
:1014C000FF3F0BD0236818F5807F23F04003236093
:1014D00004D04046BDE8F84300F0CAB8BDE8F88340
:1014E00025190108781B0108F8B50D460126C0F33F
:1014F000832120F00F0400F00F0706FA01F102200B
:10150000FFF7AAFD07FA06F00323216883406FEA7C
:10151000030C01EA0C012160216805F0030E0EFAAC
:1015200000FE4EEA01012160E2680CEA0202E2607C
:10153000E168C5F3810282400A43E2606268BE400E
:1015400022EA060666606268C5F30015BD401543D1
:101550006560A2681343A3600020F8BD2DE9F04147
:1015600000F00F0415462B4A42F8343002EBC40257
:10157000069B536006468846C0F383274FF480419C
:101580000120FFF769FD41463046FFF7ADFF042C0F
:10159000214B03DCA11D01228A4003E0092C03DC5E
:1015A0004FF400021A6002E04FF480725A601B4B45
:1015B0000120996800FA04F2D243114099609968B9
:1015C00005EA000E0EFA04FE4EEA01019960D968A0
:1015D0000A40DA60C540DA68A54004F00C0404F162
:1015E000804404F59C341543DD6006F00302A568D1
:1015F00092000F21914025EA0101A160A168974066
:10160000B0400F43A76058611A681043186000206B
:10161000BDE8F081400B002000E100E0003C01400B
:1016200020F00F0300F00F02F0B51E6857000325ED
:10163000BD4026EA05051D601D680224072A04FA3C
:1016400007F444EA050494BF002201221C6003EB66
:10165000820300F007001C6A80000F22824024EA07
:1016600002021A621A6A814041EA02001862F0BD61
:1016700020F00F02012300F00F0003FA00F0906148
:10168000704720F00F0200F00F001030012303FA22
:1016900000F0906170470000104B2DE9F0415E6949
:1016A0001A680F4F164000244FF001081D4608FA33
:1016B00004F31E4206D06B6107EBC40357F83420D5
:1016C000586890470134102CF1D1064B1B681BB1B0
:1016D000BDE8F041FFF7EEBABDE8F081003C014003
:1016E000400B0020F80200202DE9F843124ADFF8F1
:1016F000508003010746D5582E69EB6800241E4030
:1017000008EBC0090223A3401E4209D0EA68D9F8B9
:10171000040022EA0303EB60214658F8373098476B
:101720000134042CEED1054B1B681BB1BDE8F84316
:10173000FFF7C0BABDE8F883B81B0108F802002023
:10174000C00B0020032910B516D80D4B00011C1842
:101750001B586068024001F10C0003EB80004260FE
:101760001869022202FA01F120EA01021A61DA681C
:101770001143D960002010BD4FF0FF3010BD00BFF5
:10178000B81B01080001024B1B58586A704700BF84
:10179000B81B0108034B00011A58136843F00103FA
:1017A00013607047B81B010801282DE9F84305466E
:1017B000884630D81A4E1B490401371941F83020A9
:1017C00097F80C9001EBC00148464B60B968FFF7F1
:1017D00043FC36597B680024346048467460F362E9
:1017E000FFF72EFC104B7A7B13F809305843B0FBFF
:1017F000F8F3013BB36251B2012302F01F0273619F
:1018000049099340094A284642F82130FFF7C2FFB0
:101810002046BDE8F8834FF0FF30BDE8F88300BFF5
:10182000B81B0108C00B0020D81B010800E100E034
:101830000020FFF759BF0120FFF756BF70B51346D0
:101840007BB18568C468A5420BD084680668651CB6
:1018500085604568013D2C40013B345D01F8014B3A
:10186000EEE7D01A70BDC368426830B584681B1BB0
:10187000934208D0C3680468013A5D1C1340C560F8
:10188000E154002030BD4FF0FF3030BD07B50549B1
:10189000054800F031FA684600F0EBFC019800F0D2
:1018A000EBF9F8E7D01E0020B01E002000B58FB085
:1018B0001822002108A80EF04FF90423089340F2E3
:1018C000D243ADF83630BA238DF82430AD238DF8ED
:1018D0002530A5238DF8263055238DF82730172382
:1018E0008DF832302A238DF8333003A800F0C1FC84
:1018F0000EA9049B41F8303D042208AB0D4807F0C7
:1019000055FC002802DA0C480EF0B8FA00230093C8
:101910000A220A4B074805A907F0DAFB002804DA77
:1019200074300CBF0648074800E007480EF0A6FADE
:10193000DBE700BFD00B0020F41B010840420F0082
:101940000A1C0108131C01082B1C010810B51749BB
:10195000174840F2D243CB8200238CB01A4607F0DE
:1019600061FB00281CDB06AC4FF0FF33042203A907
:1019700000940F4807F0ACFB234605220D490C48A4
:1019800007F014FC002802DA0B480EF077FA039BEC
:1019900005930A4B04A8B3F9001000F0C5FBE2E779
:1019A00007480EF06BFA00200CB010BD3402002086
:1019B000D00B0020611C0108661C0108AE1E00202F
:1019C000491C010810B50821AEB0554800F054FC80
:1019D00054480EF053FA102200210AA80EF0BCF869
:1019E000102200210EA80EF0B7F807A803F028FC7B
:1019F000BA238DF82830AD238DF82930A5238DF832
:101A00002A3055238DF82B3008230093002208AB91
:101A10000221BDF91C0003F0FFF90028A4BF9DF8C6
:101A200020308DF836304FF08002A4BF9DF8213071
:101A30008DF837300AA90EA80DF090FF0023402240
:101A40000AA9BDF91C0001F097FD9DF83630172B4F
:101A50005AD19DF83720322A22D18DF846302A23D8
:101A60008DF847304FF0FF33002404932E4ABDF920
:101A70001C100192102302930EAA039400942B4889
:101A800000F078FD2A4B02932A4B009308231A4654
:101A900001944FF4C0612848FFF746F9274B31E025
:101AA0002A2A31D18DF8463032238DF847304FF055
:101AB000FF3300240493224ABDF91C100192102325
:101AC00002930EAA03940094184800F053FD1D4B96
:101AD00002931D4B0093062208234FF4C06101942A
:101AE0001A48FFF721F91A4B18801A4B02931A4B28
:101AF00000930194082305224FF4C0611748FFF7B3
:101B000013F9174B188002E016480EF0B7F9164883
:101B10000EF0B4F980220EA9144808F097F900BF1E
:101B20006C1200207A1C010824020020842300206B
:101B3000A11C0108AD180008AC180020F01E002000
:101B40004C020020B41C01084D1900086C0C002048
:101B5000AC1E0020C71C01088D180008AC12002024
:101B6000AE1E0020D41C0108DE1C0108DC1B01088D
:101B7000014808F059B800BFD01E0020014808F005
:101B800053B800BFB01E00200128F7B504460D462B
:101B900002DC09682D4829E02D4968680EF064FAD6
:101BA0000646C8B9042C02DC29682A481EE02A49E6
:101BB000A8680EF059FA18B9002466F307042BE060
:101BC0002649A8680EF050FA10B90024012321E03C
:101BD00023480EF053F90BE0224968680EF044FAEE
:101BE000064660BB042C05DC29681F480EF0BCF8D3
:101BF000012628E01D49A8680EF036FA10B9002425
:101C0000022307E01A49A8680EF02EFA0028DFD157
:101C10000024032363F30704E8680DF0F5FB07468F
:101C200028690DF0F1FB67F31F4460F30F24114B9B
:101C30000194B3F90010684600F076FA03E0084812
:101C40000EF01CF90026304603B0F0BD231D01083C
:101C50003A1D01083F1D01088C1D0108941D010853
:101C60009C1D0108B31D0108B81D0108001E0108D4
:101C7000061E0108F01E002010F0FF0310B50446F8
:101C80000BD1C0F3072007F0D9FF220C03461849F7
:101C90001848BDE8104008F024B8012B0BD1C0F360
:101CA000072007F0CBFF220C034611491148BDE87D
:101CB000104008F037B8022B0BD1C0F3072007F013
:101CC000BDFF220C03460A490A48BDE8104008F04F
:101CD0004CB8032B0BD1C0F3072007F0AFFF220C49
:101CE000034603490348BDE8104008F060B810BD42
:101CF000D01E0020B01E0020F0B5224B224F234EF4
:101D0000234885B0002201248DE8880003940296C0
:101D1000023B114607F052FF002804DA1D480EF07E
:101D2000ADF801202BE0022303931B4B1B4D0093C6
:101D300002950197023B22460021194807F03EFF19
:101D40000028EBDB17480EF099F80096164B224658
:101D500000213046FFF702FC002801DA1348DEE7D5
:101D60000095134B224600212846FFF7F7FB002879
:101D700001DA1048D3E710480EF080F8002005B0D3
:101D8000F0BD00BF02100240040C024008000240F7
:101D9000B01E00200B1E0108031002400900024083
:101DA000D01E00202B1E01087D1B0008431E0108C9
:101DB000711B00087E1E0108B91E010808B500202D
:101DC00007F0CEFEFEF704FE03F066FC03F048FECB
:101DD00005F0D2FA01F034F807F08EFB00F006F8B7
:101DE00001F050FDBDE8084003F058BE13B50E4C9D
:101DF0000E490F480BF0A6F80D49204603F060F994
:101E0000002806DA0B48002102B0BDE810400DF0B2
:101E1000ABBF0094084B094802224FF4806103F0E5
:101E2000E5F902B010BD00BF4C230020E41E0108FC
:101E3000F4220020FC1E0108361F0108F21E0020BB
:101E400070B505460C46FEF70BFB2B6806462BB912
:101E50004FF0FF332B60FEF70BFB18E0CCB10F4BBC
:101E60001C6802212046FEF701FA2B68013305D1D8
:101E700004F108032B600023A36003E021462846F9
:101E8000FEF732FF3046FEF7F3FAFEF7C5FA0120FF
:101E900070BDFEF7EDFA204670BD00BF00030020C4
:101EA00070B50446FEF7DCFA256806461DB16B1CCA
:101EB00005D100232360BDE87040FEF7D9BA28465B
:101EC0000A2150F808392360FEF7D0F9236813B9C6
:101ED0004FF0FF33236015F8034C3046FEF7C8FA85
:101EE0002046BDE87040FEF701BA0000F8B505468F
:101EF0000E46FEF7B5FA364B364A1B881BB207462C
:101F000052F82320D2F820E0BEF1000F1AD0546915
:101F10009369A34216D9631C5361D3691C4046B927
:101F2000136933B9631C04D13846FEF7A1FA204681
:101F3000F8BD002C0ADB0EEBC40393E8030085E830
:101F4000030004E04FF0FF34002EE9D0D56016699D
:101F500076B333681361002C0CDB95695169D36942
:101F6000691A8B42A9BF691C4FF0FF351D40916172
:101F70000EEBC505736893E8030085E8030016F8C7
:101F8000043C052B09D0002373600A21A6F1080048
:101F9000FEF76CF916F8034C00E00F243846FEF704
:101FA00067FA0E2C02D82046FEF7A0F90120F8BDF2
:101FB000002C09DA10460321FEF758F93846FEF7DF
:101FC00057FAFEF729FAF1E73846FEF751FAEDE73E
:101FD000FC0200204803002010B583694469C269EF
:101FE0001C1BA24201DA002010BD5C1C134084615E
:101FF000F9D4026A03C902EBC30383E8030001209A
:1020000010BD00002DE9F8431E46264B53F8215021
:10201000254B1B880380074691462DB93046FEF7B5
:1020200027FA4FF0FF3439E02B79032B28D01F4BD0
:1020300001462846D3F80080FFF7CEFF044638B1AA
:102040003046FEF715FA98F80430052B25D122E02A
:10205000B9F1000F03D13046FEF70AFA1EE098F8F6
:102060000430C8F80C70052B0CBF05210421404634
:10207000FEF7FCF8414605F11000FEF735FE07E0DB
:1020800003C8EB6883E803000A212846FEF7EEF850
:102090003046FEF7EDF9FEF7BFF901242046BDE812
:1020A000F88300BF48030020FC020020000300204A
:1020B00038B50446FEF7D4F9074B1B882380074B3D
:1020C000214605461868FFF787FF04462846FEF7B5
:1020D000CFF9204638BD00BFFC02002000030020DD
:1020E00008B50F4B53F82130B3B1212202801A7981
:1020F000032A0BD103C8DA6882E8030018460A21D4
:10210000FEF7B4F8074B0120186008BD01461846D9
:10211000BDE80840FFF760BF4FF0FF3008BD00BFCB
:1021200048030020F802002070B504460D46FEF773
:10213000A2F928B129462046BDE87040FFF7D0BF7C
:10214000094B1B881BB29D4204D12046BDE870405C
:10215000FFF7AEBFFEF784F9294603460122204669
:10216000BDE87040FFF74EBFFC02002070B504468A
:102170000D46FEF780F9064628B129462046BDE8FF
:102180007040FFF7ADBF0A4B1B881BB29D4204D1C4
:102190002046BDE87040FFF78BBFFEF761F932467D
:1021A000034629462046BDE87040FFF72BBF00BF1D
:1021B000FC0200202DE9F041124F3B881BB29342F4
:1021C00006460C46154603D10F490320FEF70CFDC9
:1021D000FEF746F93A880D4B12B2804653F822704A
:1021E00005213846FEF742F896E80300FC604346B6
:1021F00084E80300012229462046BDE8F041FFF7AC
:1022000001BF00BFFC02002025190108480300207F
:1022100070B504460D46FEF723F9B4F90020114BC2
:1022200053F8224006461CB90F490320FEF7DCFC98
:102230002379052B04D0FEF71BF94FF0FF3070BD5A
:1022400095E80300E36883E803000A212046FEF7CF
:102250000DF864793046FEF70BF92046FEF746F894
:10226000012070BD48030020251901080021FFF757
:102270003DBE0121FFF73ABE08B5074B4A1E1B6859
:102280001140186203D005490320FEF7ADFC5961E7
:102290009961DA6108BD00BF00030020251901081B
:1022A0000F4BD3F8882042F47002C3F888200D4AFF
:1022B0009A60102283F822200021DA7701F1604031
:1022C00000F561400131522980F80023F6D11A69E6
:1022D00042F010021A615A6942F400725A61704762
:1022E00000ED00E0000000080121FFF7A9BD10B5D6
:1022F0000446406908B10AF0F1FCE06908B10AF04F
:10230000EDFC00200022002360612061E061A061FB
:102310002080C4E9022310BDFEF76CBB2DE9F04F0D
:1023200089B08A4615469B460446FFF7F5FFCDE97E
:102330000401EB000393079355445346AB4205D089
:1023400013F8012B002AF9D0002300E00123002715
:1023500002936FF075030193B846B9463E46A268F2
:10236000974270D222687D0102EB050EDEE9020180
:10237000002908BFB0F1FF3F23D0DDE904239942D3
:1023800008BF90421DD200220023CEE9022322681A
:102390002A44166122682A449661226856532268AC
:1023A0002A44506920B10AF099FC22682A445661F7
:1023B00022682A44D06920B10AF090FC22682A449D
:1023C000D661039B98453CD222682A445069002874
:1023D00037D007AA51460AF0B7FC38B923681D4424
:1023E000129BCBF800500120186034E0029B13B11F
:1023F00002282DD1F2E7012814D122681544296959
:1024000011F07F4F1BD0079AB2EB116F17D3B8F1C1
:10241000000F01D0904512D20023CBF80050904617
:1024200001930AE002280AD1B8F1000F07D122680F
:10243000CDF804801544CBF800504FF00109039B00
:10244000079301378BE7129B0198C3F8009002E0D5
:102450000128F4D1D1E709B0BDE8F08F38B50546C1
:102460000C46FFF759FF4FF47A736B43C01841F1E4
:102470000001C4E9000138BD2DE9F04788B0972973
:1024800090461BBF109A0792424605AA8A461CBF77
:10249000CDF814808DF81830ADF806100292DF00E8
:1024A00000F1120500F1200600F11C046FF0010993
:1024B00035F9023FDBB1BAF1970F03D000976A46B6
:1024C000414607E0D8F8183019684B78DB000093D4
:1024D0006A46023130680AF037FC023007D0B5F99D
:1024E000002003A901A8FFF765FE4FF00009A542EF
:1024F00006F10406DCD1484608B0BDE8F0870000CC
:1025000030B587B006AA102302AD294642F8143D23
:102510000AF0FCFBA842014620D1019B102B08D1F8
:1025200028220F4807F0E8F901460E480DF01CFC80
:1025300014E00024019BA34204D3295D0A480DF056
:1025400013FC02E009480DF00FFC0134102CF1D10E
:10255000072407480DF008FC013CFAD107B030BD54
:102560005C230020401F0108461F0108142E0108AB
:10257000152E01082DE9F04F00F10C0787B0044635
:1025800038469A468B469046149EFFF7ADFE0123CF
:102590000493B8F1000F01D0119B2BB93846FFF717
:1025A0007FFC6FF00D006AE004AB0093524605AB70
:1025B00041462046FFF7B2FE012802D04FF0000945
:1025C0001CE012991198059C0AF026FB054610B9EB
:1025D0006FF00B044FE0E0690AF080FB139BE561AC
:1025E000721CA36102D004F1080139E04FF0FF3200
:1025F0000023C4E902233DE009F10109A2689145E5
:10260000E6D222684FEA49152A44D2E9020150EA8B
:102610000103F1D15146404603920AF0FDFA039AB4
:10262000506122682A44516971B1109B136122687C
:10263000129911982A4403920AF0EEFA039A139B16
:10264000D06122682A44936122682A44D169002912
:10265000D2D0A2F800B0731C216805D029440831FB
:102660003046FFF7FBFE05E00D444FF0FF3200233C
:10267000C5E9022300243846FFF712FC204607B0C4
:10268000BDE8F08F2DE9F04300F10C0585B004465C
:1026900028461F46884691460E9EFFF725FE0123D9
:1026A0000293B8F1000F00D02FB92846FFF7F8FBCE
:1026B0006FF00D002CE002AB00934A4603AB41469D
:1026C0002046FFF72BFE012802D06FF00B041BE021
:1026D00038460C99039C0AF09FFA07460028F4D06C
:1026E000E0690AF0FBFA0D9BA361731CE76105D05A
:1026F00004F108013046FFF7B1FE04E04FF0FF326D
:102700000023C4E9022300242846FFF7C9FB204622
:1027100005B0BDE8F083F0B500F10C0485B00546C6
:1027200020460E461746FFF7DFFD0123029302AB5A
:1027300000933A4603AB31462846FFF7EFFD0128E8
:1027400002D10398FFF7D3FD2046FFF7A9FB05B0A0
:10275000F0BDF8B500F10C06054630460F46FFF710
:10276000C3FD0024AB689C420AD22868630117B1FC
:10277000C25EBA4202D11844FFF7B9FD0134F1E755
:102780003046BDE8F840FFF78BBB2DE9F04F00F174
:102790000C0485B0054620469B46894692460F9E0E
:1027A000FFF7A2FD01230293B9F1000F04D0BBF1A2
:1027B000000F01D00E9B2BB92046FFF771FB6FF085
:1027C000150049E016B1BAF1000F05D12046FFF718
:1027D00067FB6FF00D003FE002AF009703AB109A6C
:1027E00031462846FFF79AFD0128804615D9119BEE
:1027F00000933246109B99212846FFF73DFE48B9C9
:1028000001230293009703AB109A31462846FFF745
:1028100085FD8046B8F1010F0CD8039B5A465146FE
:10282000D8690AF073FA58B92046FFF739FB6FF000
:10283000680011E02046FFF733FB6FF075000BE0F6
:10284000039BB3F90020A9F800200E9A9B6913603E
:102850002046FFF725FB002005B0BDE8F08FF8B556
:102860000646002546F80C5F04463046FFF73CFD5F
:1028700004F1120204F11C0304F1300122F8025F9A
:1028800043F8045F8B424FF00007F7D123792761AB
:10289000022BA2680BD123685201394618680DF04B
:1028A0005BF923689A685868D200394602E02068CC
:1028B000520139460DF050F90AF0A8FA3046BDE849
:1028C000F840FFF7EDBA00002DE9F04F044600F1A3
:1028D0000C0585B02846FFF707FDFFF71DFD23799E
:1028E000012B804689466AD1674A684B6849694826
:1028F0008DE80C00684B0DF037FA4FF0000BA36821
:102900009B456BD221684FEA4B1A5144D1E902230F
:10291000134351D04869FFF7F3FD23685F485344E0
:1029200019690DF021FA23685344196911F07F4F9A
:1029300004D0090E5A480DF017FA02E059480DF07C
:1029400013FA23685344D869FFF7DAFD2368534824
:10295000534499690DF008FA23685344D3E9026798
:10296000002F08BFB6F1FF3F1CD0B6EB080667EB9F
:102970000907002E77F1000301DA4B4913E03046D6
:1029800039464A4A00230CF0B3FB00230392304639
:10299000464A39460CF0ACFB039A014644480DF018
:1029A000E3F903E0434944480DF0DEF92368434866
:1029B00033F90A100DF0D8F90BF1010B9FE7022B48
:1029C0000CD1324B00933E4A3E4B3F493F480DF0FD
:1029D000CBF94FF0000BA3689B4505D3284605B003
:1029E000BDE8F04FFFF75CBA236819684FEA4B1A4D
:1029F0005144D1E90223134343D08B691868FFF790
:102A00007FFD23681B6853445B691868FFF778FDF6
:102A100023682F481B68534419690DF0A5F92368F2
:102A20001B685344D3E90267002F08BFB6F1FF3F8C
:102A30001CD0B6EB080667EB0907002E77F1000300
:102A400001DA194913E030463946184A00230CF0E0
:102A50004FFB002303923046144A39460CF048FBE2
:102A6000039A014612480DF07FF903E0114912481C
:102A70000DF07AF9236811481B6833F90A100DF03C
:102A800073F90BF1010BA6E7882001084320010828
:102A90009E2001081A200108112001084B2001087E
:102AA000552001085E2001086620010840420F0001
:102AB000752001087F2001086E2001086A1F0108A7
:102AC0008E200108852001089B200108AA2001080A
:102AD000CC200108034600201BB1DA685B68104473
:102AE000FAE7704710B50822094904460CF004FFC4
:102AF00048B12378FF2B08D1607800F00F00831EC7
:102B00005842584110BD012010BD002010BD00BF2B
:102B10009E220108002102F0CDBE38B5CBB20021C3
:102B200014460246084602F0A1FB054618B92046A5
:102B3000FFF7F0FF0FE094F9103001330AD1A368DA
:102B400082681B7903F03F0321462046137102F08F
:102B500071FC04466C60284638BD00002DE9F04742
:102B60008C680746104688461546FFF7B3FFA379E1
:102B700040BAFF2BA0800AD12B7C023BDBB2022B98
:102B800003D8214AD35CFF2B00D13B23A371E37907
:102B900043B90FB9402304E0384600F0CFFC90F869
:102BA000CA31E37104F108061022184930460CF0CE
:102BB000A3FE8246D0B904F11809154910224846EF
:102BC0000CF09AFE014630B9102230460CF0C4FFDA
:102BD0000123E3750AE049465246384600F088FD75
:102BE000014618B1102230460CF0B8FE4146284686
:102BF00002F0DAFB002804DA831C08BF0020BDE8DD
:102C0000F0870020BDE8F087DB200108EE220108F4
:102C1000FE2201088B6870B558800C46054600F00E
:102C20008DFC014618B919490320FDF7DDFF6668E0
:102C30003046FFF74FFFB1F8C831984204D920461B
:102C4000BDE87040FFF766BFD1F81C320133C1F810
:102C50001C323046FFF73EFFD1F824321844B1F859
:102C6000C631C1F82402DB0708D5234640F2022210
:102C70000749012002F07CF830B9E0E721462846F8
:102C800002F0AFF80028DADD70BD00BF2519010899
:102C90000000FFFF2DE9F04F85B090F910300133AF
:102CA00000AF044689460AD18368B3F9026002F096
:102CB0000FFE00286AD043680446984601E080462B
:102CC0000026404602F004FE054600285ED044453A
:102CD000836818BF60601A461B7ED0F8048008BF66
:102CE0000446FF2B2BD186B907F1080002F0A8FAA1
:102CF00000284BD0002122460846B7F90860FFF7AC
:102D00000CFF0446002800F09380B9F1000F06D0B4
:102D1000424629463046FFF721FF002836DBA268ED
:102D2000137943F040031371304600F05FFE4368AF
:102D30000133436021463046FFF76CFF78E01346CD
:102D4000183310223C4918469B460CF0D5FD40B183
:102D50005946002E39D1381D00F06EFC0646002879
:102D600038D0B9F1000F06D0424629463046FFF769
:102D7000F5FE00280ADB2846FFF7ACFE00210246DC
:102D80000223084602F0A4FC064608B9204619E0D2
:102D900083689846EA68A96840460CF0DFFDEB6856
:102DA0006D6842461A449046002DF3D12046FFF745
:102DB000B1FE224B3146B3F9000002F01FF80028A3
:102DC00036DC3046FFF7A6FE32E0304600F00CFC61
:102DD0000028C6D107F11001082301F80D3D324645
:102DE0005B4607F1080005F06FFDEA46064640B174
:102DF000B9F1000F09D042462946FFF7AFFE00287F
:102E000003DA2046FFF786FE11E02246F97807F143
:102E10000800FFF782FE044648B1304600F0E6FDA8
:102E200003680133036021463046FFF7F3FED546C1
:102E30001437BD46BDE8F08FFE220108B8230020FC
:102E40001FB50F4CB4F9003063B90E4A01930E4B15
:102E500002920093042208234FF480610B48FDF78F
:102E600063FF20800A480B4B036001230371142386
:102E70008360FFF7F4FCB4F9000004B010BD00BF9C
:102E8000B8230020D620010839310008BA230020D9
:102E900084230020C0270020292B2DE9F8438146F8
:102EA0000F4614461D4606D03A2B06D0112B0CBFF8
:102EB0000423002302E0022300E00323292D3B74B6
:102EC00001D03A2D03D1A74259D1012605E0A742EE
:102ED00002D063689F4252D100267B6893F91000AC
:102EE000022805D016B30121204602F0D1FC1DE0D6
:102EF000294602F03DFA18B986F0010836B101E022
:102F00004FF000080121204602F0C2FC234640F2A7
:102F100001221E4997F9100001F02AFF10B920463E
:102F2000FFF7F8FDB8F1000FDCD00AE0234640F2CD
:102F300001222946022001F01BFF10B92046FFF7AD
:102F4000E9FD06B3292D07D03A2D18D12146484670
:102F5000BDE8F8430AF0F6BF00232374616839B175
:102F600091F91030022B03D1204602F063FAF5E705
:102F7000022323742046BDE8F84300F00BB804494F
:102F80000320FDF731FEBDE8F88300BF0000FFFF1E
:102F9000251901082DE9F047044618B964490320B2
:102FA000FDF722FE4FF0FF3102F00FFA0546A0B107
:102FB0008368B3F90260002EF0D0304600F016FDB1
:102FC00043690133014643612046FFF783FDEA6808
:102FD0008B699B1A1844886100E0064627462546FF
:102FE00095F91030022B08D1EB68282B05D1AB687E
:102FF0001B7803F0F003602B08D0D5F804802F462F
:10300000B8F1000F6ED04546EAE73C46D5F8088097
:10301000E368B8F8041049BA89B2994203D220464D
:1030200002F0DEFB0FE022460023D068034492F951
:103030001000022803D1283B994204D95DE0526870
:10304000002AF2D1F7E708F1180910223949484659
:103050000CF052FC002855D04846FFF743FD494686
:1030600000B136B9002000F0E7FA002E08BF06468E
:1030700002E0304600F0B8FAB0FA80F040090028CB
:1030800040D008F10800FFF72DFDB0BB4846FFF720
:1030900029FD90BB98F80730013BDBB288F8073078
:1030A0005BB3284602F014FC38B34FF0FF312046E2
:1030B00002F08BF9014610B1204602F0BBF921461F
:1030C0000025084602F004FC18B92846FFF722FD47
:1030D00013E04168456005460029F2D1BDE8F0479C
:1030E000FFF7D8BDA3681B7803F0F003602B04D171
:1030F000204602F0EDFB074668B92046BDE8F047E0
:10310000FFF708BD98F80630224639463046BDE83C
:10311000F047FFF7C1BE0222282102F0F3FA87F838
:103120001080054600287FF470AF3846E6E700BF00
:1031300025190108FE22010810B5102298B00DEBE8
:10314000020000210CF008FD504B0593504B082164
:103150001B88ADF81C3008A8FFF78EF804A90220E0
:1031600002F0BAF840F20523ADF80A3000246846B0
:10317000FFF77FF8BDF802306FF400721344222B82
:10318000F5D801A252F823F0153200081D320008CC
:1031900027320008273200086F3100086F3100081D
:1031A0006F3100086F3100086F3100086F3100087F
:1031B0006F3100086F3100086F3100086F3100086F
:1031C0006F310008373200086F31000843320008C1
:1031D0006F3100086F3100087B3200086F31000842
:1031E0004B3200086F3100086F3100086F31000862
:1031F0006F3100086F3100086F3100086F3100082F
:103200006F310008533200085B3200086332000857
:10321000733200080198FFF7BDFEA8E7012101986D
:10322000FFF738FDA3E76FF0850302A96846039313
:10323000FEF7EEFF9BE7019A537E23F008035376D7
:1032400095E7019800F044FF91E7019800F0CEFF68
:103250008DE7019805F0B2FA89E7019805F004FBC3
:1032600085E7019B587C00F00F0004F0F1F804742E
:103270007DE7019805F05EFD79E7019A0023194684
:10328000B2F91A0001F012FB71E700BF0000FFFF66
:10329000FC0200200121FEF7D3BD2DE9F84300F523
:1032A000E075074628468846FFF7F4FF00244FF0F4
:1032B000380909FB04764146304606F0B6FA38B1C3
:1032C0001022002130460CF047FC0023337402E04A
:1032D0000134082CEDD12846BDE8F843FEF7E0BDE7
:1032E00008B5102203490CF007FBB0FA80F0400942
:1032F00008BD00BFEE22010810B5082209490446A6
:103300000CF0FAFA48B12378FF2B08D1607800F06E
:103310000F00831E5842584110BD012010BD0020EF
:1033200010BD00BF9E2201082DE9FF47002605467B
:103330008846924699463446AF194146384606F0CB
:1033400074FA00287FD13846FFF7CAFF10B1002C6D
:1033500008BF3C463836B6F5E07FEDD12746002C55
:1033600071D01022414620460CF0F8FA237884F8F8
:1033700011A0FF2B84F8109016D0B5F8C631DA07EB
:1033800012D501F0E1F8814670B105F5E0763046DE
:10339000FEF786FDB5F9C4014B464A46214601F0C9
:1033A00083F93046FFF776FF98F80030FF2B04D101
:1033B000237C43F00103237441E04046FFF79CFF68
:1033C0008146C8B9B5F8C62102F00602062A17D10F
:1033D00005F5E0763046FEF763FDB5F8C631DB074C
:1033E00006D54B464A464946B5F9C40101F05EFA96
:1033F0003046FFF74FFF03E0237C63F07F03237425
:10340000B5F8C63103F00303012B18D040F2FF22B8
:103410000023CDE900234FF080730293FF238DF842
:103420000C3098F80D308DF80D30B8F80E30ADF83E
:103430000E308022002369462846FFF775FF40F2D0
:10344000112363866463384604B0BDE8F0870388BF
:103450005BBA23F03F031B041B0C4FF6C062934280
:1034600009D00378FF2B08D1407800F00F00052821
:1034700018BF0E207047052070470E2070472DE9B9
:10348000F0470025804691461F460C462E464FF0D9
:10349000010A3FB13A780AFA05F31A421AD0237C9E
:1034A000DB0717D42046FFF71BFF98B94946204693
:1034B00006F0D0F937B999F80030FF2B02D0637CC1
:1034C000834207D8B04205D9B8F1000F01D0C8F83F
:1034D000004006460135082D04F13804D9D13046A4
:1034E000BDE8F08770B5134CB4F9C451A842064644
:1034F0001ED0EDB904F5E070FFF7CCFE4FF4A063E9
:10350000A4F8C831402384F8CA31A4F8C4612B461A
:10351000A4F8C651802208492046FFF705FF04F5AC
:10352000E070FEF7BDFC2046BDE8704000F06CBEC8
:1035300070BD00BF402A0020BE220108034BB3F932
:10354000C42182420CBF184600207047402A002048
:10355000B0F8C631DA0707D511B143F0020301E034
:1035600023F00203A0F8C6317047B0F8C631DB077C
:1035700001D505F09FBB70472DE9F0410D46174678
:103580009846FFF7DBFF044610B90020BDE8F08144
:103590000029FAD00846FFF7A3FE0028F5D1802FB6
:1035A000F3DC04F5E0763046FFF774FE43463A4616
:1035B00029462046FFF7B8FE04463046FEF770FC69
:1035C0002046BDE8F081000010B520B90548B0F9EB
:1035D000C43133B101E0FFF7B1FFBDE81040FFF7A0
:1035E0005CBE10BD402A00202DE9F8438946FFF754
:1035F000A5FF0446E8B100F5E0763046FFF74AFE45
:10360000002504EB05084946404606F00EF907463A
:1036100028B13046FEF744FC4046BDE8F883383513
:10362000B5F5E07FEDD13046FEF73AFC3846BDE80F
:10363000F883BDE8F883000038B5084C0546B4F9B6
:10364000C4011DB9FFF7D0FF20B938BDFFF7CCFF8B
:10365000286008B1B4F9C40138BD00BF402A002079
:103660002DE9F34102AD00260E4C45F8046D884665
:10367000074604F5E070FFF70DFE3346424621464B
:103680002846FFF7FCFE20B1019B3B60B4F9C44122
:1036900000E004460448FEF703FC204602B0BDE803
:1036A000F08100BF402A0020002C00202DE9F341CA
:1036B00002AC0027884644F8047DFFF73FFF00F581
:1036C000E07506462846FFF7E5FD20463B464246A4
:1036D0003146FFF7D4FE044628461CB1FEF7E0FB56
:1036E000019802E0FEF7DCFB204602B0BDE8F08165
:1036F0002DE9F04F87B00F461546FFF71FFF00F585
:10370000E073804618460193FFF7C4FD01220021B3
:1037100002A80CF021FA4646C3464FF0FF3A0024B7
:103720004FF001099BF80020FF2A12D05846FFF7FE
:10373000D7FD70B945B99DF8081009FA04F20A439B
:103740008DF80820A24604E05846FFF7D5FD002872
:10375000F1D10134082C0BF1380BE3D1BAF1FF3F62
:1037600000F0878004AD2246002128460CF0F4F9D1
:103770003B78FF2B04D197F8019009F00F0309E083
:103780003846FFF7B9FD20B93846FFF760FE0090D4
:1037900001E0022300934FF000094C469DF8081009
:1037A000012303FA04F2114232D039463046B346BF
:1037B00006F03BF8002855D13046FFF79DFD18B9BB
:1037C0003046FFF744FE00E00220009B834208D110
:1037D0002A5D0432D2B22A554A4588BF4FF0040907
:1037E0000AE009D92A5D0232D2B24A4513462A5567
:1037F00038BF4B465FFA83F9B2694AB12A5D01329C
:10380000D2B24A4513462A5538BF4B465FFA83F970
:103810000134082C06F13806C0D10122002102A88B
:103820000CF09AF900209DF80820014601246E5CF6
:103830004E4504BF04FA01F0024301F1010104BF47
:10384000D2B201200829F2D108B18DF8082006A8CB
:10385000002340F80C3D3A4602AB4146FFF70FFE0D
:10386000DDF80CB0BBF1000F05D1382202FB0A8B4A
:1038700001E04FF0000B0198FEF712FB584607B02D
:10388000BDE8F08F2DE9F04F8DB005A801F0D8FC10
:103890000026544F03900DF11205B146039B9E4242
:1038A00000F09D8035F9020FFFF748FE044600281E
:1038B00000F0918000F5E07A5046FFF7EBFC012321
:1038C000B5F90000009300220DF1130317218DF8C4
:1038D000139001F0A1FA86302CD09DF91330012B02
:1038E00028D108230DF13008ADF818304FF6FF73DA
:1038F00028F8103DB7F8C631B5F9000043F00303CE
:103900004FF0020BA7F8C631002206AB0521CDF817
:1039100000B001F0A7FAB5F90000CDF800B0112110
:103920004346002201F078FABDF82010B5F90000F6
:1039300005F04CFB4FF00808B5F90000CDF8008009
:1039400006AB0022414601F067FA00280FDB424631
:1039500006A90AA80CF002F84246234908A80BF071
:10396000FDFF0023402208A92046FFF7DDFC0223CB
:10397000B5F90000009300220DF11603112101F0AA
:103980004BFA002806DBBDF81630B3F5A06F28BF50
:10399000A4F8C83100231A462421B5F90000CDF857
:1039A000009001F039FAB4F8C6310028CCBF43F0DA
:1039B000800323F08003A4F8C6315046FEF770FA66
:1039C00001212046FFF7C4FDB4F8C631DB0702D55C
:1039D000204604F0BBFE013607F50C775EE70DB01C
:1039E000BDE8F08F402A00209E22010808B5FFF7AD
:1039F000A5FD00F5057008BD2DE9F3410746884691
:103A000016461C460AF062FC054640B903230093A3
:103A10003246A3B2414638460AF0EAFB20E0437E34
:103A200003F00703012B01D103210DE0027EA3B2B5
:103A30009A4200F110070CD031462C7622463846C7
:103A40000BF08CFF0321284602B0BDE8F04100F0E6
:103A50008FBE2246394630460BF04EFF0028EBD190
:103A600002B0BDE8F08100002DE9F04F1D46D3798A
:103A700091B0FF2B8046069116461A9F40F0B48005
:103A80006B78002B40F0B080172F40F2AD802B7A7E
:103A9000FF2B00F0A98002F1080955491022484681
:103AA0000BF02AFF70B105F108014046FFF79CFDBD
:103AB0000590002800F098800023183F1C46194606
:103AC0009A461BE00D224B4906F118000BF014FF3B
:103AD000002800F08980E6E70AF1180205EB020BE6
:103AE000AA5C012A0DD0212A08BF5C469BF8012060
:103AF0000AEBC20A1FFA8AFAA7EBC207002FEBDC17
:103B00000BE008AB2A780698009331465B4601F03B
:103B10000DF8031E68DB5946E8E740460793069117
:103B2000FFF70CFD0699079B18B933490320FDF7F1
:103B30005BF808AA002942D0002C40D0B0F8C6118A
:103B400001F0030103293AD12978029301924B46EF
:103B50000A4600943146404604F0A6FF002304F1D3
:103B600008020F21074604F085FF054617B9102209
:103B7000494620E0237A83F002038DF82830637AE7
:103B80008DF82930A37A8DF82A30E37A8DF82B301E
:103B9000237B8DF82C30637B8DF82D30A37B8DF843
:103BA0002E300822E37B8DF82F300AA90EA80BF0E7
:103BB000D5FE124908220CA80BF0D0FE09E04946B8
:103BC0004046FFF719FF102249460CA80BF0C6FE2D
:103BD0000025337E0095A3F1FF025342534105991E
:103BE0000CAA404600F0D4FC11B0BDE8F08F00BF35
:103BF000EE220108DE220108251901089E22010893
:103C00002DE9F04F89B003F1080992460591494624
:103C10001D468046129E0AF059FB9AF80730FF2B8A
:103C200040F0B5806C78002C40F0B180172E40F247
:103C3000AE802B7AFF2B00F0AA80002800F0A7802E
:103C4000183E2746002E27DD07F1180305EB030B6E
:103C5000EB5C022B0DD0212B16D100230293019394
:103C60002A78CDF800B04B465146404604F01CFF80
:103C70000AE006AB00932A7805985B46514600F0AF
:103C80009CFF041EC0F283809BF8013007EBC30742
:103C9000BFB2A6EBC306D5E74FF0FF31059801F0A0
:103CA00094FB08B1876800E00746494640460AF0A1
:103CB0000DFB064600286AD0437E03F00703022B63
:103CC00012D127B13B7813B17B78002B31D106A9F3
:103CD000A6F81A803476224606F110000BF03EFE5C
:103CE0002B79590616D512E01FB13B780BB17B78C2
:103CF00013BB002C49D1377E003718BF01272B7921
:103D00009A062AD44FB3A4BB2B795B0601D50721B1
:103D100001E01FB10321304600F02AFD95F904307F
:103D2000002B737EB4BF43F0080323F008037376BF
:103D30002DE0002CCBD12AE02CB3337E9C4209D05D
:103D4000224606A906F110000BF0D6FDB0FA80F06D
:103D5000400900E000200746D1E7002CD4D0A6F8A7
:103D60001A803476224606A906F110000BF0F6FD03
:103D7000CAE7737E03F00703072B08D103213046FF
:103D800000F0F6FC03E02746B9E70027B7E709B0E3
:103D9000BDE8F08F2DE9F04F87B015469846814673
:103DA0000291109FFFF7CAFBB0F8C6319A0706468A
:103DB00069D5EB79FF2B66D198F80140002C62D1D0
:103DC000072F60D905F10803083F0DF1100A03938E
:103DD000002F1FDD04F1080308EB030B18F8033074
:103DE000012B0FD198F800200298CDF800A05B4677
:103DF000294600F09BFE031E45DB524603994846C8
:103E0000FFF7FAFD9BF8013004EBC304A4B2A7EB63
:103E1000C307DDE7B6F8C63113F0040F05F1080556
:103E200028D013F0010F194B194C18BF1C4605F090
:103E30009DFE06F5FC7780463846FCF751FEB6F845
:103E4000C631DB0716D5294648460AF03FFA88B145
:103E5000B8FBF4F140F21523A6F80E320D4BC6F86C
:103E60001002B3F9003006F5037204FB11813846E5
:103E700009F026F8294648460AF028FA18B1437E88
:103E800023F00803437607B0BDE8F08F80841E005E
:103E900020A10700B82300202DE9F04F89B09246F9
:103EA000059181461E46FFF749FB0AF1080B0546BE
:103EB0000822844958460BF01FFD002840F0FF807F
:103EC0009AF80830FF2B00F0FA809AF80730FF2BA1
:103ED00040F0F5807378002B40F0F180129B0F2B9F
:103EE00040F2ED80594648460AF0F0F9074650B9CD
:103EF0000B23009302460346594648460AF078F9D8
:103F0000074668B9DBE0437E190706D5F28852BA46
:103F100092B212B923F0080301E043F008037B7664
:103F2000F3889CB264B15CBA674B68491B88A4B241
:103F30001BB207F13002614307F11C0008F0C0FF1B
:103F400033790BB185F8CA31B5F8C631C3F30D0228
:103F5000A5F8C62173791B0203F440431343A5F867
:103F6000C631B068A8B1D5F8D03190FA80F898453C
:103F70000FD005F0FBFD0A22B0FBF2F303FB1200A9
:103F8000053008FB00F0C5F8D081B0FBF2F0C5F8B1
:103F9000D401F36813B11BBAC5F8D83105F5E07048
:103FA000FDF77EFF129B103B0393002302930493C3
:103FB000039B002B58DD029B103306EB0308F35CD8
:103FC000052B1CD004D8012B0DD0032B1ED03FE0B5
:103FD000222B2AD0232B3BD14346129A3146484606
:103FE00004F0E0FE34E006AB0093327805984346D7
:103FF000514600F09BFD031E049329DA5FE0424620
:104000003178484600F013FE10BB58E04246317844
:10401000484600F029FE002851D0D8F804301BBAD9
:10402000B3B19C4228BF1C4612E04146307804F0F0
:104030000DFE002843D0B8F806305BBA9BB23BB106
:104040003C22B4FBF2F2934202D23C2202FB03F484
:1040500098F80130029A02EBC30292B20292039ADC
:10406000A2EBC3030393A3E7049B06AA5946484661
:10407000FFF7C2FC05F5EE70FCF732FDB5F8C6316E
:10408000DA071CD504EB4404042C88BFA1084FF0C8
:10409000000498BF0121384685F8CB4104F0BEFCEE
:1040A0003B463A462146B7F91A0000F0FDFAB5F84A
:1040B000C6319B0703D501212846FFF756FA09B000
:1040C000BDE8F08F9E220108FC02002040420F0054
:1040D0002DE9F041437E03F00703022B86B004462E
:1040E00001D0052B7BD194F89420B4F91A50012A01
:1040F00071D9022B11D14FF080730493FF238DF8F7
:104100001430637B8DF8153040F2FF200021E389E5
:10411000ADF81630CDE902010BE094E8030002ABE4
:1041200083E8030004F1080393E8030006AB03E906
:104130000300013A84F894201DBB01AE304601F023
:104140007FF80746BD4208D036F9150002AB22467B
:10415000002100F0A9FA0135F4E7224B04F13805FB
:10416000B3F900602846FCF7BBFC40F21223A4F828
:104170004E3004F14C0233461B49284608F0A0FE9D
:104180002DE02846FFF7DAF90646224602AB06F58F
:10419000E075B4F91A00002100F086FA01212846E2
:1041A000FDF74EFE0F4BD6F8D871B3F9008004F13D
:1041B00038063046FCF794FC40F21223A4F84E3047
:1041C0003046434604F14C02394608F079FE284651
:1041D000FDF766FE03E0214628460AF09FF806B088
:1041E000BDE8F081B823002040420F00437E03F079
:1041F0000703042B03D0072B04D1032100E0052182
:1042000000F0B6BA7047000038B500F5E075044616
:1042100001212846FDF714FE05F0A8FC0A210A4BEF
:10422000B0FBF1F202FB11000530C4F8D03143437A
:10423000B3FBF1F3C4F8D431044BC4F8D8312846A9
:10424000BDE83840FDF72CBE80C3C90140420F00D5
:1042500010B5044608462378FF2B14D000221823FB
:10426000872109F0D9FE002270B183681A715A7152
:104270009A71DA7121686268DA609960A168E2680F
:104280005A61196110BD002010BD38B50B78FF2BA5
:1042900005460C46104616D000221823882109F046
:1042A000BBFE002280B1836825F01F051D71DA7105
:1042B0009A715A7121686268DA609960A168E2684F
:1042C0005A61196138BD002038BD08B500220823A5
:1042D000852109F0A1FE28B1836800221A715A7164
:1042E0009A71DA7108BD10B5002304461046CA1D44
:1042F00002F0F802194601F0EBF920B1826814705F
:10430000C368DB08537010BDF8B516460F461A4651
:10431000B11CFFF7E8FF044660B18568C26802354A
:10432000023A002128460BF017FC3246394628464F
:104330000BF014FB2046F8BD13460A460146012047
:10434000FFF7E2BF13460A4601460220FFF7DCBF33
:104350002DE9F04180460F4616461D4600221023E7
:104360008621079809F058FE60B1069B846827F003
:104370003F0776BA2DBA1BBA84F804806771E680CD
:10438000A560E360BDE8F0812DE9F041074688466D
:1043900016462021079A03201C46FFF7A4FF054676
:1043A000C8B1806824BA0021846028F03F0800F179
:1043B000100436BA017341738173C173877080F83A
:1043C00003804660102220460BF0C6FB3A46069951
:1043D000204605F065FA2846BDE8F08110B50A468A
:1043E000044608210520FFF77EFF28B183680022DC
:1043F00024BA9A70DA705C6010BD000008B5102213
:1044000003490BF079FAB0FA80F0400908BD00BF0B
:10441000EE22010810B50822094904460BF06CFA97
:1044200048B12378FF2B08D1607800F00F00831E7D
:104430005842584110BD012010BD002010BD00BFE2
:104440009E22010870B506460846194609F06EFE20
:104450000446A0B18368FF22DA7100231A46194688
:10446000184600F003FF054620B92146204600F01B
:10447000E1FF02E083685E804460284670BD70BD45
:10448000002101F017BA0000F7B51F46537C802BBE
:1044900005460E46144603D911490320FCF7A4FB38
:1044A0001046FFF7ABFF08B1002017E02046FFF7EA
:1044B000B1FF0028F8D1217CCB07F5D43388607C8C
:1044C000626913F0010F14BF002680268DE890006A
:1044D000A3693143FFF758FF2860012003B0F0BD06
:1044E0002519010830B585B0022300930D460DF162
:1044F0000E0300220521044600F08EFC002803DB99
:10450000BDF80E30062B10D80823009300222B464E
:104510000221204600F080FC002802DBADF80E00EE
:104520000EE00023ADF80E300AE0082300930022CD
:104530002B460321204600F06FFC0628E4DDEDE762
:10454000BDF80E0005B030BD38B5002009F008FFF9
:10455000044658B1637E03F00703013B012B03D9E6
:104560000A4B00221A600EE02046EFE7074D28684C
:1045700009F0F6FE034618B909F0F2FE034610B141
:104580002B60184638BD204638BD00BF702C002077
:104590002DE9F7430A9C0F46994680461646FEF7DA
:1045A000CDFFB0F8C631990701D4002507E0404699
:1045B000FEF7C4FFB0F8C6315A07F6D5802530465D
:1045C000FFF71CFF38B11022334930460BF0C6F913
:1045D0000223737001E045F04005B9F1000F0BD0E4
:1045E00069464046FFF77EFF30B1C1B222466846B9
:1045F000FFF7A8FE68B1044624B13B7CDB0758BF37
:1046000045F02005224639462846FFF73EFE814602
:1046100008B920463BE00146002332464046FFF7FA
:1046200011FF054608B9484631E03B7CDFF874903D
:1046300013F0010F23D005F099FA184BB0FBF3F7F4
:10464000314607FB1307404609F040FE044618B9FF
:1046500013490320FCF7C8FA00F154063046FCF772
:104660003FFA40F20223A4F86A30E566B9F9003057
:1046700004F168023946304608F022FC09E00146A0
:10468000B9F9000000F0ADFB002802DC2846FFF776
:10469000F7FE03B0BDE8F083AE22010840420F00F0
:1046A00025190108B82300202DE9FF4707460D46CC
:1046B00090469946FEF742FF824618B92A490320E0
:1046C000FCF792FA35B92A4641463846FFF710F80A
:1046D000054668B102A93846FFF704FF064650B107
:1046E000C1B2002202A8FFF727FE044620B935E038
:1046F0000646044600E00446BAF8C631DB0714D586
:10470000082E0AD00823009300226B440321384668
:1047100000F082FB80B208281FD1234602AA0F2195
:10472000002004F0A7F9C0B1044621464046FFF737
:104730008FFD064688B101462B464A463846FFF7AC
:1047400081FE044608B9304608E0084B0146B3F93B
:10475000000000F046FB002802DC2046FFF790FE38
:1047600004B0BDE8F08700BF25190108B823002078
:104770002DE9F041437E23F007030B43052904464E
:10478000437620D0072903D004294BD1264E05E0DB
:10479000B0F91A00FEF7D2FED0F8D461234B04F131
:1047A0003805B3F900702846FCF79AF940F2172350
:1047B000A4F84E3004F14C023B4631462846BDE891
:1047C000F04108F07DBBB0F91A00FEF7B7FE0323F5
:1047D0000646224606F5E07584F89430B4F91A00CE
:1047E00023460021FFF760FF01212846FDF728FB43
:1047F0000E4BD6F8D871B3F9008004F13806304674
:10480000FCF76EF940F21223A4F84E3030464346CE
:1048100004F14C02394608F053FB2846BDE8F0414C
:10482000FDF73EBBBDE8F081404B4C00B8230020B3
:104830002DE9F3411B4D002918BF0D4600222946E2
:104840008046FEF755FF074670B169464046FFF7C0
:1048500049FE38B1C1B200226846FFF76DFD04463B
:1048600018B91AE0044600E004462046FFF72DFD83
:10487000064688B101463B462A464046FFF7E2FD20
:10488000044608B9304608E0074B0146B3F900007A
:1048900000F0A7FA002802DC2046FFF7F1FD02B085
:1048A000BDE8F081CE220108B82300202DE9F04FA9
:1048B0008BB0002791468A46039302900797FEF734
:1048C0003DFE964B064600F5E07801214046B9458D
:1048D00008BF9946FDF7B4FAB6F8C65115F00105C0
:1048E0001BD1344606F5E377B3465C4500F0ED8016
:1048F000627C9BF811309A4240F0E4805946204691
:1049000004F0A8FF637C834200F2DC8000E01D46D7
:104910003834A045E8D1079D4FE004F0FBF9054687
:1049200000284AD0846906F5E37BECB163689E42B7
:1049300018D1AB699C4200F0D780A268996892F8C0
:1049400011E0487C864540F0E380104605930492D0
:1049500004F080FF049A059B527C824200F2D880CA
:1049600000E01F462468E0E74FF0010B05EBD4039D
:104970009A7D04F007030BFA03F31A420CD0E0B25D
:1049800002F066FD428A417C0346007C009704F0F9
:10499000DBFA079060B107460134102CE6D12A46B5
:1049A000A98A28693B4604F0F5FA0546079020B924
:1049B0004046FDF775FA384681E0B6F8C6311B0768
:1049C00007D52946B6F8C801FFF708FD0790F8B1EA
:1049D0000546BAF1000F0FD14046FDF761FA49468E
:1049E00001220298FEF784FE012182464046FDF72F
:1049F00027FABAF1000F10D008A90298FFF772FD4C
:104A000058B1C1B22A4608A8FFF796FC079018B91A
:104A10004046FDF745FA3DE00546B6F8C62102F0EE
:104A20001004A4B20CB196F8CA4102F020039BB264
:104A30004BB1D6F8D4313A498B4206D84FF47A7B41
:104A4000B3FBFBFB03E09B4601E0DFF8DCB002F0C8
:104A50004007BFB22FB1D6F8D8714FF47A73B7FBC5
:104A6000F3F7039B13B9B6F8CC2100E000224046CF
:104A70000392FDF715FAB6F8C611039A01950912CB
:104A8000204600975B4601F0C001FFF761FC044639
:104A9000079008B9284612E0014653464A46029854
:104AA000FFF7D0FC0146079008B9204607E01D4BF0
:104AB000B3F9000000F095F900282BDC0798FFF708
:104AC000DFFC27E00BF1380B0FE72B462246394677
:104AD00007A8FFF7D9FC00283FF41AAF079B002B6B
:104AE0007FF415AF28460DE03B46A268594607A85B
:104AF000FFF7CAFC00283FF435AF079B002B7FF47B
:104B000030AF3846FFF7BCFC4046FDF7C9F901E07D
:104B10001B680FE70BB0BDE8F08F00BFBE22010895
:104B200000A493D6B823002080EE3600F8B51E46C8
:104B30009F1C5B780446154613B96FF01500F8BD4D
:104B400001F10800FFF75AFC0028F6D17CB394F974
:104B50001030013304D1A3681C78022C04D001E08A
:104B60006468F3E7082C06D17378012B14D0022B6C
:104B7000E3D1082411E0853D022D1BD884B9727859
:104B800008236FF0010413FB024402FB036616F8CE
:104B9000013D2BB9013CFAE70224853D022D09D8DD
:104BA0002246394606980AF0D9FE2046F8BD853DD2
:104BB000022DE4D96FF08500F8BD70B51D465B7815
:104BC0000446164613B96FF0150070BD01F10800D8
:104BD000FFF714FC0028F6D1882E27D1A91CA4B118
:104BE00094F91030013304D1A3681C78022C04D04E
:104BF00001E06468F3E7082C06D16B78012B0ED036
:104C0000022BE0D108240BE054B96C78E408023C94
:104C1000E4B20B1913F8013C13B9013CF8E7022484
:104C2000224604980AF09AFE204670BD70BDF8B581
:104C300017460D46FEF782FC7C78012C06460FD104
:104C4000862D0FD100F5E07521462846FDF7F8F8CE
:104C50007B681BBAA6F8C8312846FDF721F901E0A8
:104C60000020F8BD2046F8BD2DE9F0415378042B13
:104C700086B00746154671D186294ED102F110083B
:104C80004046FFF7C7FB0646002846D13846FEF7E8
:104C900055FCB0F8C631DA0703D595F90330002B7F
:104CA0003BDB41463846FEF79FFC044618B1427C88
:104CB000AB789A422AD06B6843B31022002102A835
:104CC0000AF04AFFEB785B0616D4AA78414602A8A0
:104CD00004F0E6FDEB78AA7803F0C00302A9384699
:104CE000FEF74AFC0446002839D03846FEF726FC79
:104CF000012103F0DFFF09E00821009104AB00224D
:104D0000384600F089F80028DFDA28E06B6833B90C
:104D10001CB121463846FEF757FC01261FE01BBA9E
:104D20006361AA68013312BAA2610CD00E4B6968A4
:104D30000E481B8809BA41431BB204F1300204F14A
:104D40001C0008F0BDF8237C23F07F03DBB2237442
:104D5000EA7822F03F0213432374DEE70026304650
:104D600006B0BDE8F08100BFFC02002040420F0009
:104D70002DE9F3410446884617461D4600F0F8FA2F
:104D8000064650B34146204600F0E0FA711E044644
:104D9000284600F07DFD04B3237A53B1012B17D1CF
:104DA000E068ADF8027000226946019508F0A4FFA2
:104DB00007E0B4F90C10ADF8027068460195FDF7F4
:104DC000D5F9002804DD204600F0E6FA0446E2E7C3
:104DD0000021284600F06EFDF5E7304602B0BDE840
:104DE000F08107B540F20223019101466846ADF813
:104DF0000230FDF7BBF903B05DF804FB07B540F2E4
:104E00000123019101466846ADF80230FDF7AEF985
:104E100003B05DF804FB000000B589B006930A9B5F
:104E2000ADF81C304FF401738DF81410ADF8162056
:104E3000ADF80630024605AB03A901A80293FDF7C1
:104E4000B9F9BDF80E2040F205239A4203D0044977
:104E50000320FBF7C9FE049809B05DF804FB00BF0E
:104E60002519010800B589B006930A9BADF81C30DE
:104E700040F203238DF81410ADF81620ADF806307B
:104E8000024605AB03A901A80293FDF793F9BDF80B
:104E90000E2040F205239A4203D004490320FBF779
:104EA000A3FE049809B05DF804FB00BF25190108B2
:104EB0002DE9F04384680746208F638D8FB000F0A2
:104EC000280EADF818304EF0010E0E4611B96FF0F5
:104ED00015005DE091F91030013354D18D682B79C4
:104EE0002A7813F0C00F03BF02F108035B1995F88D
:104EF00001C0294B18BF4FF0020C12B105F1080197
:104F000007E0420747BF04F12E01082204F12C01FB
:104F1000022294F8360000F1010884F836800490EB
:104F20000DF12008BDF81800ADF80800ADF8040038
:104F3000CDF80CE0CDF800C0404604F00FFB8146F0
:104F40000028C4D0304607A900F048FA0646E8B168
:104F5000816881E800032B7913F0C00FBB6815BF8F
:104F60001A69DA680132013214BF1A61DA60236803
:104F7000079A1B682046984700210446304600F0F7
:104F800099FC204604E06FF04C0001E06FF06800EF
:104F90000FB0BDE8F08300BF9C2201082DE9F0436B
:104FA00087683B685C68002387B01A461946384614
:104FB000A047041E15DD002322461946184600F0BE
:104FC00087FB054668B13B6881685E6822466B4690
:104FD0003846B047B0F1000805DC0021284600F053
:104FE00069FC002466E03E8F06F00206B6B2002E91
:104FF0005BD1A86804F046FB044608B9014637E0D7
:105000000146C0EB08083246284600F07BFB81468B
:1050100008B90146E2E7866801AA04A9304604F00F
:10502000A7FB01AA044602A9304604F04FFB002C5E
:1050300001DA00241BE00028FBDBC1B2E3B204AAC2
:1050400002A800F013F906460028F2D0022C0CD179
:105050009DF81030FF2B08D19DF81130FF2B01BFB8
:105060008268137963F07F031371344626B90021F7
:10507000284600F01FFC1DE0B3689DF801209A71DE
:105080009DF800205A710D4A12885A8097F82830EE
:105090002B744946284600F0CDF9002373602B4657
:1050A0005A680AB11346FBE75E604146284600F0A5
:1050B00097FB2C46204607B0BDE8F083FC02002099
:1050C000034B0360034B436081600020704700BFC7
:1050D000B14E00089D4F0008F0B5254E8468338816
:1050E000838195B00821054604A8FDF7C5F83088EE
:1050F000204B6360A56000B200F090F82368204662
:105100009B68984740F2032741F234266846FDF732
:10511000B0F8BDF80230BB4213D0B3F5017F08D21E
:1051200040F202229342F1D12B6801992846984718
:10513000EAE70AD0B342E9D123682046DB68984702
:10514000E2E7236801995E6902E0236801991E691C
:105150000B894A6809782046B04740F2052303903E
:1051600002A96846ADF80A30FDF752F8CCE700BF57
:10517000FC0200207951000813B50346806879B914
:1051800041F234230190B0F90C10ADF802306846BA
:10519000FCF7CAFF002822DC12480AF06FFE1EE06E
:1051A000042919D0072913D0022918D14368984738
:1051B0000446A0B103460C4990F9100040F20122C8
:1051C000FFF7D6FD014650B9204600F073FB06E01C
:1051D0009A6901329A6102E05A6901325A6102B059
:1051E00010BD00BFDE2001080000FFFF30B585B014
:1051F000089C6CB1A5685DB10293074B00930194C4
:105200000823FBF791FD0028D8BF6FF0150001E0DF
:105210006FF0120005B030BDD9500008074B10B533
:10522000B3F90040A04201D1002010BD14B16FF0CD
:105230000B0010BD1880FEF755F9F5E7742C00201F
:10524000044BB3F9003013B10380012070471846B6
:10525000704700BF742C0020034BB3F900301B1AB9
:1052600058425841704700BF742C00202DE9F0418E
:10527000174603F108020A440E46002180461D46E7
:1052800008464FF0FF3300F023FA00220446F8B13D
:1052900083681E705D705A805A719A711A71B8F1E4
:1052A000000F08D03EB180680278B24203D1414677
:1052B00008300AF053FB5FB155B1A0684378AB42A8
:1052C00006D1037808332A46394618440AF046FBCB
:1052D0002046BDE8F081000008B50B7A53B9B1F95A
:1052E0000C200B4B53F822301B6A1BB909490320D1
:1052F000FBF77AFCC3B2042B9FBF074B53F8202067
:105300000A6043F8201094BF00206FF0150008BD1C
:105310004803002025190108782C0020C3B2042B73
:1053200011D8094A52F820308B4206D11B6842F846
:1053300020307047914204D013461A68002AF9D1F0
:1053400001E00A681A607047782C0020C3B2042B71
:1053500009D8064B53F8200020B143688B4203D094
:105360000068F9E770470020704700BF782C0020E4
:10537000C3B2042B0BD8074B53F8203000202BB1BD
:105380005A681B688A4208BF0130F8E7704700205E
:10539000704700BF782C002028B14368006810B126
:1053A00042689342FAD1704749B190F91030032B0B
:1053B00003D0042B06D104F073B808F03DBE6FF0A3
:1053C000150070476FF00100704728B190F9103058
:1053D0008B4201D04068F8E77047000070B5044682
:1053E0000E4619B912490320FBF7FEFB10B9002045
:1053F000306070BD01460025496801350029FBD1A8
:105400006FF00103EA00204600F062F90028EED0B8
:105410008368002BE6D00833A26843F8082CE268C2
:10542000646843F8042C0833002CF5D1356070BD56
:105430002519010810B504468C42084601D164685C
:1054400008E023465A682AB1904201D01346F9E792
:1054500042685A600021416000F02CFA204610BDDD
:1054600070B5556804460846EDB129464B680BB146
:105470001946FBE71CB91A490320FBF7B5FB0028C6
:10548000F9D0002AF7D043685360844206D02346FF
:105490005E6826B1B04219D03346F9E71446536826
:1054A0004B60556015E0002CE5D00029E3D0002AC0
:1054B000E1D04B6853608C4206D02346596841B115
:1054C000884205D00B46F9E7144602E05A60E6E749
:1054D0005A600021416000F0EDF9204670BD00BF28
:1054E0002519010870B503461A4A072B88BF0333F4
:1054F00010688CBF23F003030823002140B34468E5
:10550000A34202D901460068F8E7E41A072C0344D5
:10551000114E05D8046809B9146011E00C600FE061
:10552000C6F108051D44B5F5C05F02D90021116020
:1055300003E009B9136000E00B60026883E814001F
:10554000064A9B1B11889BB2994201D2138070BD01
:1055500070BD00BF902C0020942C00208C2C0020CB
:1055600001210148FCF76CBC94440020204A38B566
:10557000831AB3F5C05F39D21E4D2C68002324B1C5
:10558000844202D223462468F9E707298ABF0331FF
:10559000082121F003010460141AC1F5C05222440D
:1055A000072A98BF891841600BB9286011E05A6832
:1055B00018601A44821A072A0BD818B90E4903201A
:1055C000FBF712FB026841681A60C21A0A445A606B
:1055D0001846036853B1426802449A1A072A05D84C
:1055E0001A6802601A1A5B681344436038BD00BF32
:1055F000942C0020902C0020251901082DE9F84357
:10560000814614200F4616469846FFF76BFF044666
:10561000D8B15EB13046FFF765FF054638B9204680
:105620001421FFF7A3FF2846BDE8F8833546012380
:10563000C4F80490A560E66084F81080236027B168
:105640003246394628460AF089F92046BDE8F883F3
:10565000F8B50F4D04460026CCB1631BB3F5C05F0F
:1056600003D30C490320FBF7BFFA94E88800012B11
:1056700009D1E168A0682660FFF778FF1421204671
:10568000FFF774FF01E0013B23603C46E4E7F8BD0F
:10569000942C00202519010808B5FFF761FF094A7D
:1056A000094B1360182100221A705A709A70DA7030
:1056B0001A7159719A71DA710448BDE80840FCF713
:1056C000EFBB00BF902C0020942C002094440020BD
:1056D000B2F5C05FF8B505460E4614461F460DD814
:1056E000FFF73EFF22463B4631462846FFF786FF3E
:1056F00004460348FCF7D4FB2046F8BD0020F8BD63
:105700009444002007292DE9F84388BFCF1C0D469B
:105710008CBF27F00307082704469146FFF720FFB8
:105720002DB124B1E3689D4201D8A3682BB92B4861
:10573000FCF7B6FB0020BDE8F8831420FFF7D2FE8B
:1057400006460028F3D0E3689D422ED0AF4202D82F
:105750005A1B072A29D82846FFF7C4FE074610B966
:10576000142130460BE0E068401BFFF7BBFE80468B
:1057700040B914213046FFF7F9FE29463846FFF7B5
:10578000F5FED4E72A46A16838460AF0E7F8E26851
:10579000A168521B294440460AF0E0F8E168A0687D
:1057A000FFF7E4FEC4F8088005E0A7689D4214BF37
:1057B0007B190023A360E36808485B1BE360636810
:1057C00073600123B760F56086F8109033606660FF
:1057D000FCF766FB3046BDE8F88300BF9444002028
:1057E000072970B588BFCE1C04468CBF26F003067F
:1057F00008260D46FFF7B4FE1CB922490320FBF72B
:10580000F3F9E368A06813B90028F6D106E0002890
:10581000F3D01D4A821AB2F5C05FEED29D422CD061
:105820002DB930B11946FFF7A1FEA56024E09D42D5
:1058300002D8991B072917D82846FFF753FE0646BA
:1058400020B91248FCF72CFB0C2070BDA16829B1CF
:10585000E268AA4228BF2A460AF080F8E168A068F8
:10586000FFF784FEA66007E0033323F003039E42A4
:1058700002D23044FFF77AFEE5600448FCF710FBE3
:10588000002070BD25190108942C002094440020AC
:1058900038B504460D46FFF763FE24B123682B4458
:1058A00023606468F9E70248BDE83840FCF7F8BABD
:1058B0009444002010B50446FFF752FE2046FFF73F
:1058C000C7FE0248BDE81040FCF7EABA9444002045
:1058D00038B50446FFF744FE0CB1E26822B90E4821
:1058E000FCF7DEFA002038BD2368012B0FD994F9AC
:1058F0001030A1686068FFF781FE054610B123688B
:10590000013B23600448FCF7CBFA284638BD024827
:10591000FCF7C6FA204638BD94440020F8B50026AE
:10592000074604463546002C48D02946E2682948F7
:105930000AF01AFA94F910104B1C052B31D8DFE845
:1059400003F006030F182028002123482AE04FF017
:10595000FF3122480AF008FAA06808F0E9FD28E0C3
:1059600001211F480AF000FAE168A06806F056FE1F
:105970001FE002211B480AF0F7F9A06804F072F852
:1059800017E0032118480AF0EFF9A06803F0D2FDF0
:105990000FE0042115480AF0E7F9A06807F01CF9A8
:1059A00007E013480AF0E0F91022E168A06804F06B
:1059B000A5F8E368646801351E44B4E72946324619
:1059C0000C480AF0D1F921463846BDE8F840FFF707
:1059D00071BF00BF04210108292101083D210108F0
:1059E00051210108692101087C2101089121010848
:1059F000A3210108B921010800B595B0082104A828
:105A0000FCF73AFC6FF08503039340F20523ADF8F1
:105A10000A306846FCF72DFCBDF802306FF40072C6
:105A20001344032B11D8DFE803F002040B0B0948E1
:105A300000E009480AF022FA0198FFF76FFFE8E753
:105A400002A96846FCF7E4FBE3E704480AF016FA0B
:105A5000DFE700BFE6210108FE2101081522010849
:105A60001FB50A4CB4F9003063B9094A0193094BD8
:105A700002920093062208234FF4C0610648FBF708
:105A800053F92080B4F9000004B010BD9844002000
:105A90003C220108F95900089A44002007B501A8E2
:105AA000FFF7CEFBBDF9040000F006F903B05DF886
:105AB00004FB00002DE9F043082187B07648774CBD
:105AC000774FFCF7D9FB40F20523ADF8123026469C
:105AD00002A8FCF7CEFBBDF80A30B3F5017F09D868
:105AE00040F20322934280F0CF8040F201229342A1
:105AF00077D0EDE7B3F5106F04D040F60112934272
:105B000064D0E5E7674D05F1900815F8013CD3B185
:105B1000D5F81730022B0DD9042B05D8D5F8133042
:105B20002946986900F0E0FAD5F81730023BC5F82D
:105B3000173008E0D5F81390681F01F0C7F800216E
:105B4000484601F051F93035A845DED16378ABB352
:105B500094F98C30002B20DC96F83730022B18D8C3
:105B600094F8351051BB94F83430032B07D93C23FB
:105B700084F8373084F8341084F835101EE001338F
:105B800094F82920206A84F8343000F0ADFD032316
:105B900000E0023B84F8373010E0E269002ADBD1F4
:105BA000218E4FF6FF729142D6D1023B5BB2002BA1
:105BB00084F88C30D0DC394801F0E3F8B7F90030D4
:105BC000394A3A493A4807F07BF981E703980028B7
:105BD0003FF47EAF4369002B3FF47AAF06F09EFF9F
:105BE00076E7039D1DB933490320FAF7FDFF022133
:105BF0002846FFF7EAFB4FF0FF3180462846FFF7C3
:105C0000E4FBB8F1000FEED018B18368B3F90210CD
:105C100000E00146A868D8F808204378032B2ED866
:105C2000DFE803F0020D182393885BBA9BB2009360
:105C3000043002F11803083200F098FA1FE093884C
:105C40005BBA9BB20093043002F11803083200F0F3
:105C5000A9FB14E093885BBA9BB20093043002F175
:105C60001803083200F0AAFE09E093885BBA9BB2E1
:105C70000093043002F11803083200F0F9FE00210D
:105C80002846FFF717FE23E76FF0850304A902A853
:105C90000593FCF7BDFA1BE79C4A0020A04F0020AB
:105CA0009A4A0020F54A00205C02002080841E00F1
:105CB000884B0020251901087FB51C4CB4F9005011
:105CC000064625BB1A4B1B481D701B4B02931B4BF2
:105CD00000930195082305224FF48061FBF724F817
:105CE000208000B316499B22888103204A60FFF779
:105CF000F3FA00F005FF134A13491448B4F90030D1
:105D000007F0DEF880222946114809F025FF00231C
:105D1000802210493046FDF72FFC00200D4900F08D
:105D2000E3F9B4F9000004B070BD00BF9A4A002046
:105D3000804B00209C4B002054220108B55A0008DB
:105D4000DC4A00205C02002080841E00884B00207A
:105D50003050002044220108012380F82F30002316
:105D600080F82C3080F82D3070473C2380F82F309D
:105D7000002380F82C3080F82D30704710B50121B9
:105D800004460948FCF75CF8084B1878421C1A7066
:105D900014B140F0800401E000F07F040248FCF7F9
:105DA0007FF8204610BD00BF844B0020804B0020B0
:105DB00013B50C4612B11846FFF7E0FF2146022248
:105DC00001F0E2F8044678B30022032180F8252090
:105DD00080F82710012314220A2180F8243080F84B
:105DE000262080F8281084F82F3084F832304FF4C1
:105DF0008073238694F83630052043F0030384F83B
:105E0000290084F836303C20094B6085F02084F866
:105E10002E00B3F9000001910092082340F6011210
:105E200004F1380106F0A0FE204602B010BD00BF0C
:105E30009A4A00200021FFF73DBD10F0800F4BB2C1
:105E400002D0002B11DA01E0002B10DB884204D2D3
:105E5000C1F1800303440F2B09DD884205D9401AA4
:105E60000F28CCBF00200120704700207047012080
:105E700070470000F8B5074615461E460C4639B96E
:105E800020461949FDF7D8FB044608B9384625E0F5
:105E900035B916492046FDF709FC05460028F5D01E
:105EA000114A2946002E18BF3246384608F03EF9FE
:105EB00006460028EAD000231A4619461846FFF77E
:105EC000D5F983680A495C8005464660034640F27E
:105ED00002220220FEF74CFF20B92846BDE8F84018
:105EE000FFF7A8BFF8BD00BF442201089E220108A9
:105EF0000000FFFF002370B510220C46194606462D
:105F0000FFF7E6FB054618B93046FFF793FF24E09C
:105F1000836804221A7000210E225A709970A27FA1
:105F2000DA70E27F1A7194F820205A71A269B2F8EF
:105F30008A2052BADA80A269B2F8882052BA1A814D
:105F4000A269D2F884201288197352BA5A8194F83F
:105F500021205A73628C52BADA81284670BD002320
:105F600070B520220E4619460446FFF7B1FB0546E0
:105F700018B92046FFF75EFF1EE080680823037013
:105F80001E2343704023C37033695A6942609A6983
:105F900082605B7C8370002100F110040173417307
:105FA0008173C1731022204609F0D6FD3369314652
:105FB0005A7C204603F074FC284670BD2DE9F3415D
:105FC0000F460446002800F0898090F8363003F030
:105FD000020300F1080603F0FF0533B1314600204B
:105FE000FFF7BDFF0546002878D094F83630DB0770
:105FF0000CD528463146FFF77DFF054600286DD0B9
:1060000094F8363023F0010384F836300023182248
:1060100019462846FFF75CFB804608B9284637E05A
:10602000836822781A7094F82E205A7094F83220DF
:10603000022A04D14FF0FF329A70DA7002E0228E09
:1060400052BA5A8094F8802094F82F10D20042EA75
:10605000C11294F825100A431A7194F824205A7139
:1060600000229A71DA713546083304F1180E2A4677
:1060700003CA724518605960154603F10803F6D14A
:10608000042301229B21404607F0C6FF28B9404661
:1060900002B0BDE8F041FFF7CDBE03460022D9684B
:1060A0005B680A44002BFAD10E4B17B13978FF29EF
:1060B0000DD1996901319961D9690A44DA61B4F95C
:1060C0002C1000963B460022FFF7D4FE06E019692B
:1060D0000131196159690A445A61F0E702B0BDE81B
:1060E000F08100BF30500020F0B51E4B85B000227B
:1060F0000546186803900F460A239B21104607F0B7
:106100008BFF064658B38068002404714471042252
:1061100003A9063009F022FC32462346D1685268B2
:106120000B44002AFAD1104A17B13978FF290FD150
:10613000916B01319163D16B0B44D36305B1083589
:10614000002200953B4611463046FFF793FE06E0DD
:10615000116B01311163516B0B445363EEE705B0D2
:10616000F0BD00BF582201083050002030B419485B
:10617000BDF808505BB11978FF2908D0046A0134D2
:106180000462446A2C444462052D07D820E0846AE6
:1061900001348462C46A2C44C462F5E71B780E485B
:1061A000FF2B09D143789BB190F83230022B0FD0EE
:1061B000383030BC06F0C2BC43784BB190F8363072
:1061C00043F0010380F83630114630BCFFF7F6BECD
:1061D00030BC704730500020A04F00202DE9F04F18
:1061E0008BB00026159F07933E600C46154600F0C5
:1061F00048FF8246002800F0CF80B0464FF47A7BFB
:10620000079B434540F2C8802B78082B00F2BD80E5
:10621000DFE803F0050FBBBB147698BB4C003B686E
:1062200008F1010843F001033B601FFA88F80135CB
:10623000E6E73B6843F002033B60A6E03B6843F0BF
:1062400010033B6094F8363043F0010384F8363095
:10625000688940BA80B200F05BFC10B1C4F88400D9
:1062600003E000F055FCC4F88400E87884F82600C8
:1062700095F804E084F827E0697984F82810EB8821
:106280005BBAA4F88A302B895BBAA4F888306B7BA0
:1062900084F82930EA8984F83900012352BA03FAD4
:1062A0000EF36285E36384F838106EE03B68B4F95E
:1062B0002C0043F480733B6094F83630082143F09F
:1062C000020384F83630009108AB0022FEF7A4FDEB
:1062D000002802DAEB785B0657D5082208A905F1F9
:1062E000100905F1180009F039FB0023AA78B4F968
:1062F0002C004946FDF740F9002846D0A06144E053
:106300003B68B4F92C1043F020033B6094F829005B
:10631000638DEA7843430BFB03F3002E08BF2E4640
:106320000493802A4FF0010394BF120600221498B0
:10633000039310230190009202932A1D1848FCF742
:1063400019F922E03B6843F040033B600EB9002698
:106350001BE04FF010096A79638DCDF8009053432C
:106360000BFB03F3029395F902300D48DB43DB0F7F
:106370000193311D149B1022FCF784F973780233CA
:106380001E443378052BE6D0E1E76B78023398445E
:106390001FFA88F81D4433E750460BB0BDE8F08F74
:1063A000842300202DE9F04786B01746002203928F
:1063B00004460D46BDF83860A74A5BB11B78FF2B39
:1063C00008D01368013313605368334453601B2EA5
:1063D00007D83DE1936801339360D3683344D360B9
:1063E000F5E71C3E03A92078B6B200F0ABFB00280D
:1063F00000F0898063885BBA9BB24FF6FF729342CC
:1064000000F023812379DDF80C80C3F3C20388F800
:106410008030002000F07CFBC8F884004DB928468D
:106420008E49FDF709F9054618B98D490320FAF799
:10643000DBFB2A46002304F10801039800F0B2FBBD
:10644000039D06AA05F10808002342F8083D3946D5
:10645000404600F0E7FB18B9049B002B00F0F580E4
:10646000637885F82E3023790399DB0985F82F307E
:10647000237903F0070385F825306388049A5BBA13
:10648000D38206AB002243F8042D0120019300972C
:10649000334604F11802FFF7A1FE002800F0D58072
:1064A000059810F0100407D1039800F06AFC3946F3
:1064B0002046FFF719FECBE0AB6943B94146B5F979
:1064C0002C00FDF7F3F8002800F0BF80A8614046DB
:1064D000FFF742FC634A95F82730B2F9000095F8BF
:1064E0002820019295F826200092012202FA03F357
:1064F00005F1380140F6011206F036FB04994046DA
:1065000000F072FCA4E0039D002D00F0A18005F1D5
:106510000808102204F10801404609F0EDF981460F
:10652000002840F09580039A237992F88020C3F3E5
:10653000C2039A4240F08C80627895F82EA01046F3
:106540005146FFF77AFCC8B195F83230012B0FD1D4
:10655000130601D5FF2A00E07F2A1ABF0132D2B20A
:106560004A4685F82E2005F1380006F0E7FA0BE0E0
:1065700085F82E20404600F015FC05E011465046F7
:10658000FFF75BFC002837D195F83230012B0BD197
:1065900063885BBA9BB24FF6FF72934205F13800F5
:1065A0002CD006F014FB53E006AA002342F8083D65
:1065B0003946404600F036FB049B08B9002B47D013
:1065C0001BB105F1380006F002FB049900293FF4E5
:1065D0002CAF63885BBACB82404600F005FC049B7D
:1065E0001A7972B963885BBA9BB24FF6FF72934215
:1065F0002ED12A8E9A422BD005F1380006F09EFA51
:1066000026E0EA69934223D15A7D63799A4202D007
:106610004046FFF7A1FB049B62795A7523790399E1
:10662000DB0985F82F30237903F0070385F825303F
:1066300006AB002243F8042D012001930097334656
:1066400004F11802FFF7CAFD10B9039800F099FB96
:1066500006B0BDE8F08700BF30500020442201089A
:10666000251901089A4A0020F8B500230C46164661
:10667000194614220746FFF72BF8054618B9384685
:10668000FFF7D8FB11E0836805221A7012225A70B6
:1066900000229A70DE702146043304F1100251F892
:1066A000040B43F8040B9142F9D12846F8BDF8B524
:1066B00000230E461546194606220746FFF708F83E
:1066C000044618B93846FFF7B5FB0AE0836806228E
:1066D0001A7004225A70ED0100229D70DA701A714E
:1066E0005E712046F8BD00002DE9F04F8DB00E46DA
:1066F00006920546002800F0FD8090F83230012B0C
:1067000000F0F88021B9C669002E00F0F38005364C
:106710000CA805F108030024194640F8044D059320
:1067200009940A94FCF79CFF0B9B002B00F0E2807D
:1067300001217248DFF8D8B1FBF782FBA046049430
:106740000394DBF808309C4268D2DBF8007007EB5A
:106750004417D7E9022313435ED0BB69DA070CD490
:10676000039BD3B9012206991846FFF7A0FF0A90B0
:1067700088B96248FBF794FBBCE0049B83B91A46D6
:1067800006991846FFF793FF804609900028F0D03D
:106790000123049304E0012303930DF1280901E090
:1067A0000DF124097B699A78FF2A03F1020A07D1C7
:1067B000D87800F00F00A0F10E035842584120E0B5
:1067C00008224F490793504609F096F8079B08B9ED
:1067D000002016E09A78FF2A04D1DB7803F00F033B
:1067E000022BF5D010224749504609F085F80028C1
:1067F000EED010224449504609F07EF8003018BF10
:10680000012048B1FA7CD9F800005146FFF72CFF6F
:10681000C9F800000028ACD0013492E73748FBF7F4
:106820003FFB0A9BB8F1000F02D0C8F8043000E02B
:10683000099380220B990998FFF716FF04460990E7
:10684000002857D095F90070002F07DA0023102296
:106850000599FEF73DFF0A9030B30990DDF82480DA
:106860000023042219464046FEF732FF04460A90F0
:1068700008B9404619E083682A781A70002FB4BF1F
:10688000402200225A705A78099062F07F025A70B2
:1068900095F83320DA7000279F70022204239B2191
:1068A00007F0BAFB0A9018B92046FFF7C3FA21E0B7
:1068B000099002463B46D16852680B44002AFAD13F
:1068C0003278FF2A114A0ED0116D01311165516DD8
:1068D0000B445365059BB5F92C10009300223346F9
:1068E000FFF7C8FA06E0916D01319165D16D0B4457
:1068F000D365EFE70DB0BDE8F08F00BF9023002017
:106900009E220108EE220108FE22010830500020DC
:10691000842300202DE9F7430E46914604460028C3
:1069200046D090F90080B8F1000FACBF08231823BF
:1069300003229B21002007F06FFB0546002837D07B
:10694000876823783B71B8F1000F09DA80237B71E7
:10695000102204F1080107F1080008F0FFFF01E030
:1069600000237B71002387F80690FB712A46D168CB
:1069700052680B44002AFAD10F4A16B13178FF2928
:106980000FD1916F01319167D16F0B44D367B4F987
:106990002C1008340094334600222846FFF76AFA88
:1069A00006E0116F01311167516F0B445367EEE739
:1069B00003B0BDE8F08300BF305000202DE9FF4157
:1069C00017460546BDF82840284A8BB11B78FF2B97
:1069D0000ED0136C01331364536C234453646B78EF
:1069E00013F0400F0CBF082318239C423AD306E053
:1069F000936C01339364D36C2344D364EFE728781A
:106A000000F0C2F8064668B36B785B0605F1040136
:106A100006F1080801D4083C07E01022404608F0BF
:106A20006BFFF8B905F11401183C96F83220022AE0
:106A3000A3B217D004AA002042F8040D00970192D7
:106A400002200A463146FFF7C9FB58B195F90130DB
:106A5000002B04DAEA7839463046FFF75BFF404600
:106A6000FFF77AF904B0BDE8F08100BF3050002094
:106A700070B5224A0446BDF81000A3B11978FF2969
:106A800011D0116E01311166516E014451661B78AF
:106A9000FF2B32D094F90130002BACBF0823182310
:106AA00098422AD106E0916E01319166D16E01447F
:106AB000D166ECE7207800F067F80546E8B194F974
:106AC0000130002B05F1080602DBE37843B90CE046
:106AD0001022211D304608F00FFF0028F5D070BDB0
:106AE000A27895F833309A4207D1012385F83530E2
:106AF0003046BDE87040FFF738B970BD3050002017
:106B000008B500F021FB014B186008BDB050002013
:106B1000054B1B680BB900F017BB1A8882420CBFEB
:106B200018460020704700BFB050002090F8322077
:106B3000022A02D1383006F047B80149FFF73EBAC1
:106B40004422010810B500230E4A0B6054780CB99A
:106B50000A6004E01478844201D10A600FE00B68F7
:106B60006BB118700B68012058700B6800224FF44D
:106B70008071A3F88A20A3F88810DA6110BD184646
:106B800010BD00BFA04F0020054A53782BB11378E9
:106B900083420CBF1046002070471846704700BF64
:106BA000A04F0020F8B5044608B1407818B91B4939
:106BB0000320FAF719F80D4604F1080701F1100E49
:106BC000286869683E4603C6083575453746F7D1DB
:106BD0004FF6FF7121861249E164142184F82610D2
:106BE000032184F827100A2184F82810052184F84D
:106BF00029103C216185F020002184F8330084F8BD
:106C0000321084F8241084F83410246584F8351088
:106C10002462A285A3610120F8BD00BF25190108E7
:106C20002D6B00082DE9F8430026264F166080469C
:106C30000D4614464FF0010917F8013C33B9B9F17C
:106C4000000F14D07A1F2260994610E0D7F8133055
:106C500043450CD12946384602F0E7FD38B11A4ABF
:106C6000302303FB062626600020BDE8F8830136AA
:106C7000032E07F13007DFD1206800B3C0F8188079
:106C8000236800221A60D8F8143033B11A680AB1A8
:106C90001346FBE722681A6002E02368C8F8143044
:106CA000236801221A7123682946053305F1100271
:106CB00051F8040B43F8040B9142F9D10120BDE8CF
:106CC000F88300BFF54A0020F04A002030B50446A2
:106CD00087B018B920490320F9F786FF85696B69E9
:106CE00098422AD110221D491D48FBF714FD236844
:106CF000D3B10020FAF746FD22681A4BB0FBF3F03F
:106D0000D369B5F92410181A4FF47A735843053231
:106D10000123039301921023002204900092029316
:106D20000E4A0F48FBF726FC6B699C4205D123688D
:106D30006B6108E0944204D013461A68002AF9D126
:106D400001E022681A6030220021204608F004FF8A
:106D5000012007B030BD00BF25190108EE2201084F
:106D60008423002040420F0038B50446406920B11A
:106D70000568FFF7ABFF2846F9E74FF6FF73238559
:106D800038BD10B504460830FFF7EEFF04F13800B7
:106D900005F01AFF90220021204608F0DDFE0120B8
:106DA00010BD000010B5037F01330377436904462B
:106DB00033B1FFF7D9FF102209490A48FBF7ABFCB2
:106DC000228D4FF6FF739A4208D0238504F13000DC
:106DD00005F0B4FEA369052283F88C2010BD00BF26
:106DE000EE220108842300202DE9F04F0A4689B0E5
:106DF0000446E1B1438C90F821105943D1614169B7
:106E00008A4214D1B0F9241090F8210043434FF482
:106E10007A704343053204930123039301921023B4
:106E2000002200920293564A5648FBF7A3FB63697F
:106E3000228D0692002B00F099804FF0010B00226A
:106E40006669626192469146002E36D00AF1010AC7
:106E5000354600272D6801370DB9D84610E05F454B
:106E6000F8D1FAE7B8F1000F0DD12A463546366859
:106E7000013FB9F1000F1CD0C9F80050A9461546D2
:106E8000002FEFDC01E02DB9EFE7B8F1000F12DDC4
:106E90008DB157B1A2690793D2F884202946D268F0
:106EA000304690470028079BDFDD2A6808F1FF384D
:106EB000DFE76561E2E72E46C6E7B9F1000F01D0D2
:106EC000C9F80060BAF1010F4FEA4B0BB7DC6269F9
:106ED000D08A4FF6FF71884248D0934223D0A069F0
:106EE00090F88020023A012A06D80022591DFFF7A7
:106EF000FBFB2046FEF730FF638C94F82120B4F9A9
:106F0000241020485A434FF47A7353436269049320
:106F10000532012303930192102300220092029371
:106F2000174AFBF727FBA3696069D3F88430002177
:106F30005B689847069B2085834203D004F13000AC
:106F400005F0FCFD606978B1A369228DB3F8881063
:106F5000C38AB2FBF1F2B3FBF1F39A42056801D8A0
:106F6000FFF7B4FE2846EEE763692BB9204609B067
:106F7000BDE8F04FFFF716BF09B0BDE8F08F00BFC6
:106F8000EE22010884230020334BB3F900302DE9B1
:106F9000F34106460C4615460BB9002058E0002385
:106FA00001930B78FF2B0BD14B7803F00F030E2BC3
:106FB000F3D121466846FCF73FFB074608BBECE7E8
:106FC00008222649204608F097FCA0B12378FF2B21
:106FD00004D1637803F00F03022B0CD01022204958
:106FE000204608F089FC30B110221E49204608F0E6
:106FF00083FC0028DDD123780433DBB2012BD8D900
:10700000CBE7DDF80080B8F1000FC6D001A930460B
:10701000FFF798FD0028C0D00020019EFFF778FD03
:10702000C6F8840001984FF48073A0F888300023DC
:10703000A0F88A30214680F8805043463A46FFF750
:10704000B1FD0446019814B9FFF79BFEA5E7006265
:1070500002B0BDE8F08100BF9A4A00209E220108DC
:10706000EE220108FE220108022380F82A300021C6
:107070008069FEF7A3BF002380F82A30303005F086
:107080005DBD70B500249C422ED21578082D25D800
:10709000DFE805F005242424091319240E00013427
:1070A000A4B20132EFE7012822D155780E2D14E069
:1070B00001281DD155781E2D0FE0022818D15578D2
:1070C000122D0BD914E0022812D191F88050567875
:1070D000012D14BF04251425AE4209D1557802357F
:1070E0002C44A4B22A44CEE70CBF0120002070BD7E
:1070F000002070BD704711B970B1C18A00E020B1A5
:1071000083699B69B3F8880001E04FF480700844FC
:10711000814201DC80B270474FF6FF707047C28A2F
:10712000CB8A9A4203D38CBF0120002070474FF0D6
:10713000FF30704738B50446FFF7F1FF0028CCBF99
:107140000846204638BD704700487047640200205A
:107150000021FEF7AFBB00002DE9F0419EB01022E8
:1071600000210AA808F0F8FC804B0B93804B082103
:107170001B88ADF834300EA8FBF77EF80AA9012071
:10718000FEF7AAF840F20523ADF81A3040F20324C6
:1071900040F2012504A8FBF76CF8BDF81230B3F5F6
:1071A000017F09D8A34280F0D880AB420CD040F2D6
:1071B000022293426ED0EDE740F225229342E9D1BC
:1071C000059800F0EDF9E1E7059D2846FEF780FB04
:1071D000044600287ED00121FEF7F7F8054608B1E5
:1071E000C3681BB92046FFF7B3FFCFE783681B785E
:1071F000412B11D1FEF76CFB05460028F2D001228D
:107200001146FEF77FFA01460028EBD02046FEF734
:1072100011F90223044631E003F0D802C02A03D159
:10722000204600F0B1FAB1E703F0E003602BD9D1BA
:107230000021022328220846FEF74AFA089010B9D6
:10724000089890B9CEE703AB0093002321461A4675
:1072500008A800F0DFFC01460028F1D001222046FA
:10726000FEF750FA014618B90898FFF771FFB9E721
:107270002046089AFEF7F4F8002304462B7440F2E7
:107280000122234639490220FDF772FD00287FF4D0
:107290007DAFA7E7059DEDB1EB68072B1AD96B68A9
:1072A000C3B193F91030022B14D12846FEF710FB1E
:1072B000044678B18768B7F9020001F095FE61686D
:1072C0008046002619B1CB6849681E44FAE7B8F138
:1072D000000F01D1284686E798F8043023B12046F4
:1072E00000F086FF70B97DE701231A460846FEF7D5
:1072F000EFF900283FF476AF63684360606083680D
:1073000041221A70626800231AB1D16852680B4496
:10731000FAE7B8F80210994208D32146B7F90200FB
:10732000FDF75FFD00283FF731AF5BE7114B596870
:1073300000297FF457AFB6F5006FBFF453AF7988DB
:107340009A8108A840F2252219805C609E60ADF801
:1073500022200993FAF7ACFE18E76FF0850306A91F
:1073600004A80793FAF754FF10E700BF0000FFFFDF
:10737000FC020020B45000201FB50A4CB4F90000F4
:1073800000280DDC084B029300230193074B009368
:10739000032208234FF480610548F9F7C5FC2080DB
:1073A00004B010BDC45400205C22010859710008CB
:1073B000C450002038B50E4B142404FB003405469D
:1073C000638A63B10020FAF7DDF90A4BB0FBF3F0F2
:1073D000094B53F82530834206D800236382637C2F
:1073E00023F01003637438BD1B1A638238BD00BFDD
:1073F000C654002000879303085600202DE9F04171
:10740000012180461048114DFAF71AFD0024264646
:107410002746E0B2FFF7CEFF2B7C53B1414628460A
:1074200002F018FA2B7C834203D8B84284BF2E4660
:1074300007460134102C05F11405EAD10248FAF789
:107440002FFD3046BDE8F08148560020C65400208C
:107450000F2838B5044615D801210B48FAF7F0FC7F
:107460002046FFF7A7FF094B142000FB0435064810
:107470002C7C1CB1FAF714FD284638BDFAF710FD34
:10748000204638BD002038BD48560020C654002094
:107490002DE9F8430F280646884615461F469DF8F5
:1074A00020903FD8002A40D001212148214CFAF7F2
:1074B000C7FC002F4FF0140303FB064308BF4FF037
:1074C0000009802D88BF80225F828CBF1A741D74D2
:1074D000B9F1000F02D046F0100300E0334614204B
:1074E00000FB064441466374204602F09EF90146C3
:1074F00040B91022204608F02FFB227C414620464E
:1075000002F0CEF90020FAF73DF90B4BB0FBF3F097
:107510000A4B0744064843F82670FAF7C1FC204698
:10752000BDE8F8830020BDE8F8831046BDE8F88385
:1075300048560020C65400200087930308560020B8
:107540000021FEF7B7B9F8B50E4601784378174623
:1075500001F10802024405460830FDF787FE0446A3
:10756000E0B18368B5F902205A802A791A716A79E4
:107570005A71AA799A71B7424FF000013A464FF01A
:10758000010328BF32460846FEF7A2F8054620B997
:107590002046FFF7D5FF2846F8BD60602046F8BDBD
:1075A0002DE9F04F054685B0B0F9000001F01CFD53
:1075B000D5F80480D8F8044083464FF0000A1CB187
:1075C000E36864689A44FAE7BBF1000F05D14046CE
:1075D000FFF7B6FFC5F804B0D0E0B5F80C90B9F1EC
:1075E000000F42D1674FAE683B88D8F808000133DE
:1075F0003B80CAEB06039AB2BBF80230043B13444B
:1076000003F0F8039B1A1FFA83F909F104025146AB
:10761000FFF799FF034600283AD04268D2F808A045
:1076200076BAAAF800609AF8002062F03F028AF861
:1076300000203A8852BAAAF80220D8F80470002F25
:107640007CD0FA68B9680093C4EB0906964228BF5B
:107650001646201D344432465044A4B208F07EF948
:10766000A145009B6AD97F68E9E7D14580F0828017
:10767000BBF80260D8F80800AF68053E06F0F806CF
:10768000C9F10501721D5144FFF75DFF034628B99A
:107690006868FFF755FF00236B606FE042689268EF
:1076A000511D009179BA1180117861F01F0111709C
:1076B00034494F440988CAEB070A49BA4FEADA0A43
:1076C000518082F804A0D8F80470FFB1A1451BD006
:1076D000FA68A11889B2894513D2C4EB09041FFACC
:1076E00084F9C9EB0204B442B9680098019328BF39
:1076F00034462246494408F031F9A4B27F68019B20
:1077000005E07F680C46E0E7002400E03C46A64226
:1077100014D99FB1FA680193C4EB06089045009B09
:10772000B96828BF9046181944444246A4B208F0EC
:1077300015F9A642019B01D07F68EAE71946BBF91B
:1077400000000093FDF74DFB0028009B02DC18466B
:10775000FFF7F6FE002C9BD0AB8903951C44AC814F
:1077600040F2252302A8ADF80A30FAF7A1FCF9F798
:10777000A1FA03E04046FFF7E3FE6C6005B0BDE808
:10778000F08F00BF4C56002010B58268137803F0CC
:10779000F803C02B044606D0E02B0DD11379C26844
:1077A000DB00053A02E0C2680023043A6068214623
:1077B000806800F013F82046BDE81040FFF7C0BE17
:1077C000002203682BB119689A80DA801A60016080
:1077D000F7E7436070470021FEF76CB82DE9F04FE2
:1077E0008FB081460020924604911F468E68AA4DB4
:1077F000F9F7C8FFA94A834605F190082C4660684E
:1078000058B1A368C3EB0B03934206D90292FFF76A
:10781000E2FF2046FFF7D4FF029A24344445EED11C
:1078200099F800B009F1080307930BF108034B44E2
:10783000069399F80130029333885BBAC3F30A03C5
:10784000059373885BBAADF8263000209BB20A938B
:10785000F9F798FF002308901C4603936A68A8462E
:10786000002A00F02581D2680599914223D1EA8B44
:107870000A998A421FD12A7F93451CD16A7F0299B7
:10788000914218D15A4607990B9305F10C0008F064
:1078900033F80B9B78B9029A069905F1140008F0A9
:1078A0002BF80B9B38B97C4C039A242303FB02442E
:1078B000089BA3604EE014B96A6802B92C463BB13C
:1078C000A9689A68521A76498A4294BFA84698468F
:1078D000039B0133042B039305F1240501D0434698
:1078E000BCE784B9B8F1000F03D16E490320F9F762
:1078F0007BF9D8F804000028F7D0FFF76CFF40466A
:10790000FFF75EFF444600210223059A0846FDF773
:10791000DFFE6060002800F0DD8083680021002029
:10792000C3E90001089BA3605A46079904F10C00C3
:1079300008F014F8029A069904F1140008F00EF801
:107940009DF808306377BDF82630E383002384F880
:107950001CB0238425680FBB3379412B03D1053636
:107960000AF1FF331FE003F0E003602B06F1040689
:1079700018D10EAB204643F8047D50F8042F009335
:10798000D2680499042300F045F900287CD00D9AB0
:1079900028320AEB020306441B1A05E0053653465B
:1079A000002201E053463A466068C16803EB070EC7
:1079B0008E456AD81FFA87FE0EF1FF31194489B24D
:1079C0006DB1B5F804804145C0F08280B5F806C0BD
:1079D000E6457DD8C6456FD161456DD178E01FFA87
:1079E00083F80EF1FF314144DFF8C0A089B2AC4604
:1079F0000AEBCC05B5F806B0BBF1000F11D1ADB163
:107A0000E98021682960A5F804E0218C2560806860
:107A10004144174421849A1A3146384407F09EFFA6
:107A200004E00CF1010CBCF1340FE1D16368228C4D
:107A3000DB689A424ED1637F217F04F1140204F186
:107A40000C00FDF713FCF8B18368B9F902205A80E5
:107A500099F804201A7199F806209A7199F805206E
:107A60005A710023436063682BB15A680AB1134608
:107A7000FBE7586000E0606063680B4940F2012258
:107A80000220FDF775F910B96068FFF7A4FE2046E3
:107A9000FFF796FE1EE000BF50560020C0C62D0026
:107AA000FEFFFF7F251901080000FFFFE0560020C0
:107AB000002C7FF404AF01E7FFF78DFE2046FFF7AF
:107AC0007FFE3B46524604994846FFF787FE01E099
:107AD0002D6875E70FB0BDE8F08F00BF037823F085
:107AE0000F0343EA11130370437803F00F0343EAD3
:107AF00001114170704700000822014907F02EBFB4
:107B00009E2201081022002108F026B810B5082294
:107B10000949044607F0F0FE48B12378FF2B08D14D
:107B2000607800F00F00831E5842584110BD0120BC
:107B300010BD002010BD00BF9E22010873B5154680
:107B4000194A04460E46106851686B4603C32CB3AD
:107B5000637CDB0624D4227C802A1DD0402A1FD9D6
:107B6000D208D11F501C2944C2F10F02304407F043
:107B7000C3FEA8B9237CD9080D44725C15F8080C23
:107B800003F0070302A90B44424013F8083C1A42D1
:107B90000CBF0120002004E0012002E0204600E0AC
:107BA000002002B070BD00BF602201080023042A3B
:107BB00010B54370037016D0082A02D0022A26D1CD
:107BC00018E00B7883F0020303704B7843708B78D6
:107BD0008370CB78C3700B7903714B7943718B79C8
:107BE0008371CB7911E00B7883F0020303704B783B
:107BF00043700223FF240022C470FE2482700471AB
:107C00004271CA5C82710B445B78C37110BD184627
:107C100010BD00002DE9F74F1E464B6800920F463D
:107C2000D3F808A0D1F808B0019018B9C0490320D2
:107C3000F8F7DAFF019B1B68002BF7D0DA68272AD8
:107C4000F4D90BEB06089D6898F90130002B2B78CE
:107C500003F00F0343F060032B701BF8063003F0B2
:107C60001803ACBF02240324082B27D017D8002BFD
:107C700052D118F804102846FFF730FF08EB040132
:107C80004B7803F00F026B7813436B708978AA78F6
:107C9000E31C0A43AA7018F80320043429E0102BCF
:107CA0002AD0182B38D100212846FFF717FF6B7810
:107CB00023F00F036B700023AB702CE018F8043036
:107CC0009B099B0043F060032B706B7803F00F015E
:107CD000697018F8043003F00F0308EB04020B433B
:107CE0006B705178AA78A31C0A43AA7018F8032075
:107CF0000334EB7813430EE018F804102846621C96
:107D0000FFF7ECFE6B7823F00F036B700023AB7072
:107D1000EB70144600E0EB701BF806305B075CBFAD
:107D200018F80430AB711BF8063003F0030358BF9A
:107D30000134022B08D0032B08D0012B07D018F8F0
:107D40000430EB71013403E0402300E0FF23EB71CA
:107D500098F8013003F0400202F0FF0972B11806F2
:107D60004ABF98F802000020000913F0300905D03E
:107D7000FFF76EFB8146002800F0318298F8013051
:107D800003F07003302B42D00FD8102B1CD0202BC7
:107D900026D0002B40F08C8008EB0401102205F166
:107DA000080007F0DBFD103482E0502B3BD006D8F2
:107DB000402B7DD105F10800FFF7A4FE78E0602B91
:107DC00045D0702B62D073E005F10800FFF794FEF8
:107DD000082208EB040105F1100007F0BFFD34E0B4
:107DE00005F10800FFF788FE4FF0FF320023EA7428
:107DF0006FF001022A752B746B74AB746B750222E1
:107E000008EB040105F1160007F0A8FD3CE051461F
:107E100005F1100011F8082BFFF7C8FE05F1080066
:107E2000FFF76AFE44E0B9F1000F3FF4FFAE08220D
:107E300008EB040105F1100007F090FD99F81020FF
:107E4000494605F1080001F02BFD083430E0B9F196
:107E5000000F3FF4EBAE4FF0FF320023EA746FF0F7
:107E600001022A7508EB040102222B746B74AB74B7
:107E70006B7505F1160007F071FD99F81020494661
:107E800005F1080001F00CFD023411E0B9F1000F1A
:107E90003FF4CCAE514605F1100011F8082BFFF766
:107EA00085FE99F81020494605F1080001F0F8FC1C
:107EB00098F8013059070FD51A064ABF98F8020002
:107EC000002000F00F0013F00B0F05D0FFF7C0FAF1
:107ED0008146002800F0838198F8013003F00F03F9
:107EE0000C2B00F27C81DFE813F00D00160025005A
:107EF00042007A015100610082000D009400A6004A
:107F0000B800C60008EB0401102205F1180007F0C4
:107F100025FD1034D9E005F11800FFF7EDFD08222A
:107F200008EB040105F1200007F018FD3CE000BF5C
:107F30002519010805F11800FFF7DEFD4FF0FF32AB
:107F4000002385F823206FF0010285F8242085F8AE
:107F5000203085F8213085F8223085F8253002223E
:107F600008EB040105F1260007F0F8FC3DE09AF863
:107F700000109AF801200831514405F12000FFF764
:107F800015FE05F11800FFF7B7FD9EE0082208EB8B
:107F9000040105F1200007F0E1FC99F810204946A2
:107FA00005F1180001F07CFC08348EE04FF0FF3240
:107FB000002385F823206FF0010285F8242008EBC8
:107FC0000401022285F8203085F8213085F822301E
:107FD00085F8253005F1260007F0C0FC99F810203F
:107FE000494605F1180001F05BFC02346DE09AF897
:107FF00000109AF801200831514405F12000FFF7E4
:10800000D5FD99F81020494605F1180001F048FC0B
:108010005BE005F11800FFF775FDFF232B7618F8DC
:1080200004306B76611C0522414405F1230007F002
:1080300095FC063449E005F11800FFF763FDFF23C6
:108040002B7618F804306B76611C0322414405F14D
:10805000250007F083FC043437E005F11800FFF732
:1080600051FDFF232B7602236B7618F8043085F838
:108070002730013429E005F1180099F810A0FFF726
:1080800041FD99F81030402B84BF402389F810300F
:10809000FF232B7618F804306B7608EB040349466F
:1080A0005B78AB7699F81030EB7699F8102005F1F3
:1080B000580001F0F5FB211D0422414405F1240084
:1080C00007F04CFC063489F810A0009B13B9FB683C
:1080D0001B1B01E0009B283B5BBAAB801BF8063002
:1080E0005B077ED518F8043003F0F803F02B78D145
:1080F000019BBD68D3F800A0009BDAF808903444D7
:1081000004F1010815F804B04BB9009904230822C2
:108110000846FDF7DDFA002865D0826802E009F123
:10812000280200200BF00303022B14D0032B1FD0D6
:1081300015F808101170012B05EB040399785170A4
:1081400004D0D978917005341B790FE0DB780434C2
:10815000A3F5805318E015F80830A3F580535BBAF7
:1081600013802B19043499789170DB78D3700DE06B
:1081700015F808301909A1F5756149BA03F00F0324
:1081800002341180A3F575635BBA53801BF0040FB2
:1081900003D00021FDF78EFB25E02B5D9371A31C1E
:1081A0002C446178D17118B1F9680831C91A01E01D
:1081B0000099283949BA9180112189F806109288CE
:1081C000A9F8042018B1019AC0F804A0106053B1B6
:1081D0009C1B0C9B0C9A1B680833136001E0002069
:1081E00003E0204601E00024F3E703B0BDE8F08F90
:1081F0002DE9F04F4268D0F808909668D2680021C7
:1082000089B0824601230846FDF762FA029038B32E
:108210008568AB4960232B7006F1080B00236B7057
:108220001022584607F068FB38B15846FFF7E6F8C9
:10823000804610B1437CD90601D44FF00008337E4C
:10824000FF2B00F0628206F11800FFF7D7F807460F
:10825000002800F05A82437CDA0640F1568201E0A1
:10826000029858E2B8F1000F04D098F811301B07BB
:1082700003D15FB17B7C1C0708D06B7863F07F0370
:108280006B700023AB70032401E047460224316881
:108290003378727821F4704121F0FF011B01A9B9F4
:1082A00043EA121313F0FF0F2B7803D143F01803A6
:1082B0002B7036E043F010032B70737831781B0974
:1082C000621C43EA01132B5594B22AE05BB203F01F
:1082D00030011209114304F101010ED12B7843F052
:1082E00008032B7032688BB2317812BA8910C2F34E
:1082F000034242EA81122A5509E013432B553268A2
:1083000089B212BAC2F30342A31C6A549BB2326808
:1083100012BA120AEA549C1C01339BB20022EA549E
:10832000A4B2B379112B6DD1DAF8043058688368A0
:108330001A88B3F802E052BA92B222F00F0C1FFA78
:108340008CFC4FF2B0018C451AD19EFA9EF121F0BF
:108350000F010904090C614512D10322B271598839
:1083600049BA1FFA81FE198849BA89B20EEB011188
:1083700001F5AA61197099795970D979997026E037
:108380009EFA9EFE0EF47F4EBEF5704F04D1012280
:10839000B2715A8852BA0CE002F47F42B2F5704FC3
:1083A0000ED10222B2711A8852BA1A709A785A7093
:1083B000DA789A709A79DA70DA791A71052206E019
:1083C0000022B2719A791A71DA795A710622B1795A
:1083D00061F00F01C2F1080EB1711A44C168C3EB1C
:1083E000020CCEEB01018C4504D212F80E1002F8FB
:1083F000011BF3E7FDF7F4F92B7843F004032B702E
:10840000012303E0621C2B5594B200230393F379FC
:10841000402B07D0FF2B0AD0012B0CD12B7843F037
:10842000010302E02B7843F002032B7006E02B7867
:1084300043F00303F9E7621C2B5594B21022204944
:10844000584607F059FA18B96B7843F0400335E005
:10845000B8F1000F0CD06B7843F040036B7098F8C4
:10846000112010070AD0AB7843EA0213AB7005E085
:108470005846FFF74BFB002800F0408108AB002076
:10848000002163E9040199F80020082A00F2248100
:108490004FF48A71D140C90740F11E8109F10801EA
:1084A0001846FFF783FBDDE90423716930699942BF
:1084B00008BF904206D16B7843F030036B7021E027
:1084C000EE22010804AA59464046FFF737FB002870
:1084D000F1D13369B3F17F4F05EB04006B7840F0C5
:1084E0000381B28A52BA92B2B2F57E4F40F0FC805C
:1084F00043F020036B70022206F1160107F02EFAFA
:108500000234A4B2337EFF2B72D16B7843F00802A1
:108510006A70728BCABBF269BABB328CAABB727E1C
:10852000022A0FD1326A6AB9B28C5AB996F826205B
:1085300042B943F00B036B7096F827202A55631C51
:108540009CB2B4E0728C8AB996F8242072B943F0D8
:108550000A036B70737E2B55601C032206F1250104
:1085600015FA80F007F0FAF904349FE096F822201B
:10857000002A40F0948043F009036B70737E2B5502
:10858000601C052206F123012CE0B38BADF81030FE
:10859000F38BADF81230338CADF81430738CADF82A
:1085A000163004A8FEF72AFF002878D0437CDB06AB
:1085B00075D5027CF37E9A4271D16B7843F0040347
:1085C0006B70437C13F00F031EBFAA781343AB708C
:1085D000737E2B55631C9BB2B27EEA54A01C04220E
:1085E00006F1240115FA80F007F0B8F906345DE0D1
:1085F0001FB199F801303BB951E006F11800FFF7BF
:1086000085FA0028F5D14AE057B16B7843F00403AE
:108610006B707B7C13F00F031EBFAA781343AB7003
:1086200099F8001099F801200831494404A8FFF78F
:10863000BDFADDE90423716A306A994208BF9042AD
:1086400004D16B7843F003036B7030E004AA06F1A9
:1086500018013846FFF772FA0028F2D1336AB3F1F5
:108660007F4F05EB04006B780FD1B28C52BA92B2F7
:10867000B2F57E4F09D143F002036B70022206F17E
:10868000260107F06BF9023410E043F001036B7030
:10869000082206F1200107F061F9083406E02819E4
:1086A000102206F1180107F059F91034A4B2039B07
:1086B0001BB1631CB2792A559CB221460298FDF782
:1086C0008FF8DAF804105046FCF7B4FE029A4368BB
:1086D0005360426001201EE00821B9F902000091B8
:1086E0000022FCF799FBDEE643F010036B700822D2
:1086F00006F1100107F032F9083402E728191022B8
:10870000594607F02BF91034FBE6B8F1000F3FF49F
:10871000BCAD0027A9E509B0BDE8F08F10B508226F
:108720000949044607F0E8F848B12378FF2B08D13F
:10873000607800F00F00831E5842584110BD0120A0
:1087400010BD002010BD00BF9E220108F8B5B0F892
:10875000C631DB07044603D415490320F8F744FA71
:1087600000F5E0760121002504F5EE773046F9F7B3
:1087700067FB384684F8CB51F8F7B2F94FF4087329
:10878000A4F8F2310B4B0C49B3F90030C4F8F441B2
:1087900004F5F872384604F093FB3046F9F780FB95
:1087A0002946B4F9C401BDE8F840FCF741B800BF60
:1087B00025190108B823002080969800F8B5B0F874
:1087C000C631DB07044603D424490320F8F70CFA2A
:1087D00000F5E07601213046F9F732FB94F8CB3111
:1087E000022B03D8013384F8CB3116E0DD1E01F0F3
:1087F000BDF90123AB403B2BB0FBF3F505FB1300A8
:108800009EBF94F8CB31013384F8CB31092804D9C9
:108810003C2828BF3C20054600E00A2504F5EE77F9
:108820003846F8F75DF94FF40873A4F8F2310C49B3
:108830000C4BC4F8F4416943B3F9003004F5F87205
:10884000384604F03DFB3046F9F72AFBB4F9C40181
:108850000021BDE8F840FBF7EBBF00BF2519010878
:1088600040420F00B823002010B50446B0F91A00AA
:10887000FAF764FEB0F8C631DA0703D410490320D2
:10888000F8F7B2F9637E1B070BD4002005F068FDF2
:10889000A8B9B4F91A00FAF751FEBDE81040FFF785
:1088A00055BF10220749204607F026F80028ECD0D3
:1088B0002146B4F91A00BDE81040FBF7B9BF10BD5E
:1088C00025190108EE2201082DE9F04380468DB0FC
:1088D0001846894614461F46FFF720FF0546B8B9DB
:1088E00010230693029308AE07AB07900390009302
:1088F000019706AB32460DF116014748F9F745FFDF
:10890000002806DB069B102B0CBF3546002500E037
:1089100000253946204605F0D9FC0646002D74D0C6
:1089200030B93946BDF9160005F0D0FC0646E0B175
:10893000B6F91A00FAF702FE18B1B0F8C631DA0734
:1089400006D5737E03F03003302B08BF3D4600E0B0
:108950003D4645B93846FFF7E1FE002851D03D4677
:10896000002D3CD00EB1AF4204D02946204605F080
:10897000ADFC06462846FFF7D1FE58B326B1737EFC
:1089800003F03003202B25D107AE3046FCF758FC0E
:108990000822074689F80020A918404606F0DEFFA5
:1089A00098F8003083F0020388F80030CCB9BC425C
:1089B00015D036F91400FAF7C1FD48B1B0F8C63148
:1089C000DB0705D50CAB03EB440434F9140C1FE0B2
:1089D0000134ECE7737E03F03002202A03D100203B
:1089E00016E0204614E003F00703032B03D1042113
:1089F0003046FBF7BDFE32464946404605F0E6FCF0
:108A000006E0FBF7A1FD0546AAE70028A2D08FE704
:108A10000DB0BDE8F08300BF8423002070B50E4682
:108A200018B911490320F8F7DFF80029F9D0B0F997
:108A30001A00FAF783FD00F5EE7504462846F8F7AC
:108A40004FF84FF40873A4F8F2310849084BC4F802
:108A5000F44104F5F87271432846B3F90030BDE8DB
:108A6000704004F02DBA00BF2519010840420F00E4
:108A7000B8230020F8B507460D46164610211A46C1
:108A80002120FBF730FC044660B1806800236DBAFA
:108A90000822877043710371C370C580314610444A
:108AA00006F05CFF2046F8BD2DE9F04F85B080460A
:108AB0000E9E7578022D0F4692461C4640F0B880F7
:108AC0000823009300226B440321FCF7A5F900283A
:108AD000C0F2AE804046FAF731FD2146814640465D
:108AE00005F0F4FBBAF1870F04464ED0BAF1880FB7
:108AF00040F09E80B9F8C631D90740F19980DDE990
:108B00000223D6F80CB0D6F808A05B4508BF524542
:108B100040F08E80002800F08B80B578012D2ED09B
:108B20000BD3022D40F08480404607F1080105F088
:108B3000F5FB4846FFF70AFE7AE009F5E0790121E6
:108B40004846F9F77DF9F6883D4B04F13807384679
:108B500076BAB3F90080B6B2F7F7C2FF394940F2EE
:108B60001223013EA4F84E303846434604F14C022D
:108B7000714304F0A5F94846F9F792F95BE007F173
:108B800018014046FAF720FD52E0B9F8C6319A07BD
:108B90004ED0B378002B4BD1083710222A493846E3
:108BA00006F0AAFE002843D0D4B1637E9B060CD504
:108BB000D4F88C20D4F8903052EA030105D0F16843
:108BC000B0688B4208BF824234D1B6F80690B9F142
:108BD000000F05D13946404605F0A0FB4D462AE07E
:108BE000F3882BB384B9032300930F9A109B394663
:108BF000404605F0FDFA0446E8B1324600F18C0328
:108C000052F8080F516803C3637E0E4823F0300307
:108C100043F030036376F188094B49BA89B2414386
:108C2000B3F9003004F1840204F1700004F048F953
:108C3000002500E00125284605B0BDE8F08F00BF03
:108C4000B823002000879303EE22010813B58A7829
:108C50004B78402A01D8022B00E0032B0ED1862846
:108C60000ED1C878CB88C0F300145BBA00949BB2D5
:108C7000083100F00F00FEF70BFC01E0002000E0DF
:108C8000012002B010BD000008B50146074800F001
:108C9000CCFD48B910220649044806F02DFE0028F4
:108CA000024818BF002008BD004808BD80580020B9
:108CB000EE22010838B50446E1B1012380221449AF
:108CC000B0F9C401FAF758FCA0B104F5E0752846E4
:108CD0000121F9F7B5F8B4F8C63143F00403A4F85C
:108CE000C6314FF4E163A4F8CC312846BDE83840E2
:108CF000F9F7D6B8B4F8C631B4F9C401044923F081
:108D00000403A4F8C631BDE83840FAF75DBC00BFE3
:108D1000CE22010808B510220449054806F0ECFDF2
:108D20000028034808BF002008BD00BFEE2201084C
:108D3000805800202DE9F0470024054600F1160771
:108D40004FF00109A2464FEAD40804F0070617F8CD
:108D5000083009FA06F633420AD0E0B2FEF778FB93
:108D600080F810A017F8083023EA060607F8086014
:108D70000134102CE7D10026AC695CB12368AB61EB
:108D80006368A168B3F9C401FAF71EFC2660666047
:108D9000A660F1E710222146284606F0DDFE2C6190
:108DA000BDE8F0872DE9F04F87B003F1080A029083
:108DB0005046039117461E46FFF766FF04460028FB
:108DC00000F0B480F3885BBA9AB21AB942F2107319
:108DD0008382ABE0DFF860918382103F4FF00008A0
:108DE000002F70DD08F11003039AD518D35C032B14
:108DF00002D0222B4AD05EE00298FAF79FFB6B78F4
:108E00000190042B42D105F1100B08224949584624
:108E100006F072FD002839D02A7CFF2A04D16A7C32
:108E200002F00F02022A31D0EA7851062ED413063E
:108E30002CD46A6852B359460298FAF737FCAA78DC
:108E400004905946D9F80800059200F003FD059AF0
:108E5000824209D8D9F808305B7C9A4204D1D9F80B
:108E60000430019A9A4207D0334B986820B11022FF
:108E7000324906F041FD48B92F4B5A6832B9019A80
:108E80005A60049A9A60A2691A60A361AB783F2B7A
:108E90006B7801D8022B00E0032B0CD1EA7804F1A7
:108EA0001603C2F3C001012002F0070200FA02F229
:108EB000585C02435A546B7808EBC3081FFA88F8D1
:108EC000A7EBC3078CE773885BBA9BB22361B288B8
:108ED00052BA43EA02432361DAF80000DAF80410D8
:108EE000234603C356F8100F7168022203C3002102
:108EF00004F1160006F030FE0023A361A58A104B92
:108F000004F11C0630465D43F7F7EAFD40F22323E7
:108F100063860C4B6463B3F9003004F130022946D8
:108F2000304607B0BDE8F04F03F0CABF07B0BDE858
:108F3000F08F00BF9E220108B8580020EE220108E1
:108F400000879303B82300202DE9F0418846C1082B
:108F5000064614460831069A22201F46FBF7C3F93D
:108F60000546A0B18068002164BA01714171C480D6
:108F7000867080F80380EA6800F10804083A204609
:108F800006F0EAFD32463946204600F089FC2846C4
:108F9000BDE8F08170B505460E46144618211A4604
:108FA0002320FBF7A0F980B183686ABA2D0C6DBA53
:108FB00076BA5A809D80DE8022689A606268DA60A4
:108FC00054F8082F1A6162685A6170BD054BB3F9F5
:108FD0000020904204D01AB90122188059801A71D9
:108FE000704700BFC4580020034BB3F900208242F1
:108FF0000CBF184600207047C458002008B518B9A7
:1090000007490320F7F7F0FDC31C133013F8012FB5
:109010001AB98342FAD1012008BD002008BD00BF63
:10902000251901082DE9F0410C46154698460646DB
:1090300018B926490320F7F7D7FD11B1CB8A002BC9
:10904000F7D02DB1EB8A002BF3D00CB1A28AB2BBC2
:1090500006F1680718220021384606F07DFD5CB154
:109060002368042B03D06FF06900BDE8F08118225B
:109070002146384606F072FC06F1800718220021CE
:10908000384606F069FD7DB12B68042BEBD12846EC
:10909000FFF7B4FF18B16FF01500BDE8F08118229A
:1090A0002946384606F05AFC24B1E28A04213046AB
:1090B00005F0B0FAA6F898800020BDE8F081AB8AF0
:1090C000002BC5D09A42C3D0E5E700BF251901089F
:1090D0002DE9F04188B090460E461A460E9F044690
:1090E00018B111B1B8F1000F03D12E490320F7F7E1
:1090F0007BFD836E002B50D008AD01A945F8183DCB
:109100002B4605F09FFA002849DB0198C368984573
:1091100005D20021FCF7CEFB6FF068003FE0042190
:10912000FCF753F90028E0D0D0F8088047B11822A6
:109130002946384606F012FCB8F800305BBAFB82CC
:10914000D4F88030E3B1B8F80030B4F896205BBAB8
:109150009BB29A4206D001980021FCF7ABFB6FF05E
:1091600046001CE0843410220F49204606F0C4FB60
:1091700030B1102203A9204606F0BEFB0028EAD138
:10918000019B30469968DA6806F0E8FB01980021F7
:10919000FCF790FB019BD86801E06FF07C0008B001
:1091A000BDE8F08125190108EE2201082DE9F04102
:1091B0000F4686B090461D46044628B9002B7CD148
:1091C00042490320F7F710FD0AB10029F8D0ADB1EC
:1091D000EB8A13B96FF0150074E02846FFF70EFF15
:1091E0000028F7D12B68042B5ED16CB1B4F87C2039
:1091F00042B1AB8A33B19A4204D0EBE7D4F8803065
:10920000002B54D0A36EF3B918220021684606F053
:10921000A3FC2F4A138803EB03166FEA86466FEA16
:1092200096460133B6B21380ACB1A4F87E6015B98E
:10923000D4F8803000E02B68A36632460421204633
:1092400005F0E8F907E0182204F168016846B4F86F
:109250007E6006F083FB25B904F18005B4F89640E2
:1092600000E0EC8A009A2B680AB9009301E09A4268
:10927000B0D10023394642461846FCF729FA074682
:10928000C0B13146224600F025F9014618B93846EA
:10929000FCF710FB0EE011232A46694605F036FA6A
:1092A00000280FDD08380DE06FF069000AE06FF06C
:1092B0007F0007E06FF00B0004E0002A88D000294F
:1092C00086D17DE706B0BDE8F08100BF2519010811
:1092D000CA5800200021FCF7EDBAF8B5074684898A
:1092E0000E46154600204DB900230822B96800F04B
:1092F00075FA96F91030022B25D10DE0BD42F3D05E
:10930000B542F1D02346AA89A96800F067FAEB6854
:109310006D681C44A4B2E6E702194FF6EE739A4258
:10932000C4BF013080B2B168113420440023202230
:10933000083180B200F052FA4FF6FF73984203D022
:10934000C04380B2F8BD0020F8BD000070B5102207
:1093500098B000210DEB020006F0FEFB4D4B05938B
:109360004D4B1B88ADF81C3040F20523ADF80A3098
:1093700008216FF0850308A80393F8F77DFF04A97F
:109380000420FBF7A9FF6846F8F773FFBDF8023029
:109390006FF400721344032BF5D8DFE803F0023BAF
:1093A0007575019D2846FCF793FA044608B92846CE
:1093B00067E00221FCF709F8064618B9374903208F
:1093C000F7F712FC606830B190F91030042B02D12D
:1093D000C368082B06D0042208212046FCF792F926
:1093E00000284DD0002385682374EB885BBA9BB2BC
:1093F000002B45D022463146FFF76FFF4FF6FF7333
:1094000098423DD1698849BA234640F2012289B287
:10941000042031E0019E304696F91050FCF758FACE
:10942000044608B930462CE0406826460028C5D0DE
:1094300090F91030042B07D0FCF74AFA0346F8B134
:10944000706040681E46F1E7FCF742FAC0B18268DE
:1094500070600023C16840680B440028FAD15BBAF1
:1094600093806B1C08BF63680A4908BF93F91050CA
:1094700040F2022223462846FBF77AFC002882D1DC
:109480002046FFF727FF7EE702A96846F8F7C0FEEF
:1094900079E700BF0000FFFFFC020020251901084A
:1094A00010B5044668B161B190F91030042B0BD1AE
:1094B0004268FFF712FF50B1A36840BAD88000207D
:1094C00010BD6FF00D0010BD6FF04C0010BD6FF0BF
:1094D000010010BD38B50D461446042308220021B2
:1094E000FCF7F6F838B1836800226DBA64BA1D80C3
:1094F0005C809A71DA7138BD1FB50A4CB4F900303E
:1095000063B9094A0193094B02920093052208238B
:109510004FF480610648F7F707FC2080B4F900009B
:1095200004B010BDCC5C0020682201084D930008F7
:10953000CC58002010B5044601784278054806F062
:1095400013FC6188044849BA89B2BDE8104006F0AE
:109550000BBC00BF6C22010889220108F8B5044643
:109560009DF8245025701E4605F0070310250F4670
:10957000657006989DF8281015460AB1002F68D02E
:1095800018B1002E69D13046F8BD23B1022B02D0AC
:109590000DB9002873D0A17080B39DF82030E3701E
:1095A00002289DF82130237104D0082816D0002805
:1095B00051D120E002463249304606F09DF918B9F3
:1095C000237823F020032370637843F0080363704B
:1095D000737863713378A371072040E01C236370B4
:1095E000221D06F1080313F8011D02F8011F9E4217
:1095F000F9D10D2033E005201DB9F8BD0320002D61
:109600003DD0431C9DF81C2022549DF81D20E2549F
:109610000230022D03D0082D0CD0E5B9F8BD6378D7
:1096200063F07F0363707A782254431C3A78E254E3
:109630000230F8BD637863F03F03637007F10803FD
:10964000044413F8012D04F8012BBB42F9D1083072
:10965000F8BD3846F8BD0020F8BD63B90DE075B11E
:10966000BDF81C20BDF820309A42CAD1237843F0BF
:1096700040032370CDE7022B8AD1A1708DE7F8BD9E
:109680009C220108427802F00C03082B07D00C2B17
:1096900007D0CBB90178490614D4032302E007238D
:1096A00000E00D2312F0C0020CD00178490658BF2B
:1096B0000233802A01D1981C7047C02A04D103F1DB
:1096C00008007047184670470020704770B501B118
:1096D0001AB926490320F7F787FA437803F00C03F9
:1096E000082B07D103785C0617D5C378137003796C
:1096F000537012E00C2B07D103785B060FD5C378AB
:109700001370037953700AE013B16FF0150070BD48
:1097100003785E06F9D4032302E0072300E00D235B
:10972000447814F0C00411D005786D0605D4C65CE9
:1097300016705D1C0233455D5570802C08D1C25CEB
:109740004A70034402205B780B7070BD204670BDE8
:10975000C02CDAD1034401F1080213F8010B02F81E
:10976000010D8A42F9D1082070BD00BF25190108FA
:1097700008B501B11AB918490320F7F735FA43784B
:1097800003F00C03082B09D1C378137003795370CD
:1097900043794B7083790B70022008BD0C2B0ED1DE
:1097A000C378137010F8043F537001F1080310F8E8
:1097B000012F03F8012D8B42F9D1082008BD3BB9D8
:1097C000037813F0400F14BF6FF01500002008BDA0
:1097D0006FF0150008BD00BF25190108F0B51AB3D8
:1097E000DC0705D511F8014B013A204492B2013350
:1097F000570801EB47054C1C03350234AC4207D037
:1098000014F803EC14F8026C06EB0E263044F4E76F
:109810001A44D30703D511F8173000EB0320030CCB
:1098200080B201D01844FAE7F0BD30B54B68456806
:1098300004680A689D4208BF944209D1C568CB6894
:1098400084688A689D4206BF94420120002030BD92
:10985000002030BD30B510B3E1B188421CD00138D2
:109860000139002210F8015F11F8014FA54202F101
:10987000080303D1DAB2802AF4D10FE085EA0401AB
:10988000D8B20B060AD40132D2B249008242C9B220
:10989000F7D130BD084630BD802030BD104630BD08
:1098A000802A28BF8022F8B5D50814462A460646E5
:1098B0000F4606F053F863070ED0A4EBC504725DA3
:1098C000FF23C4F1080403FA04F422EA04027255E7
:1098D0007B5D1C4014437455F8BD10F8013F43B143
:1098E0008B42FAD100230370437813B1013005F0A5
:1098F0008BBD1046704700002DE9F04707468AB03F
:1099000008B90020A8E00029FBD000204FF0FF3468
:1099100006462346054631F810E0BEF1000F07D198
:10992000B3F1FF3F13BF013503B201252DB20BE0A8
:10993000B3F1FF3F08D0B4F1FF3F01D0B54201DDE4
:109940002E461C464FF0FF3301300828E3D1581C47
:1099500004D0601C7DD0B54202DD7AE0601C03D0EB
:10996000012ED8BF4FF0FF343D4800256B46E84636
:109970004FF03A09AC4203D183F80090A5194EE0AC
:1099800015B183F80090013311F815E01EF0F00FC7
:109990004FEA450C17D04FEA1E1A0EF00F0E10F8C2
:1099A0000AA010F80EE083F801E001EB0C0E83F83A
:1099B00000A09EF801E04FEA1E1E033310F80EE0EF
:1099C00003F801EC21E0BEF1000F10D010F80EA05A
:1099D0009E460EF802AB01EB0C0A9AF801A04FEA82
:1099E0001A1A10F80AA083F801A073460DE001EBE3
:1099F0000C0E9EF801E01EF0F00F1FBF4FEA1E1E76
:109A000010F80EE083F800E001338C4401359CF837
:109A100001E00EF00F0E10F80EE083F800E0072DC5
:109A200003F10103A6DD611C05D03444082C02BFFC
:109A30003A2119700133002103F8011BC8EB03031D
:109A400093423FF65EAF4146384606F077FC384613
:109A500002E02E461C4683E70AB0BDE8F08700BF4F
:109A60000E23010810B5017801F0F003602B8AB0D5
:109A7000044603D009091B4806F076F9227863787A
:109A8000110149B21B0901F030001943C2F38102F0
:109A90000343C9B2144806F067F92168134809BAAC
:109AA000C1F3130106F060F9A188E379A2791048A7
:109AB00049BA89B206F058F9282204F1080168462B
:109AC000FFF71AFF01460B4806F04EF9282204F171
:109AD00018016846FFF710FF0146074806F044F9F1
:109AE0000AB010BD1F2301083C2301086D230108A3
:109AF00082230108AF230108C32301082DE9F8439D
:109B00001546814613480F4604F0E6F9002D08BFBC
:109B10001025002407F1FF38A74218D00E4804F0A2
:109B2000DBF9661C19F8040004F0BEF9B6FBF5F386
:109B300005FB13630BB1A04507D1084806F09EF959
:109B4000A04502D0304604F0BBF93446E4E7BDE856
:109B5000F88300BFDC230108142E01089D4701088B
:109B60000146014802F076BFD05C0020124BF0B5F0
:109B700093E83400D8681E691C6084EA050122F06D
:109B800000424A4082EA420280EA5000504059694D
:109B9000D86040F3000782EA802239404A4004EB53
:109BA00012249A609A693E40604044F30004754074
:109BB00014405D606040F0BDD05C0020F8B50E46FA
:109BC0001D464FF47A730446174600211A46304664
:109BD00002F06EFE002802DA4FF0FF30F8BD069B5F
:109BE000E360089B2361079B63610023A361099BDA
:109BF000A56084E8C000E36101212846F7F774FC02
:109C00000028E9DB0121E068F7F76EFC0028E3DBC0
:109C100001216069F7F768FC0028DDDB012120697C
:109C2000F7F762FCC017F8BD8269C1690132826131
:109C3000014806F099B800BFE523010808B505F012
:109C40008DF8034905F092F905F02CFA08BD00BF24
:109C5000BE9F823F38B5044680680D46F7F708FD81
:109C6000E068F7F70EFD2A4621792068BDE8384004
:109C700002F092BE38B5044680680D46F7F701FD44
:109C8000E068F7F7F5FC2A4621792068BDE83840FE
:109C900002F082BE70B50446164640690D46F7F7DD
:109CA000E7FC002E2946204603DDBDE87040FFF7A3
:109CB000D1BFBDE87040FFF7DDBF38B5044640694D
:109CC0000D46F7F7D5FCA068F7F7DBFCE068F7F77F
:109CD000D8FCA868F7F7D5FCE868BDE83840F7F786
:109CE000D0BCF8B51E460023836105460C461746D6
:109CF0008B61AB69B3420DDAA3699E420ADD394636
:109D000028460122FFF7C6FF012239462046FFF709
:109D1000C1FFEEE721462846FFF7CFFF0023AB61E6
:109D2000A361F8BDF8B51E460023836105460C46C5
:109D300017468B61AB69B3420FDAA3699E420CDD13
:109D4000394628464FF0FF32FFF7A4FF4FF0FF32AD
:109D500039462046FFF79EFFECE729462046FFF7ED
:109D6000ACFF0023AB61A361F8BDF8B51E4600232C
:109D7000836105460C4617468B61AB69B3420EDA28
:109D8000A3699E420BDD394628464FF0FF32FFF7AC
:109D900081FF012239462046FFF77CFFEDE721468F
:109DA0002846FFF78AFF0023AB61A361F8BDF8B531
:109DB0001E460023836105460C4617468B61AB693E
:109DC000B3420EDAA3699E420BDD394628460122D2
:109DD000FFF760FF4FF0FF3239462046FFF75AFF8A
:109DE000EDE721462846FFF768FF0023AB61A3613A
:109DF000F8BD00000C4B0146186882689368013B6F
:109E0000002B10B4936005DA9469A34208DBCBB24F
:109E10000A2B05D01368581C1060197010BC7047CD
:109E200010BC06F0FDBC00BF8C02002008B53E202F
:109E3000FFF7E0FF2020FFF7DDFF034B1B6898686A
:109E4000BDE8084005F0B8BB8C0200202DE9804831
:109E500085B0814600AF0E469246FFF7E7FFB04659
:109E60000AF1FF340025C6EB0803A342F5DA844B60
:109E7000186841684B68013B002B4B6004DA06F020
:109E800005F8002804DAE8E70B685A1C0A6018781D
:109E90000D2801D00A280FD100240D2088F8004099
:109EA000FFF7A8FF0A20FFF7A5FF4645D5D03346A8
:109EB0002246254620462BE0082801D07F280DD1D8
:109EC0004645D0D0082008F8015CFFF793FF20201A
:109ED000FFF790FF08F1FF3B082003E008F1010BBA
:109EE00088F80000FFF786FFD846BCE7222913D187
:109EF0005C781CB35C2C25D001331C788C42F7D1E4
:109F0000597820291AD80135197811B303F8010BB3
:109F100019782029F8D9E9E7272906D1E8E74B1C69
:109F2000497822290AD02029EDD91C785C2C1946C1
:109F3000F5D1591C5B780132002BF0D1514805F066
:109F40009DFF8AE79C1C9B780132002BF6D02346AC
:109F5000D3E7002D81D0AB000E3323F00703EB468F
:109F6000ADEB030D6C464DF82510304690F800E03F
:109F700003460130BEF1000FF8D0BEF1220F02D02F
:109F8000BEF1270F00D1013344F8213018460133C8
:109F900090F800E0BEF1000FF8D101318D42E5D11B
:109FA000201FBAB150F8043FA3B1194613F801EBD2
:109FB000BEF1000FF5D0BEF15C0FF6D191F800E0D4
:109FC000BEF1000F04D091F801E001F801EBF5E7D4
:109FD000013AEAD12C4B2268FB60C7F808900023B5
:109FE00007F1080151F82380B8F1000F0DD10133BA
:109FF000022B16D0F4E711463B607A6006F034F885
:10A000007A683B6830B108F10C08D8F800000028E5
:10A01000F1D1ECE7D8F808301BB121462846984723
:10A020002CE02168194806F01FF8054610BB184AB5
:10A030001849194805F098FE184805F01FFF124B03
:10A04000C7F80890FB602C4607F1080353F824502A
:10A050000DB10C3503E00134022CF5D10EE00C35C6
:10A0600055F8181C0029F6D055F8142C0A4805F0AC
:10A070007BFEF4E721680A4805F076FEDD46ECE653
:10A080008C020020F9230108E025010812240108B0
:10A0900017240108232401082B240108993D0108F5
:10A0A0003524010808B503F0ADFE002008BD08B551
:10A0B000F6F7FCFE002008BD012810B506D10020EF
:10A0C000F7F760FB04460146074805E0486805F0DD
:10A0D0009BF904460146054805F046FE2046FFF779
:10A0E0003FFD002010BD00BF642601088A2601083C
:10A0F00008B5FFF73BFD0146024805F035FE00209C
:10A1000008BD00BFB61F01080146062814D8DFE8C5
:10A1100000F004060B0D0F110900094800E0094882
:10A1200005F022BE0848FBE70848F9E70848F7E7CA
:10A130000848F5E70848F3E7084805F015BE00BFF2
:10A14000AC260108B0260108B6260108BE26010883
:10A15000C3260108C6260108C9260108CF26010822
:10A16000102828D00BD803281BD003D8E8B1022828
:10A1700015D07047052816D006281AD07047262813
:10A1800015D004D8162818D0202818D070472A28AF
:10A1900017D02B2817D0272818D10D4814E00D48C8
:10A1A00012E00D4810E00D480EE00D480CE00D489F
:10A1B0000AE00D4808E00D4806E00D4804E00D48AF
:10A1C00002E00D4800E00D4805F0CEBD704700BF2D
:10A1D0005B270108D4260108E4260108F1260108BE
:10A1E000072701080F27010814270108272701085E
:10A1F000392701084E270108722701087D27010829
:10A2000008B50146034805F0AFFD0348BDE8084026
:10A2100005F034BE8C270108B127010813B50446A8
:10A2200001A8FBF70DF820B1BDF90400031B58424B
:10A23000584102B010BD00001FB504AB012403F863
:10A24000012D00940022FAF70DFE002804DA0948D7
:10A2500005F014FE20460BE09DF80F10064B074A50
:10A260000748002914BF1146194605F07DFD00205E
:10A2700004B010BD3F2B01083C2B01089D4701088D
:10A280005B2B0108A0F13003DAB2092A04D9A0F14E
:10A290006103DAB2052A01D8184670474138C3B2C3
:10A2A000052B88BF4FF0FF30704700007FB50C468C
:10A2B000082105460DEB0100164604F0D1F808B957
:10A2C00011480FE0009002AB002221462846FAF721
:10A2D000C9FD00280ADA0D4805F046FD2046FFF7C3
:10A2E0003FFF0B4805F0CAFD01200BE0094805F0CF
:10A2F0003BFD2046FFF734FF32462946064805F06D
:10A3000033FD002004B070BD722B0108E52B01085D
:10A310009D470108FB2B0108092C01087FB5064663
:10A3200010460D4605F070F804AB012403F8010D4A
:10A330000022009429463046FAF794FD00280ADAF4
:10A340000C4805F011FD2846FFF70AFF0A4805F002
:10A3500095FD20460CE0094805F006FD2846FFF76C
:10A36000FFFE9DF80F200648314605F0FDFC002059
:10A3700004B070BDE52B01089D470108FB2B0108C7
:10A38000222C01087FB506460D461046531E13F8D1
:10A39000014F1CB1303C092CF9D908E00A222146B2
:10A3A00006F026FA0390013009D11C481CE0102267
:10A3B000002106F01DFA03900130F6D00124039B22
:10A3C000B3F5803FF1D202230093002203AB29466C
:10A3D0003046FAF747FD00280ADA114805F0C4FCB8
:10A3E0002846FFF7BDFE0F4805F048FD012012E0AA
:10A3F0000D4805F0B9FC2846FFF7B2FE31460B4880
:10A4000005F0B2FC039924B1094805F0ADFC002029
:10A4100001E00848F9E704B070BD00BF3B2C01081B
:10A42000E52B01089D470108FB2B0108892C010839
:10A430009F2C010867500108022808D0FF2808D087
:10A44000054A064B01280CBF1846104670470448C1
:10A4500070470448704700BFB82C0108A72C0108BA
:10A46000AF2C0108B42C010870B5012988B00C4646
:10A47000164609D104230093002207AB2921FAF7DD
:10A48000CBFC051E0EDA09E0022905D1F9F7AEFA78
:10A49000079008B1012505E06FF08505154805F026
:10A4A000EDFC24E0E4B266B11C220021079805F01F
:10A4B00053FB2046FFF7C0FF01460F4805F054FC50
:10A4C00015E02046FFF7B8FF079AD3685168049358
:10A4D0009368039313690293019113680B440093EB
:10A4E000936952690146054805F03EFC3546284609
:10A4F00008B070BDC02C0108FA2C01081B2D010802
:10A500002DE9F04790B002AF00260446FE70F9F73F
:10A5100015F821460546CB4805F026FC0823009394
:10A520003246FB1802212046FAF776FC061E1CDB99
:10A5300006EB460808F1070323F00703E946ADEBF5
:10A54000030D0DF1080AC04805F00EFC334607F173
:10A5500008024146504603F057FF0146BB4805F04C
:10A5600003FCBB4805F000FCCD460223002200930B
:10A5700011463B1D2046FAF74FFC002803DBB98843
:10A58000B44805F0F1FB0223009300223B1D262175
:10A590002046FAF741FC002803DBB988AE4805F0F5
:10A5A000E3FB0223009300223B1D06212046FAF71D
:10A5B00033FC002803DBB988A84805F0D5FBA84880
:10A5C00005F0D2FB082300930022FB18032120464C
:10A5D000FAF722FC061E1EDB06EB460808F107030D
:10A5E00023F00703E946ADEB030D0DF1080A9D4882
:10A5F00005F0BAFB334607F108024146504603F026
:10A6000003FF0146984805F0AFFB9848CD4605F09A
:10A61000ABFB012600E00026022300930022BB1DB5
:10A6200010212046FAF7F8FB002804DBB7F90610E2
:10A630008F4805F099FB012300930022BB1C1821D1
:10A640002046FAF7E9FB002808DB8A4805F08CFB76
:10A65000B878FFF759FD7E4805F086FB012300938B
:10A660000022FB1816212046FAF7D6FB002803DB50
:10A670007978814805F078FB4FF00108CDF800802B
:10A6800007EB0803002220212046FAF7C5FB00282B
:10A6900010DBCDF80080FB1C00221F212046FAF7BA
:10A6A000BBFB002806DBFB78434503D17978734870
:10A6B00005F05AFB6A4805F057FB0123009300227E
:10A6C000FB1C13212046FAF7A7FB002808DB97F8AC
:10A6D0000380B8F1010F03D1694805F045FB4646F8
:10A6E000012300930022FB1C14212046FAF794FB5F
:10A6F000002808DB97F80380B8F1010F03D1614807
:10A7000005F032FB4646012300930022FB1C152175
:10A710002046FAF781FB002808DB97F80380B8F1A0
:10A72000010F03D1584805F01FFB46460123009353
:10A730000022FB1C12212046FAF76EFB002808DBE2
:10A7400097F80380B8F1010F03D1504805F00CFBD6
:10A750004646012300930022FB1C19212046FAF7EC
:10A760005BFB002808DB97F80380B8F1010F03D1E9
:10A77000474805F0F9FA4646012300930022FB1CE6
:10A780001F212046FAF748FB002808DB97F80380D2
:10A79000B8F1010F03D13F4805F0E6FA4646012320
:10A7A00000930022FB1C1E212046FAF735FB0028EF
:10A7B00008DB97F80380B8F1010F03D1364805F0A4
:10A7C000D3FA4646012300930022FB1C2321204696
:10A7D000FAF722FB002808DB97F80380B8F1010F95
:10A7E00003D12E4805F0C0FA4646FDB1B5F8C811B0
:10A7F0002B4805F0B9FA95F8CA112A4805F0B4FAC1
:10A80000B5F8C631D80702D5274805F0ADFAB5F836
:10A81000C631990702D5254805F0A6FAB5F8C63124
:10A820005A0702D5224805F09FFA01262046FEF776
:10A83000DBFB002840D00379002B3DD01D4805F0FC
:10A8400093FA3AE0C62D0108FD2D01080D2F0108ED
:10A85000152E0108D22D0108E12D0108ED2D01086A
:10A86000F52E0108F92D0108072E01080B2E01080D
:10A87000172E01082A2E0108332E0108472E010841
:10A880005A2E0108642E01086E2E0108782E010848
:10A89000822E01088C2E0108932E01089D2E01089E
:10A8A000AC2E0108B62E0108BE2E0108C42E0108E8
:10A8B000CA2E0108D42E010816B1394805F054FA01
:10A8C0000223009300223B1D05212046FAF7A4FA3B
:10A8D000002803DBB988334805F046FA002D58D02C
:10A8E000B5F8C6313049314813F0800F304B08BFFE
:10A8F000194605F039FA2A4805F036FA05F5E076EA
:10A9000010222C49284604F0F7FF002831D02A48AD
:10A9100005F02AFA2822294607F11000FEF7ECFF7D
:10A9200008B36A7C254807F1100105F01DFA0822DA
:10A930002349284604F0E0FF38B12B78FF2B06D1DD
:10A940006B7803F00F03022B01D11E4800E01E4874
:10A9500005F00AFA2B7CDB0708D52B78FF2B0CBF00
:10A960001A481B4800E01B4805F0FEF90C4805F0AA
:10A97000FBF93835B542C3D1174805F07FFA0022FC
:10A9800001212046FFF770FD002202212046FFF73B
:10A990006BFD114805F072FA3837BD46BDE8F08707
:10A9A000F52E0108DB2E0108B72D0108022F010842
:10A9B000BD2D0108EE220108102F01081D2F0108EE
:10A9C0009E2201082C2F0108322F0108392F01087F
:10A9D000462F0108512F01089D4701082DE9F04F2E
:10A9E000012889B0804602AF0E460BDC07F1080053
:10A9F000FAF726FC18B1B7F90800FFF781FD00242B
:10AA000000F06EBC4868431E13F8014F3CB3303C65
:10AA1000092CF9D93168A94805F0A6F93068FFF783
:10AA2000EFFB3168A64805F09FF93168A54805F0AD
:10AA30009BF93168A44805F097F93168A34805F0FF
:10AA400093F93168A24805F08FF93168A14805F003
:10AA50008BF9A14805F012FA012400F041BC04F082
:10AA6000D3FC05B22846FFF7D9FB002800F0198473
:10AA7000B8F1020F04D12846FFF742FD00F030BCC8
:10AA80009649B06805F0F0FA002840F02482B8F149
:10AA9000040F01DC30681BE2D6F80C809048D6F831
:10AAA00000903669414605F0DFFA10B932460221BE
:10AAB0000CE041468B4805F0D7FA0028F6D0414615
:10AAC000894805F0D1FA28B9324603212846FFF714
:10AAD000EDFBACE34146854805F0C6FA10B93246B5
:10AAE000002151E04146824805F0BEFA0028F6D028
:10AAF0004146804805F0B8FA10B93246262143E0B5
:10AB000041467D4805F0B0FA10B9324606213BE0D7
:10AB100041467A4805F0A8FA0028F6D04146784820
:10AB200005F0A2FA0028F0D04146764805F09CFADC
:10AB3000044610BB304604F067FC07F118030222FC
:10AB400023F8100D1021009228462246FAF78AF9C0
:10AB5000002807DA6C4805F007F96C4805F004F99D
:10AB60006B4877E76B4805F0FFF8684805F0FCF89C
:10AB7000B7F908206848294607E34146674805F0C9
:10AB800073FA28B9324605212846FFF7FBFB4EE34E
:10AB90004146634805F068FA0446002863D131460F
:10ABA000604805F061FA08B9002332E031465E489A
:10ABB00005F05AFA0028F7D031465C4805F054FAFF
:10ABC00008B9012325E03146594805F04DFA00281F
:10ABD000F7D03146574805F047FA08B9022318E084
:10ABE0003146554805F040FA0028F7D03146534821
:10ABF00005F03AFA08B905230BE03146504805F054
:10AC000033FA0028F7D031464E4805F02DFAB8B98E
:10AC1000062301263B720022009607F10803182143
:10AC20002846FAF71FF9002812DA474805F09CF881
:10AC3000387AFFF769FA364805F020F934464FE3D1
:10AC40003146424805F010FA0028E1D0404801E7BB
:10AC50002946404805F088F8387AFFF755FA2C481D
:10AC600005F00CF93CE341463B4805F0FDF910B90D
:10AC7000324616210EE04146384805F0F5F910B984
:10AC80003246202106E04146354805F0EDF928B965
:10AC9000324627212846FFF741FBC8E241463148AA
:10ACA00005F0E2F90446002840F0978031462E482E
:10ACB00005F0DAF9002859D1012363E0A83601082C
:10ACC000883301084D3401083B360108363201084B
:10ACD0003B330108BD360108E8360108423001085F
:10ACE000003001080530010810300108072701086D
:10ACF0001A3001080F2701081F300108233001080E
:10AD0000273001082E300108E52B0108272701080C
:10AD10009D470108FB2B0108222C01083430010853
:10AD2000EC1901083C300108AC2601081635010871
:10AD3000B0260108B3190108BE26010840300108F9
:10AD4000C9260108463001088F300108B6260108DF
:10AD50004E300108AE300108D6300108DE3001085F
:10AD6000EB300108F9300108622F01083146B04884
:10AD700005F07AF900289FD03146AE4805F074F905
:10AD8000C8B900234FF001083B720022CDF80080C3
:10AD900007F108032A212846FAF764F8002812DA96
:10ADA000A54804F0E1FFA54804F0DEFFA44805F043
:10ADB00065F8444694E23146A24805F055F900286A
:10ADC000DFD0A14846E6A14804F0CEFF9B4804F03E
:10ADD000CBFF324629469E48D7E141469D4805F0C3
:10ADE00043F90446002872D1304605F009FB4FEACA
:10ADF000500909F1070323F00703EA460E28ADEBDB
:10AE0000030D83460DF1080801D1934806E0102890
:10AE100001D1924802E0202804D1914804F0A4FF17
:10AE2000002117E0302801D18E48F7E7402801D1F2
:10AE30008D48F3E7802801D18C48EFE78C4804F077
:10AE400093FF17E0421C12D04A0800EB031008F8E9
:10AE5000020002318B450FD9705CFFF713FA7218AC
:10AE600078605078FFF70EFA7B685A1CEAD1814867
:10AE700005F004F8012428E0CDF8009043460022B4
:10AE80002B212846F9F7EEFF002807DA6A4804F07C
:10AE90006BFF794804F068FF6948E9E76B4804F004
:10AEA00063FF754804F060FF2946744804F05CFFB6
:10AEB0004546C144A94505D015F8011B704804F06A
:10AEC00053FFF7E75E4804F0D9FFD54608E248464D
:10AED000FFF796F9C0E56B49B06805F0C5F8044680
:10AEE00000286AD1B8F1030F01D1316827E0A8F139
:10AEF0000308B8F1010FD6F80C9022D06249D6F8B9
:10AF000000A0484605F0B0F820B9D6F810904FF0F0
:10AF1000020A17E05D49F06805F0A6F820B9D6F8F6
:10AF200010904FF0010A0DE05949F06805F09CF8C7
:10AF300020B9D6F810904FF0000A03E0514655486A
:10AF4000ABE182462F2140224846FEF7C6FC431E55
:10AF5000802B0646494628BF402607F108005FFAC5
:10AF600086FB03F031FC00283AD0B8F1010F07D07E
:10AF70003B7AFF2B04D1BAF1010F07D0464869E5AF
:10AF8000BAF1020F14BF4023412300E040235A4688
:10AF900007F108012846F8F7EFFA18B93F4804F01E
:10AFA000E3FE59E54FF0FF334361836132462B46A0
:10AFB00049463B4804F0D8FE92E13A49B06805F0B2
:10AFC00053F80446B8B9B8F1030F02D131683648D6
:10AFD00063E1F66807F10800314603F0F5FB08B9B4
:10AFE000324837E507F108012846F8F7EDFA2A4616
:10AFF00031462F48C9E02F49B06805F035F80446BE
:10B00000002869D1B8F1030F02D131682A4844E120
:10B01000F06804F0F9F9A0F5A063B3F57B4F06469C
:10B020004ED34FF6FF724FF4A06124489FE000BF5B
:10B03000013101083C300108E52B010872270108A5
:10B040009D470108AC26010804310108FB2B0108CB
:10B05000092C010817320108343101085131010867
:10B060006E3101088C310108AA310108C83101088C
:10B07000E6310108003201087D2701081B32010872
:10B08000461F010832320108823201088A32010863
:10B090009432010836320108C1320108ED3201084C
:10B0A00010330108373301083B3301089C32010893
:10B0B0005E3301088433010888330108A333010893
:10B0C0002846F8F73BFA08B98848C3E4A0F8C861F5
:10B0D0002A463146864858E08649B06804F0C4FFE5
:10B0E000044670BBB8F1030F17D08349F06804F031
:10B0F000BBFF002800F0EA808049F06804F0B4FF4C
:10B10000002800F0E6807E49F06804F0ADFF0028DA
:10B1100000F0CA80F1687B48BAE04FF0FF0919F0EF
:10B12000010F04D0224601212846FFF79DF919F0AE
:10B13000020F3FF491AC224602212846FFF794F912
:10B140008AE47149B06804F08FFF044600BBB8F18F
:10B15000030F02D131686D489FE0F06804F054F9A4
:10B16000FF28064606D96A484FF6FF72002104F010
:10B17000FBFD71E42846F8F7E1F908B9654869E490
:10B1800080F8CA6164482A46314604F0EDFDA7E024
:10B19000D6F80880614998F80030D6F800902D2B39
:10B1A00008BF08F1010840460CBF0026012604F044
:10B1B0005BFF10B93246132136E05949404604F08E
:10B1C00053FF10B9324612212EE05649404604F092
:10B1D0004BFF10B93246142126E05349404604F093
:10B1E00043FF10B9324615211EE05049404604F095
:10B1F0003BFF10B93246192116E04D49404604F094
:10B2000033FF10B932461F210EE04A49404604F090
:10B210002BFF10B932461E2106E04749404604F094
:10B2200023FF30B9324623212846FFF705F80446AC
:10B2300056E04249404604F017FF044678B92846D4
:10B24000FDF7D2FE08B93E4804E426B1012303719C
:10B2500029463C481CE0067129463B4818E03B491A
:10B26000404604F001FF0446A8B92846F8F766F9FD
:10B2700010B93748FFF7EEBB2EB10121F8F775F989
:10B280002946344804E03146F8F76FF93248294638
:10B2900004F06AFD24E03148494604F065FDFFF7FB
:10B2A000DBBB2F48FFF7D6BBB8F1040F0AD04FF035
:10B2B000020905222B49306905F010F9B0FA80F433
:10B2C00064092CE704464FF0020930E74FF0FF090C
:10B2D00001E04FF00109B8F1040FEAD1002421E7A1
:10B2E00020461C37BD46BDE8F08F00BFCB330108B8
:10B2F000E533010808340108B42C01080E340108B4
:10B30000D6200108113401084A3401084D340108DF
:10B310006734010895340108B5340108DE340108AA
:10B32000E6340108EE340108F6340108FE34010861
:10B3300002350108073501080F3501081C350108E1
:10B34000213501083F350108663501088E350108B1
:10B3500096350108CA350108023601083B36010856
:10B360008E2F0108403001082DE9F04F87B006AF5D
:10B370000546884691469A4605F042F8284485429B
:10B38000A0EB050413D010F801392F2B05D1601C58
:10B39000284404F039F806460BE03A2B01D02E2B56
:10B3A000EDD1284605F02CF80026044601E00024E3
:10B3B000264604F1080323F00703ADEB030D0DF15E
:10B3C000180B621C0021584604F0C6FB2946224691
:10B3D000584604F0C3FA404605F012F8594616489C
:10B3E00003F0F2F9D0B1144D10244146134803F094
:10B3F000EBF9D0B1114B10220021360603910292D5
:10B400000193CDF810A0009623462A4649460C48E1
:10B41000F7F7B0F80437BD46BDE8F08F03F0FCFF46
:10B420006A230360074D0424DFE703F0F5FF6A2376
:10B4300003600422044BDFE7FC5C0020EC5C00208E
:10B4400084230020105D00200C5D002001282DE9E0
:10B45000F34105460C4603D17A48F7F735FABBE0CD
:10B4600002281AD14968784804F0FEFD002800F04F
:10B47000B1806168754804F0F7FD08B97448B8E018
:10B480006168744804F0F0FD014620B96D48F7F793
:10B4900060F97148ADE07148ABE053DD49686A4836
:10B4A00004F0E2FD58B16168684804F0DDFD30B198
:10B4B0006168684804F0D8FD08B1694899E0032D37
:10B4C00025D16168634804F0CFFD054690B9A068B6
:10B4D00003F09AFF04B22046F9F7BEFE214628B1D8
:10B4E0005848F7F736F921465E4800E05E4804F018
:10B4F0003BFCA2E0A1685D4803F066F90546002820
:10B500006CD0102259494F48F7F705F964E0052D32
:10B5100018D161684C4804F0A7FD002868D1E168A3
:10B52000534804F0A1FD0546002861D101A8F9F7B0
:10B5300087FE012831D14FF0FF33BDF90420216986
:10B54000A0683DE0072D3ED161683F4804F08CFDC6
:10B55000C8B9E168464804F087FDA0B9616945486B
:10B5600004F082FD054670B901A8F9F769FE0128CB
:10B5700013D1A069BDF90480A668276903F044FFD0
:10B58000424603461AE061682F4804F06DFD20B979
:10B59000E168374804F068FD08B1374829E061697F
:10B5A000364804F061FD05460028F6D1A069A6687A
:10B5B000276903F029FF4FF0FF3302B239463046C6
:10B5C000FFF7D2FE39E0092D12D161681E4804F060
:10B5D0004BFD90B12A480CE000252EE003F01CFF43
:10B5E0006A230360042227491648F7F794F824E0F9
:10B5F000254804F043FC01251FE0E1681C4804F0E5
:10B6000033FD0028E6D161691C4804F02DFD0028B7
:10B61000E0D1E169174804F027FD05460028D9D19B
:10B62000A069A668276903F0EFFE8046206A03F050
:10B63000EBFE0FFA88F20346C0E7284602B0BDE8E9
:10B64000F08100BF84230020323201083733010823
:10B6500002390108963901089C390108BD390108F1
:10B660003A3A01088A3A0108BE3A0108FC5C002017
:10B67000DC3A0108523C0108E03A01085B3C010851
:10B6800022370108105D00205F3C010813B5044615
:10B6900001A8F9F7D5FD20B1BDF90400031B5842FC
:10B6A000584102B010BD000000F00700072813D871
:10B6B000DFE800F00406080A0C0E121008480CE03F
:10B6C00008480AE0084808E0084806E0084804E09E
:10B6D000084802E0084800E0084804F045BB00BF05
:10B6E000AF3C0108BC3C0108C93C0108D63C01083C
:10B6F000E33C0108F03C0108FD3C01080A3D01085B
:10B7000000F03000202805D0302805D0102805D1C1
:10B71000044804E0044802E0044800E0044804F05F
:10B7200023BB00BF173D01081A3D01081F3D01085A
:10B73000BF3D0108F0B5012893B006460D4607D17C
:10B740006B4804F09BFB6B4804F098FB002005E07D
:10B750004968694804F088FC30BBF1E702F0E8FD75
:10B760000446002800F0C1802822214608A8FEF7E0
:10B77000C3F8237EB4F91A60054604F110021821BB
:10B7800002A802F041FE3246034629465B4804F017
:10B79000EBFA607EFFF788FF607EFFF7B1FF584845
:10B7A00004F06CFB2046D9E7012E40F39680022E70
:10B7B00074D06968534804F057FC0446002857D1F8
:10B7C000023E012E02D0022E0CD022E008A8F9F78A
:10B7D00037FD012898BFBDF92060AF6888BF2646B5
:10B7E00000251CE0AF6808A8394602F0EDFF28B933
:10B7F000A86803F009FEEF6806B2F1E702A8F9F7BE
:10B800001FFD012898BFBDF90860ED6888BF264676
:10B8100005E0A86803F0F8FDEF682D6906B2304630
:10B82000FFF734FF08B9384805E0394608A802F0A8
:10B83000CBFF20B9354804F021FB012455E04DB180
:10B8400008212A460DEB010002F00AFE034610B95A
:10B850002F48F0E72B460022009208A902AA3046A2
:10B8600002F0C6FC08B92B48E5E739462A4812E041
:10B8700069682A4804F0F8FB044678B9AD6808A85E
:10B88000294602F0A1FF0028D4D008A9204602F0E2
:10B8900045FD2348294604F067FA26E069682148F7
:10B8A00004F0E2FB0446C0B902F042FD2146054621
:10B8B00055B119B1B1F91A0002F030FD284602F075
:10B8C00037FD29460546F3E719B1B1F91A0002F030
:10B8D00025FD154804F048FA07E02B6800931A4646
:10B8E0001946124804F040FAA7E7204613B0F0BD0D
:10B8F000233D0108723D01089D250108C13D010855
:10B900009D47010832320108D63D01089C320108EA
:10B91000F63D0108213E0108513E01083733010878
:10B92000833E010840300108AC3E0108CB3E0108CF
:10B9300070B501288AB00C460DDD486803F064FD3F
:10B9400005B22846FFF7A2FE30B92168164804F078
:10B950000BFA012025E00025144804F08FFA144862
:10B9600004F08CFA002002F0FBFC0446C8B1B4F9E4
:10B970001A600DB1AE4212D1282221466846FDF769
:10B98000BBFF314602460B4804F0EEF9607EFFF73C
:10B990008BFE607EFFF7B4FE074804F06FFA204686
:10B9A000E1E70AB070BD00BF773F0108903F010892
:10B9B0008D3D0108C43F01089D47010808B50146B7
:10B9C0000B4804F0D1F90B4804F058FA0A4804F087
:10B9D00055FA0A4804F052FA094804F04FFA0948A7
:10B9E00004F04CFA0848BDE8084004F047BA00BF2C
:10B9F000D23F01082E4001083840010846400108A6
:10BA0000A0400108B4400108C54001080C4AF0B547
:10BA100014880830260AE5B200238B4209D2FF2C95
:10BA200085BFC718C654C5547D708CBF023301331F
:10BA3000F3E781BF138809181B0A01F8013CF0BD28
:10BA4000880200202DE9F0430D4685B0022104460E
:10BA5000F9F7BBFC032107462046F9F7B6FC07B10E
:10BA600008B9274845E08668264AB388F4881288D2
:10BA70005BBA9BB264BA9A42A4B239D12249234B31
:10BA80000A881B889A4203D9944203D3012307E012
:10BA9000944204D39C428CBF0023012300E0002386
:10BAA00033B3BF68D0F80C901948944298BF013264
:10BAB00007F1080898BF0A8028224146FDF71CFFBD
:10BAC0004FF47A72B388B5FBF2F102FB1155029183
:10BAD0000395FA7901925BBA02469BB249460094FB
:10BAE0000C4804F041F9404602F042FC012003E01A
:10BAF000094804F0C3F9002005B0BDE8F08300BF99
:10BB0000E0400108880200203C5D00203E5D0020EE
:10BB1000145D0020174101085A4101082DE9F04F3A
:10BB200099B081460C461022002114A804F014F8A4
:10BB300081231593994BB9F1010F1B88ADF85C3047
:10BB40003BDDB9F1020F00F0C281606803F05CFCDC
:10BB5000051ED4BF4FF000084FF0010808F10103A3
:10BB60004FEA830754F82330089308F10203D8BF43
:10BB70000325994505DDE319586803F045FC049059
:10BB800001E00423049308F10303994505DDE3195B
:10BB9000986803F039FC064601E04FF47A7608F124
:10BBA0000408C14505DD2744F86803F02DFC099021
:10BBB00000E00995049B002B03DA2068FFF7FEFEE6
:10BBC0003FE04FF0FF3225210898FDF786FE04B2D2
:10BBD000621C089910A808BF002402F0F5FD08B9FE
:10BBE0006F482CE008226F4910A803F085FE50B181
:10BBF0009DF84030FF2B05D19DF8413003F00F0335
:10BC0000022B00D0A4B10EA8F9F71AFB44B100280A
:10BC100000F05881BDF938309C4240F0538106E075
:10BC2000012802D1BDF9383001E05F4807E01C4629
:10BC300014A90320F9F750FB002804DA5B4804F04C
:10BC40001DF901204BE1F4F7D5FE4FF47A737343ED
:10BC50000D9300220023CDE90A010027CDE9062338
:10BC60004FF0FF332E460593BA46BB46013E731C88
:10BC70004F4A00F006814E4B19884E4B1A8801320C
:10BC800092B21A80049B00938020002302F0EEF908
:10BC9000804698B104998068FFF7B8FE10AA002189
:10BCA000404602F043FA814640B1ACB14FF0FF3359
:10BCB00008220021F9F70CFD814618B93E4804F02E
:10BCC000DDF8D3E7836800221A705A705A719A71AE
:10BCD0001A715A8083685C800020F5F753FD4B464B
:10BCE000804640F2022235490220F9F741F80C90D3
:10BCF00038B9334804F0C2F80C994846F9F7DAFD30
:10BD0000B4E7304A00230EA801F0F4F800282DDB38
:10BD1000BDF83A2040F201239A4220D10020F5F7E5
:10BD200031FDDDF83C90C8EB000841464846FFF77E
:10BD300089FE002183444846F9F7BCFD059B474531
:10BD400038BF4746434528BF43460593DDE90623F0
:10BD500012EB080243F10003CDE906231AE00F4B72
:10BD600019880EA809B2F6F7DFF913E0164804F0B7
:10BD700085F80FE00EA8F6F779FA002828DDBDF85F
:10BD80003A304345F6D1114803F0EEFF00210F98F9
:10BD9000F9F790FD40F20128ECE700BFFC0200201B
:10BDA000774101089E22010890410108DE41010807
:10BDB000880200203E5D0020D02F01080000FFFF18
:10BDC000FE41010840420F002942010836420108A5
:10BDD0001EB100210D9801F049F8099B0AF1010AF2
:10BDE000534502D0002E7FF441AFF4F703FE0899CB
:10BDF00080463C4803F0B8FFBBF1000FC6EB050AD4
:10BE000038DD5246DDE90601D31703F071F9DDE9AB
:10BE10000A23B8EB02029046334AB8FBF2F16423DE
:10BE200002FB11828DE806000C905A46514603FB36
:10BE30000BF32E4893FBFAF3C3F1640303F094FF72
:10BE40004FF47A72B7FBF2F002FB107E01900C986F
:10BE50000C9BB3FBF2F302FB1300009005980599CD
:10BE6000CDF808E0B1FBF2F102FB1102204803F02B
:10BE70007BFF03E051461F4803F076FF4FF0000AB6
:10BE8000F4E61D4B00211980138814A90133032007
:10BE90001380F9F743FA40F201240EA8F6F7E6F909
:10BEA00000280BDDBDF83A30A342F6D1134803F069
:10BEB0005BFF00210F98F9F7FDFCECE7BBFA8BF074
:10BEC00040090CE021460E4803F04EFFB9E66368D6
:10BED000089304274FF000080325049753E619B090
:10BEE000BDE8F08F7B42010840420F0097420108F5
:10BEF000E0420108144301083E5D0020364201087B
:10BF00004B4301089368013B002B10B4936008DA9F
:10BF10009469A34202DBCBB20A2B02D110BC04F01D
:10BF20007FBC1368581C10601970C8B210BC7047F1
:10BF300010B503F069FA04B22046F7F7FFFA20B90A
:10BF4000064803F09BFF012010BD2046F9F7B4FE20
:10BF50002146034803F008FF002010BD714301088B
:10BF60008D43010830B58FB00D4603F04DFA2946D8
:10BF7000C4B2684602F028FC18B90E4803F07EFFF0
:10BF800010E000231A4669462046F9F711FF58B918
:10BF90002822694604A8FDF7AFFC22460146064860
:10BFA00003F0E2FE012003E0044803F0DDFE002080
:10BFB0000FB030BDBB430108EA4301081C4401082F
:10BFC00010B503F021FAC4B22046FAF7DDFD10B92E
:10BFD0002146084804E0FAF7D4FE214620B9064875
:10BFE00003F0C2FE012010BD044803F0BDFE002096
:10BFF00010BD00BF40440108694401089044010895
:10C0000030B58BB003F000FAC5B22846FAF7BCFD94
:10C01000044620B90A4803F031FF01200EE0383011
:10C0200000F08CFD282204F108016846FDF764FC4D
:10C030002A460146034803F097FE00200BB030BDAE
:10C04000B0440108D844010830B58BB003F0DCF9E6
:10C05000C5B22846FAF798FD044620B90A4803F00D
:10C060000DFF01200EE0383000F0AEFD282204F173
:10C0700008016846FDF740FC2A460146034803F0E4
:10C0800073FE00200BB030BDB04401081745010815
:10C0900070B58CB003F0B8F9C6B23046FAF774FD4B
:10C0A0000125044620B9134803F0E8FE28461EE0A7
:10C0B000114A90F82730B2F9000094F82820019234
:10C0C00094F82620009205FA03F340F6011204F1D9
:10C0D000380100F049FD282204F1080102A8FDF70B
:10C0E0000BFC32460146054803F03EFE00200CB032
:10C0F00070BD00BFB04401089A4A002058450108AD
:10C1000008B504490020F9F7EFFF034803F0B6FE35
:10C11000002008BD442201089945010813B5234CAD
:10C12000234803F0ABFEA36900932269A36821684A
:10C13000204803F019FEE36900936269E3686168CF
:10C140001D4803F011FEA36B0093226BA36A216AC2
:10C150001A4803F009FEE36B0093626BE36A616ABD
:10C16000174803F001FEA36D0093226DA36C216CB0
:10C17000144803F0F9FDE36D0093626DE36C616CAC
:10C18000114803F0F1FDA36F0093226FA36E216E9F
:10C190000E4803F0E9FDE36F0093626FE36E616E9A
:10C1A0000B4803F0E1FD002002B010BD305000202C
:10C1B000AE450108F145010823460108554601082E
:10C1C00087460108B9460108EB4601081D470108EA
:10C1D0004F4701082DE9F041514C524892B003F00D
:10C1E000C3FD63780BB9504800E05048504DDFF86C
:10C1F0006C8103F0B9FD286809218268FFF782FE8F
:10C2000028680A218268FFF77DFE4A4803F0ACFDEA
:10C21000002606EB08031B790BB9434800E04348AE
:10C22000434F03F0A1FD2868092182683036FFF7EB
:10C2300069FE902EEDD13868394D82680A21FFF7EA
:10C2400061FE38680A218268FFF75CFEF4F7D2FBD2
:10C25000637806460F46002B5DD0B5F88A0095F846
:10C2600080302978B5F92C200290B5F8880001902B
:10C27000D5F88400008800902F4803F075FDE86E23
:10C28000296F801B61EB0701002871F1000305DBBA
:10C290002A4A002302F02CFF064600E00026236A0B
:10C2A000274993F98C50282208A8FDF725FB94F81C
:10C2B000363094F83270228E069613F0020F214B1E
:10C2C000214918BF1946638F059394F838300493B9
:10C2D00094F82630039394F8273001269E4025EAEF
:10C2E000E5758DE86200194B1949022F08BF0B460E
:10C2F0000146184803F038FDE46964B1611D282245
:10C3000008A8FDF7F9FAE369E28A0146124803F04A
:10C310002BFD2468F1E7002012B0BDE8F08100BFDA
:10C32000A04F00208D4701089E470108A247010841
:10C330008C020020A6470108B547010840420F00C3
:10C34000A84F0020622F01083C30010886470108F1
:10C3500081470108F947010850480108F04A0020C8
:10C3600038B50546084603F04FF8C4B22046FAF740
:10C370000BFC28B921460B4803F0F6FC012038BD20
:10C38000083015B1FAF770FE01E0FAF774FE064BBB
:10C39000064A0748002D08BF1A46214603F0E4FC70
:10C3A000002038BD40440108864801088148010842
:10C3B0008D48010838B50C4603F026F8C5B228466A
:10C3C000FAF7E2FB28B929460B4803F0CDFC01201F
:10C3D00038BD90F83630094923F0020343EA44039C
:10C3E00080F83630064B0748002C08BF194603F08A
:10C3F000BBFC002038BD00BF404401089D47010838
:10C4000067240108B6480108012838B505460C46DE
:10C4100003DCBDE83840FFF7DDBE6349606803F028
:10C4200023FE0028F5D0032D09D16049606803F090
:10C430001BFE88B9A068BDE83840FFF779BD042D20
:10C440000AD15B49606803F00FFE28B9E168A06873
:10C45000BDE83840FFF786BD5649606803F004FE2A
:10C4600030B9032D7AD1A068BDE83840FFF7A8BDE8
:10C470005149606803F0F8FD00BB042D6ED14F49AF
:10C48000A06803F0F1FD20B9E068BDE83840FFF78F
:10C49000B7BD4B49A06803F0E7FD20B9E068BDE8EF
:10C4A0003840FFF7D1BD4749A06803F0DDFD002803
:10C4B00054D1E068BDE83840FFF7EABD4249606802
:10C4C00003F0D2FD58B9032D48D14049A06803F0CC
:10C4D000CBFD002842D1BDE83840FFF711BE3C49F2
:10C4E000606803F0C1FD20B9032D37D1A168012098
:10C4F00007E03849606803F0B7FD30B9032D2DD14E
:10C50000A168BDE83840FFF72BBF3349606803F0EE
:10C51000ABFDD0B9022D21D03049A06803F0A4FDB5
:10C52000E0B9052D1AD12E49E06803F09DFD08B948
:10C53000012105E02B49E06803F096FD014668B94A
:10C540002069BDE83840FFF735BF2749606803F030
:10C550008BFD18B9BDE83840FFF7E0BD234803F074
:10C560008DFC234803F08AFC224803F087FC224814
:10C5700003F084FC214803F081FC214803F07EFC99
:10C58000204803F07BFC204803F078FC1F4803F0B0
:10C5900075FC1F4803F072FC1E4803F06FFC1E4838
:10C5A00003F06CFC002038BDDE480108B42401080B
:10C5B000E3480108E8480108EB4801084030010859
:10C5C000F3480108F84801080C1B0108FE4801085F
:10C5D00081480108864801084230010802490108E3
:10C5E000622F01083C30010808340108064901089F
:10C5F0001E4901085849010891490108CA49010822
:10C60000034A01083A4A01087D4A0108C64A01085E
:10C61000034B0108284B0108734B0108F8B5064687
:10C620000F46044623783D1B412B35440ED17B48F1
:10C6300003F024FC282D40F2EF80601CFDF712FA75
:10C640001022A5F1290104F12900E1E013F0C00F47
:10C6500006D1734803F012FC102229462046D7E089
:10C6600003F0F802C02A11D16E4803F007FC2188BC
:10C670006D4849BAC1F30A0103F076FB61886B4843
:10C6800049BA89B203F070FB0434CBE7E02A17D132
:10C69000674803F0F3FB2188634849BAC1F30A01F4
:10C6A00003F062FB6188614849BA89B203F05CFB20
:10C6B0002179604803F058FB1022691F601DA7E034
:10C6C00003F0E003602B40F0A7805B4803F0D6FB4B
:10C6D000237803F01803082B09D002D863B9574810
:10C6E00008E0102B05D0182B06D1554802E055481C
:10C6F00000E0554803F0C2FB237803F0040303F085
:10C70000FF0213B122B1514800E0514803F0B6FBDB
:10C71000237803F00303022B06D0032B06D0012B52
:10C7200014BF4C484C4802E04C4800E04C4803F031
:10C73000A5FB637859060BD54A4803F015FB6378CF
:10C7400003F03003102B15D00ED8C3B9464814E0BF
:10C75000464803F009FB637803F03003102B09D03F
:10C7600002D863B9424808E0202B05D0302B06D10F
:10C77000404802E0404800E0404803F07FFB637817
:10C7800013F0080F03F004031FD05BB13C4803F023
:10C7900075FB637803F00303013B022B8CBF394820
:10C7A000394822E0394803F069FB637803F003035A
:10C7B000022B06D0032B06D0012B14BF344835487A
:10C7C00013E0354811E035480FE03BB1344803F041
:10C7D000CBFA63789A070AD1324806E0324803F070
:10C7E000C3FA63789B0702D1214803F047FB94F911
:10C7F0000130002B08DAA1782C4801F00F0209095A
:10C8000003F0B2FA032000E00220291A102220448B
:10C81000BDE8F840FDF772B9F8BD00BF9F4B0108B5
:10C82000B84B0108D24B0108EF4B0108034C01083B
:10C830000F4C0108314C01083F4C01084D4C0108D8
:10C84000AB4C0108734C0108924C0108DE4C010806
:10C85000D34C0108ED4C0108FA4C0108024D0108C7
:10C860000B4D0108154D01083B4D01088A4D01088B
:10C87000B14D0108724D0108544D0108634D010886
:10C88000C14D0108F44D0108264E0108334E010840
:10C89000674E0108834E01089E4E0108B94E0108FB
:10C8A000D34E01082A4E0108FD4E0108284F010809
:10C8B0002DE9F74FDFF8DC8001922C24444308EB8C
:10C8C0000407054697F829B0584689461E46F4F7EE
:10C8D000B7FB012D824604D8019A02FB06F5A84257
:10C8E00003D82B490320F4F77FF958467968F4F709
:10C8F000B3FB58F80440002323604FF00108636045
:10C90000BB466363A363E363236457F838305A1C60
:10C910000FD0012118460193F4F7E6FD019B9BF827
:10C920002810184608F10108F4F77AFEB8F1050F4F
:10C93000EBD1BAFBF5F5731E013DB9F1010FA5620C
:10C94000E3620ED00AD3B9F1020F0ED10023A36126
:10C95000E361236843F06003236006E046F260036E
:10C9600001E047F27003A361E3614FF400436364A5
:10C9700041F211132362236843F001032360A06A8C
:10C9800000FB0660BAFBF0F003B0BDE8F08F00BF1B
:10C9900025190108404F0108012838B50AD8032994
:10C9A00008D82C23013143430F4D03EBC1042C590C
:10C9B000013403D10D490320F4F716F9EC58E36A6A
:10C9C0009A424FF02C0303FB00F000EBC10005EB93
:10C9D000000188BFE26A0B7903F10C0304EB8304C6
:10C9E00088BF92B2626038BD404F01082519010826
:10C9F00030B5036845688468C168056085EA04024B
:10CA000023F00043534083EA430381EA510183EA60
:10CA1000010242F3000583EA8223C2600169426990
:10CA200029402A404C4053404460836030BD036835
:10CA300023F0004363B9436853B9836843B9C368BB
:10CA400033B9542149224E234FF0590C80E80E107F
:10CA50007047000038B503694360436983608369A8
:10CA600001600446C3600F4801256B1E03F00303F9
:10CA700005F0030254F8233054F8221083EA93732C
:10CA800000FB035301354B40082D44F82230ECD114
:10CA90002046FFF7CCFF2046FFF7AAFF013DFAD161
:10CAA00038BD00BF6589076C2DE9F34185680446F0
:10CAB0001DB919490320F4F797F842784368934069
:10CAC000C268C2EB05086A0093424FF000072CBF12
:10CAD00082608360478038BF5D088668FDF746F84E
:10CAE000711BB0FBF1F202FB11000544B4F91030E8
:10CAF000E5604FF47A7245446A43019304F11C03E4
:10CB00000093A262E7623B4604F1300000F0E2F9D4
:10CB100002B0BDE8F08100BF2519010810B54288B8
:10CB200003789A42044600D313B96369A069984711
:10CB30002046BDE81040FFF7B7BF00008268436899
:10CB40009A4210B5044603D806490320F4F74CF87E
:10CB50003030F3F7C5FF6368A3602046BDE810409E
:10CB6000FFF7A2BF25190108F8B50C46174606467F
:10CB70009DF818109DF81C201D461BB91049032074
:10CB8000F4F732F803FA01F00E4B9842F6D800237E
:10CB900063802270656026826170FCF7E7FFC5EB59
:10CBA0008503B0FBF3F202FB13000544E560A560CA
:10CBB00026822462E7832046BDE8F840FFF774BF71
:10CBC00025190108FEFFFF7F3030F3F789BF438846
:10CBD000013343807047000010B501884288044645
:10CBE00049BA52BA92B289B2064803F0BDF8A18898
:10CBF000E288054849BA52BA92B289B2BDE81040FB
:10CC000003F0B2B8984F0108BB4F01080121014859
:10CC1000F5F716B9405D00202DE9F04780460E4635
:10CC2000FFF7F4FF294C002514F8013C9E420AD17D
:10CC300032464146204602F05FFE20B9244B1224C2
:10CC400004FB053428E00135282D04F11204EBD152
:10CC5000204B1B68272B33D81D4B0025122202FBCB
:10CC600005F91B4F19F803A0BAF1000F25D107EB06
:10CC7000090463789E4207D010225146A01C02F09E
:10CC80006BFF07F809A06670122000FB05703246A2
:10CC90004146023002F062FE23780F480133DBB2D6
:10CCA000012B08BF0B4A237002BF136801331360C6
:10CCB000F5F7F6F82046BDE8F0870135282DCED1EE
:10CCC0000548F5F7EDF80020BDE8F0874A5D002043
:10CCD000485D0020445D0020405D002010B5044602
:10CCE000FFF794FF4CB123783BB1013BDBB22370DB
:10CCF0001BB9044A1368013B13600348BDE81040A8
:10CD0000F5F7CEB8445D0020405D002070B51546B3
:10CD100006460C46FFF77AFF72782B6893420AD3D7
:10CD2000B11C204602F01AFE73782B600548F5F717
:10CD3000B7F8204670BD2A600248F5F7B1F8002028
:10CD400070BD00BF405D00202DE9F041174606464A
:10CD50008846FFF75BFF72783B68B3EBC20F05D1E3
:10CD6000B01C002501244FF0FF3316E02648F5F7EC
:10CD700097F86FF00100BDE8F081591C37D190F8A9
:10CD800000E018F80510714537D02B46C4B1BEFA43
:10CD90008EF46409A4B1013501309542EDD33CB164
:10CDA00000233B601848F5F77BF80220BDE8F081CE
:10CDB0005D1C05D11448F5F773F82046BDE8F081F5
:10CDC0001E4418F80310B2784A40072142FA01F4D1
:10CDD000E40748B202D40139F8D1084600EBC30396
:10CDE0003B600948F5F75CF80120BDE8F081002CB4
:10CDF000E6D00478B4FA84F4CBE7002CCBD0B1FAB7
:10CE000081F46409C7E700BF405D002070B5FFF7FB
:10CE1000FDFE0A4C002504F5347604F8025C04F8A3
:10CE2000015C204610220021123402F095FEB4422B
:10CE3000F3D10348BDE87040F5F732B84A5D0020F1
:10CE4000405D0020F5F72CB8B0F90010F5F748B9AF
:10CE500038B504460020F4F795FC05460020F4F7A9
:10CE600091FC401BA042F9D338BD000030B587B01B
:10CE700004460D46F3F7FFFA40B11DB10E490320F9
:10CE8000F3F7B2FE2046FFF7E3FF13E00B4B0090F1
:10CE900003900290012168460493CDF814D0F4F772
:10CEA000CFFF214601A82A46F3F74CFE0121684630
:10CEB000F4F7C6FF07B030BD2519010845CE0008BC
:10CEC00030B4034DC560026130BC1380F3F71ABE65
:10CED00049CE000870B41146039ABDF91050044EB3
:10CEE000C660026115801A4670BCF3F72BBE00BF06
:10CEF00049CE000870B58AB000210791069110490B
:10CF0000098803AC09B2054643F23906019105A828
:10CF10000094ADF80E600494FFF7DCFF2846F5F7A7
:10CF2000A8F96B88B34202D16B68A34204D005A86C
:10CF3000F3F7D6FD012001E04FF0FF300AB070BDDD
:10CF4000FC02002010B5084B0446182240F83C3B78
:10CF500002F004FD082384F85630002384F854308E
:10CF600084F8573010BD00BF1050010837B5044693
:10CF700000F03CFB94F854301BB90321204600F02C
:10CF800060FA00250821684684F83650258701F0AC
:10CF9000B7FC9DF80030019A23F0010343F002032F
:10CFA0008DF80030009B12BA1BBA204600F000F941
:10CFB000BDF8001049BA204689B200F0E5F82046D5
:10CFC000232100F028F920461A2100F015F92946FE
:10CFD000204600F03DF920460122202100F0B8F95A
:10CFE000204601224FF4807100F0B2F92A46204613
:10CFF0004FF4005100F0ACF9204601224FF480417B
:10D0000000F0A6F9204601224FF4805100F0A0F96B
:10D01000012384F82830802220460C2100F057FAA2
:10D020000421204600F065FA042100F0FD022046AC
:10D0300000F04DFA0321204600F05BFA032100F0D6
:10D04000F002204600F043FA082220460E2100F0AC
:10D050003EFA0F21204600F04CFA1621204600F03F
:10D06000F0F903B030BD10B590F8573001330446E5
:10D0700080F85730204600F094FAA0F11103DBB29B
:10D08000012BF7D9192818BF84F85600192120461A
:10D0900000F0D7F9022384F8553010BD70B51D4655
:10D0A00090F855306E1C1344144680F855301346E2
:10D0B0000A46F1B200F02FFA601970BD10B50123D5
:10D0C00000F155020021044600F025FA0222114623
:10D0D000204600F0FCF963683BB1228F120504D5AD
:10D0E00020460321BDE81040184710BDF8B50821BF
:10D0F000044600F0A6F915210746204600F0F9F98C
:10D1000060F07F02D2B215210646204600F0DFF91A
:10D110000621204600F095F90821204600F0E9F9A3
:10D1200060F07F02D2B20821204600F0D0F9012140
:10D13000204600F0DEF903060546F8D532462046C3
:10D14000152100F0C4F90821204600F07AF939468B
:10D15000204600F076F9C5F38010F8BD38B50D46CD
:10D160000221044600F0B3F9162D07D0204600F046
:10D1700018FA8542FAD184F8545038BD204600F0A0
:10D1800010FA1F28FAD0F6E710B50A0A044601F093
:10D190007F0180F82D2080F82C10202100F097F9D5
:10D1A00094F82C2020462121BDE8104000F08FB9D2
:10D1B0002DE9F843054616461F4600F12D080024C8
:10D1C0006FF00709E2003046394601F001FD09FB26
:10D1D00004F208F8010F38323046394601F0F8FC05
:10D1E00004F12401C2B2C9B22846013400F06FF93B
:10D1F000082CE7D1BDE8F883A1F10B020F2A07D86C
:10D2000090F837208A4203D080F8371000F00ABA2D
:10D2100070470020704737B50D0A4185CAB22221F8
:10D22000044600F054F92A462321204603B0BDE805
:10D23000304000F04CB9000008B5052100F059F964
:10D24000024B00F00F0033F9100008BDF04F010849
:10D25000113109B21429A8BF142121EAE171024B4E
:10D260005A5C052100F033B9DB4F010808B52C21C9
:10D2700000F03FF9C0F3071008BD38B50C462C216B
:10D28000054600F036F9072C28BF072400F00F00F0
:10D2900040EA0412D2B228462C21BDE8384000F002
:10D2A00016B908B52C2100F024F9C0F3420008BDDE
:10D2B0000529A8BF0521002938B50C46A8BF0C4692
:10D2C0004FF02C010546B8BF072400F012F920F0FA
:10D2D0000E0040EA4402D2B228462C21BDE8384074
:10D2E00000F0F5B838B505460C4699B10A782D21FD
:10D2F00000F0EDF82E21284600F0FBF8637800F0EE
:10D30000F80203F007031A4328462E21BDE83840EF
:10D3100000F0DDB838BD08B5092100F0EAF800F0EA
:10D320000F0040005B3840B208BD0029C4BF49422D
:10D3300049B25B31C1F3430242F0C002092100F05F
:10D34000C6B808B5072100F0D4F85B3840B208BD74
:10D3500010B5038F0446B2B30B43B1F5807F03874A
:10D360000AD002D8202925D010BDB1F5007F0ED0FB
:10D37000B1F5005F20D010BD00F12E01FFF7B2FF24
:10D3800004212046FFF794FF53222F2153E02E2142
:10D3900000F0AFF840F01002D2B22E21204600F08B
:10D3A00096F81721204600F0A4F840F00202D2B20D
:10D3B000172140E02E212BE00E2100F09AF840F0DA
:10D3C0000402D2B236E023EA0103B1F5807F03877D
:10D3D0000AD002D8202921D010BDB1F5007F09D094
:10D3E000B1F5005F21D010BD4FF0FF31BDE8104016
:10D3F000FFF75EBF172100F07CF8172100F0FD0257
:10D40000204600F064F8238F9B0619D52E21204674
:10D4100000F06FF800F0EF022E210CE02E2100F05A
:10D4200068F840F01002D2B2F6E70E2100F061F881
:10D4300000F0FB020E212046BDE8104000F047B886
:10D4400010BD70B504460D46204600F0AAF8A0F1C4
:10D450001103DBB2012B0646F6D91F28F4D0032DA9
:10D4600002D12A46082126E0A84227D0162801D159
:10D47000192D02E0192807D1162D0AD109221146CB
:10D480002046FFF76BFE04E00F2802D1204600F093
:10D4900094F80F2D0DD103212046FFF7D2FF294626
:10D4A000204600F026F8E06CF4F7E2F884F85450D7
:10D4B00004E02A4629462046FFF750FE304670BD5C
:10D4C00090F84030416CC06B0022F3F741BF70B55B
:10D4D00004460D461646FFF7F3FF334645F0C002FB
:10D4E000616CE06B01F05DFBE06BBDE87040F3F751
:10D4F0006FBF38B504460D46FFF7E2FF45F08002E6
:10D500000023616CE06B01F04CFB0546E06BF3F728
:10D510005FFF284638BDF7B504460F4615461E4640
:10D52000FFF7CEFF616CE06B4023012201F028FB86
:10D530003B46616CE06B012201F022FB0022E06BB4
:10D54000019600922B46616CF3F75EFFE06B03B02F
:10D55000BDE8F040F3F73CBF10B50446FFF7B0FF5D
:10D56000616CE06B20230122BDE8104001F008BB94
:10D5700007B58DE806000023416CC06B0122F3F76C
:10D5800043FF03B05DF804FB10B50446416CC06B6B
:10D590000123002201F0F4FAE06BBDE81040F3F73C
:10D5A00017BF08B590F854300F2B04D00121FFF7B6
:10D5B000A0FF00F01F03184608BD10B50446FFF792
:10D5C000F0FF0F2811D1E06CF4F75BF800214FF465
:10D5D0009970FFF74BFC01212046FFF78AFF00F00E
:10D5E0001F00082884F85400F5D110BD10B504467A
:10D5F000006DF4F746F800213E20FFF737FC206D60
:10D60000F4F736F800213E20FFF730FC01212046D8
:10D61000FFF76FFF00F01F0310F0170F84F854306E
:10D62000F4D110BD38B508210446FFF70AFF0821E0
:10D6300005462046FFF75DFF94F8373000F0E00222
:10D6400003F01F0320461A430821FFF740FF294635
:10D650002046BDE83840FFF7F4BE43680BB1002117
:10D66000184770472DE9F0470446884616461F467E
:10D67000FFF797FF8146002C00F0D3800F2840F081
:10D68000DF80B8F1180F66D02046FFF796FFB8F19B
:10D69000270F00F22B81DFE818F042002901280053
:10D6A0003300290129013B00290129012901290110
:10D6B00029012901290129012901550029018B008E
:10D6C0008F007E002901840029012901290193008E
:10D6D00097009B009F002901A300AA0029012901AE
:10D6E0002901290129014E00BA00022F03D98B49D3
:10D6F0000320F3F779FA31882046FFF745FD94E0DF
:10D70000082FF4D8D6E900232046FFF751FD8CE01E
:10D71000022FECD831882046FFF77DFD85E0012FF0
:10D72000E5D03178A1F10B030F2B00F2EC802046FD
:10D73000FFF762FD79E0012FD9D03378002B40F05C
:10D74000E2806CE0022FD2D8B6F900102046FFF735
:10D750007FFD0225D9E0012FC9D83378013B052B85
:10D7600063D8DFE803F00507620C1403082102E028
:10D770000F2100E016212046FFF763FECBE0238F48
:10D780005A0540F1C8802046FFF798FCC3E02046C8
:10D79000FFF7ECFBBFE0327820212046FFF7D8FDF1
:10D7A00043E0012FA3D831782046FFF766FD36E02D
:10D7B00032784FF4806116E032784FF4007112E055
:10D7C00032784FF400510EE032784FF480410AE095
:10D7D00032784FF4006106E032784FF4805102E075
:10D7E00032784FF480712046FFF7B2FD17E0012F29
:10D7F0003FF67DAF238FDB0503D43378052B40F252
:10D80000828096F900102046FFF752FD07E0012FB5
:10D810003FF66DAF96F900102046FFF786FD012513
:10D8200073E06FF01200BDE8F087B9F10F0F5DD023
:10D830003B46324641462046BDE8F04701F022B95A
:10D84000B8F1270FF4D801A353F828F01FD7000828
:10D8500031D80008EBD6000801D7000831D80008FD
:10D8600031D8000811D7000831D8000831D8000895
:10D8700031D8000831D8000831D8000831D8000864
:10D8800031D8000831D8000831D8000845D7000841
:10D8900031D80008B1D70008B9D7000897D70008D9
:10D8A00031D80008A3D7000831D8000857D700089E
:10D8B00031D80008C1D70008C9D70008D1D700085F
:10D8C000D9D7000831D80008E1D70008EFD7000801
:10D8D00031D8000831D8000831D8000831D8000804
:10D8E00031D8000837D700080FD80008B8F1180F52
:10D8F0009ED06FF085050F212046FFF7A2FD15F1A0
:10D90000860F05D194E76FF01505B9F10F0FF2D02E
:10D910002846BDE8F0870120BDE8F08725190108F9
:10D920002DE9F0410446FFF73CFE0F2806464CD097
:10D930000F212046FFF7DDFD022107462046FFF7B5
:10D94000D8FD7B07054603D563680121204698472B
:10D9500038073AD5162E01D0112E05D1238F590440
:10D9600033D5636802212CE0192E01D0122E2CD160
:10D9700094F857301BB916490320F3F735F9013BEA
:10D98000DBB284F8573023B994F856102046FFF7DD
:10D9900058FD6368CBB1228FD20416D505F0E000A4
:10D9A000202809D002D838B1BDE8F081602807D01E
:10D9B000A02803D0BDE8F081042102E0062100E0A8
:10D9C00007212046BDE8F0411847BDE8F08100BFBF
:10D9D0002519010813B50446416CC06BF3F78AFCA6
:10D9E0000121E06CF3F780FDE06CF3F74AFE0121C2
:10D9F000206DF3F779FD206DF3F73AFE0D4B00949F
:10DA000001220021A06CF3F7A9FD2046FFF7AEFA32
:10DA10001C212046FFF76DFD032807D11C220021A1
:10DA200004F10C0002F098F8002001E04FF0FF3004
:10DA300002B010BD5BD600082DE9F34104460F4645
:10DA400090461E46FFF788FD01220DF10301204696
:10DA5000FFF78EFD9DF8035005F07F05023D37B3BB
:10DA6000454505D92046FFF78FFD6FF0680521E099
:10DA7000236A01332362636A2B442A4639462046CF
:10DA80006362FFF775FD022201A92046FFF770FDD2
:10DA90006EB10122B1182046FFF76AFD2046FFF75C
:10DAA00073FD07212046FFF724FD307002E0204679
:10DAB000FFF76AFD284602B0BDE8F0812DE9F0418C
:10DAC00006460D469046FFF7CEFA00273C464745EE
:10DAD00012D06A68A31C13447F2B05F1080514D8E3
:10DAE000F36955F8081C2344F36130462346FFF7D9
:10DAF000D5FA01370446EAE7338F5B0502D4304696
:10DB0000FFF7DCFA2046BDE8F0816FF08A00BDE83F
:10DB1000F081000008B5FFF744FD0838C0B21128B5
:10DB20009ABF024B185C022008BD00BF28500108B4
:10DB30002DE9F8430F46164698460546002800F0A2
:10DB4000B780A1F11103152B4DD8DFE803F018279A
:10DB5000344C4C4C4C204C383C40444C484C4C4C85
:10DB60004C4C4C0BB8F1010F03D857490320F3F785
:10DB70003BF800237370FFF74CFB307004E0B8F102
:10DB8000010FF2D9662333800220BDE8F883B8F193
:10DB9000000FEAD0FFF7BEFF307009E0038F13F4E7
:10DBA000806F03D001203070BDE8F883002333700C
:10DBB0000120BDE8F883038F13F4007FF1E7038FA2
:10DBC000C3F34033F3E7038FC3F38033EFE7038FEF
:10DBD000C3F3C023EBE7038FC3F30033E7E7038FFF
:10DBE000C3F30023E3E74346324600F097FE10F10B
:10DBF000860F044660D12846FFF7D3FC0F288146E4
:10DC000011D12846FFF7D9FC162F1CD004D8012FBC
:10DC100035D0102F0ED046E0272F28D02F2F36D00A
:10DC2000202F1DD03FE0162F0DD013D8012F26D066
:10DC3000102F44D1B8F1010F97D92846FFF7FCFA0D
:10DC4000022430802CE0B8F1000F8ED02846FFF778
:10DC50000DFB23E0272F0AD02F2F18D0202F2ED1F5
:10DC6000B8F1000F81D02846FFF71BFB16E0B8F192
:10DC7000000F3FF47AAF2846FFF74DFB0EE0B8F1F6
:10DC8000000F3FF472AF2846FFF730FA06E0B8F114
:10DC9000000F3FF46AAF2846FFF753FB30700124B2
:10DCA000B9F10F0F08D10F212846FFF7CAFB03E097
:10DCB0006FF01200BDE8F8832046BDE8F8836FF0EE
:10DCC0008500BDE8F88300BF25190108094B70B530
:10DCD0001C6806460D4620460821F2F7C7FA214681
:10DCE0003046F3F701F82846F2F7C2FBBDE8704072
:10DCF000F2F7E0BF000300202DE9F04104460E4694
:10DD00001546F2F7ADFB27688046A7B13B68236054
:10DD100096E803007B6883E803000A21A7F1080066
:10DD2000F2F7A4FA17F8034C4046F2F7A1FB20469D
:10DD3000F2F7DCFA1FE0A268E3689B1A22699342BB
:10DD400007DDDDB14146201DFFF7C0FFF2F788FB7C
:10DD500080460D4BE1681B8833804B1CE3602369D0
:10DD600062690B4096E8030002EBC30383E80300FB
:10DD70004046F2F77DFB0120BDE8F081F2F778FB29
:10DD80002846BDE8F08100BFFC020020F8B504463B
:10DD90000F461546F2F764FBA168E3688B4206461E
:10DDA0001CD04B1CA3602369626965680B4002EBC1
:10DDB000C30393E8030087E80300E5B128460A217E
:10DDC00050F808396360F2F751FA15F8034C304601
:10DDD000F2F74EFB2046F2F789FA0FE03DB1084B0F
:10DDE0001B680146DF602046FFF770FF06E0F2F790
:10DDF0003FFB2846F8BD3046F2F73AFB0120F8BD5C
:10DE000000030020BFF34F8F0549064BCA6802F498
:10DE1000E0621343CB60BFF34F8F00BFFDE700BF4D
:10DE200000ED00E00400FA0538B1054B0A0901F0E5
:10DE30000F019A5C5B5C027043700220704700BF68
:10DE40003A50010803461A78591C0AB10B46FAE702
:10DE5000181A7047F8B505460F4616468C18BC428E
:10DE600006D0284614F8011DFFF7DEFF0544F6E74B
:10DE70007000F8BD07B502AB042243F8041D194633
:10DE8000FFF7E8FF03B05DF804FB38B505460C4624
:10DE90004CB122462946012002F0B6FC002802DBE4
:10DEA000241A0544F4E738BD07B5014601A8FFF779
:10DEB000BBFF022101A8FFF7E8FF03B05DF804FBF8
:10DEC00007B501466846FFF7D5FF08216846FFF70A
:10DED000DCFF03B05DF804FB10B50446FFF7B2FFAA
:10DEE00001462046BDE81040FFF7CFBFF8B5064613
:10DEF00084890F46154600206DB90023B289B168A8
:10DF0000FBF76CFC4FF6C57302199A4239680EDDB7
:10DF1000013080B20BE0AE42EFD02346AA89A96857
:10DF2000FBF75CFCEB686D681C44A4B2E4E73A3490
:10DF3000204400232022083180B2FBF74FFCC0436D
:10DF400080B2F8BD2DE9F3410C46804603212046FE
:10DF5000F7F73BFA054618B92E490320F2F744FEBD
:10DF60000221F7F732FA07460028F5D0EB68032BB9
:10DF70004CD900F1080122462846AE68FFF7B6FFEB
:10DF8000002843D13378803B082B30D8DFE803F0FA
:10DF9000052F2F2F2F0C151E2700AB89B96832468D
:10DFA000404600F081F822E0EB680093BA683346FF
:10DFB00021464046F5F7EEFE19E0EB680093BA689B
:10DFC000334621464046F5F767FF10E0EB680093C3
:10DFD000BA68334621464046F5F746FD07E0EB6850
:10DFE0000093BA68334621464046F5F709FE31787A
:10DFF000234640F201220320F6F7BAFE014628B973
:10E00000204602B0BDE8F041F7F754BC02B0BDE8CD
:10E01000F08100BF2519010838B50D4614460021CE
:10E020001A460323F7F754FB28B1836800221D70BA
:10E030005C709A70DA7038BD10B5044668B190F91A
:10E040001030032B0CD142680831FFF74FFF50B15D
:10E05000A36840BA5880002010BD6FF00D0010BDBD
:10E060006FF04C0010BD6FF0010010BD2DE9F041C4
:10E07000DDF81880154600220E461F46014608F1BD
:10E0800008031046FFF7C8FF044650B1806876BA0F
:10E090006DBA8680C58027B142463946083001F006
:10E0A0005DFC2046BDE8F081F7B506460C46002A27
:10E0B00038D0072B36D99188D088083B40BA49BA66
:10E0C000009389B202F1080382B28120FFF7CEFFEC
:10E0D000074638B3237EFF2B04F108020CBF002152
:10E0E00004F1180100F022F8054610B9014638463F
:10E0F00013E000231A4619461846F7F7B7F8836865
:10E1000009495E8004464560034640F2022202202F
:10E11000F6F72EFE014628B9204603B0BDE8F040D0
:10E12000F7F7C8BB03B0F0BD0000FFFFF8B50F461E
:10E130001646022328220021F7F7CAFA054600B343
:10E140008468102204F10800394617B101F006FC7A
:10E1500001E001F001FD04F118001022314616B172
:10E1600001F0FCFB04E001F0F7FC012384F8273008
:10E17000602200232270FF226370A370E370A271FB
:10E18000E3712846F8BD38B505460C4619B301F1D0
:10E190007000F2F7A5FC2846F5F7D0F938B1D0F8B1
:10E1A00010329C4203D100F5FC70F2F799FC04F1A7
:10E1B0001C00F2F795FC04F13800F2F791FC04F131
:10E1C0005400F2F78DFC10220021204601F0C4FC1F
:10E1D00000236383637638BD08B51022034901F03C
:10E1E0008BFBB0FA80F0400908BD00BFEE220108A9
:10E1F0002DE9F74F904600901E469DF830708946F5
:10E2000009B900205CE0082BFBD80846FFF7E4FFC3
:10E210000028F6D1824604464FF0980B2A4B0BFBA0
:10E220000AF29D18494628460192FBF7FEFA019A28
:10E2300078B1B8F1000F42D0002E40D0224B02F14D
:10E24000100041463246184401F088FB2E766F7666
:10E2500035E02846FFF7C0FF10B1002C08BF2C4660
:10E260000AF1010ABAF1080FD8D1002CC9D0BDF8C3
:10E270000030638310224946204601F06FFBB8F15D
:10E28000000F07D036B13246414604F1100001F0CC
:10E2900065FB2676677607F00707022F04BF032386
:10E2A00084F894304FF40973A4F886304FF4047363
:10E2B000C4F88840638664632465204600E02846ED
:10E2C00003B0BDE8F08F00BF186000202DE9F041D9
:10E2D00007460E4611B90020BDE8F0810846FFF759
:10E2E0007BFF0028F7D10C4D0446A846B5F91A303B
:10E2F00013B10FB1BB4209D131462846FBF795FA5D
:10E3000020B1982000FB0480BDE8F0810134082C86
:10E3100005F19805EAD1DEE71860002010B5044643
:10E32000FFF7D4FF01462046BDE81040FFF72BBFA2
:10E3300038B510B100F1980400E0074C074DAC422D
:10E3400005D22046FFF748FF18B19834F7E70020C0
:10E3500038BD204638BD00BF18600020D8640020BA
:10E3600008B5FFF7E5FF10B1437E1B07F9D508BDDF
:10E37000F8B501460020FFF7A9FF044610B3437E1D
:10E3800013F0050F1ED0B0F91A00F5F7D7F80E4BB1
:10E39000D0F8D461B3F9007004F138052846F2F7DB
:10E3A0009FFB40F21723A4F84E3004F14C023B4689
:10E3B00031462846FEF784FD637E23F0070343F0D1
:10E3C000070363762046F8BDB823002010B5144635
:10E3D00000B119B90B490320F2F706FC2AB1537EAC
:10E3E00003F00703013B012B01D8002010BD137E71
:10E3F0000B70127E04F1100101F0B0FAB4F91A00AA
:10E4000010BD00BF25190108F0B503EB43048C4291
:10E410004FF0000122D8017005465E1E0F464FF0F6
:10E420003A0E994219D014782409092C94BF30343B
:10E43000573494462C709CF8004004F00F04092CCB
:10E4400094BF30345734B1426C700CBF3C467446B4
:10E45000AC70013201310335E3E7F0BD0846F0BD91
:10E460002DE9F04112B90020BDE8F0811378002BAE
:10E47000F9D01446264601347378002BFAD10746AA
:10E480004FF0010C964217D33478A4F130055FFAAF
:10E4900085F8B8F1090F06F1FF3E23D9A4F1410533
:10E4A000052D02D8A4F137051CE0A4F16105052D66
:10E4B00011D8A4F1570515E0BCF1000FD3D1013FED
:10E4C000B84205D23A780178397000F8012BF6E7A6
:10E4D0001846BDE8F081BCF1000FC4D14FF0010C2B
:10E4E0007646CFE7724518D8A6F1020E16F8016CF1
:10E4F000A6F130045FFA84FCBCF1090F0ED9A6F135
:10E500004104052C02D8A6F1370407E0A6F1610406
:10E51000052C02D8A6F1570400E0002401338B42F9
:10E52000A1D845EA04143C704FF0000C0137D7E73E
:10E5300010B5044686B0B0F90210214801F014FC71
:10E540006179204801F010FCA1791F4801F00CFC12
:10E550001E4801F009FC237963B11A0602D51C4854
:10E5600001F002FC23795B0602D51A4801F0FCFB9E
:10E57000194800E0194801F081FC237853B104F1F7
:10E58000080218216846FFF73FFF0146144801F0D2
:10E59000EBFB02E0134801F071FC63785BB1227879
:10E5A0000832224418216846FFF72EFF01460E4824
:10E5B00001F0DAFB02E00D4801F060FC06B010BD8E
:10E5C0004A50010857500108625001086B50010879
:10E5D000735001087E5001089D47010889500108C9
:10E5E0008D5001089D500108AF500108BF5001082F
:10E5F00013B5074A044692E8030000228DE80300A1
:10E60000694604F11000FFF777FB02B010BD00BFB0
:10E61000D450010803460846002110B483E80600E0
:10E62000072401221C621A7203F1280403F110026C
:10E63000196159619961D9615C62DA60194610BC4F
:10E64000F6F74ABE70B51C46531E03330E4688B01B
:10E65000114600F1100506D8294B079003A8069330
:10E66000F2F750FA00E02AB1012201A92846FFF78B
:10E670008DFB05E001A92846FFF788FB002838D06C
:10E6800003A8F2F72DFABDF8063040F201229342BA
:10E690000CD048F2744293422ED1029A194B9A42FE
:10E6A00014BF6FF003006FF0730027E0029D02219A
:10E6B0002846F6F78AFE10B1C368272B03D8124903
:10E6C0000320F2F791FA816810220831201D01F031
:10E6D00045F9042323604FF0FF312846F6F775FE15
:10E6E00008B9A08202E083685B88A38235600020BD
:10E6F00004E06FF00A0001E06FF0030008B070BDA5
:10E70000F1E50008630B8AF3251901082DE9F047AC
:10E710008946064690469A460146002419B1CB68C0
:10E7200049681C44FAE7D9F80030D8F80020934231
:10E7300016D1042B14D108F1040209F1040130466A
:10E74000FFF7F4FC0746C8B396F910500DB902253F
:10E750003574BB6883F806A0B9F8146056B906E0B2
:10E760003046F7F7A7F86FF06900BDE8F087B8F812
:10E77000146086B1002319461A461846F6F776FD4E
:10E7800036B2014618B93846F7F794F816E08B68A8
:10E790005E804F600F460B493B4640F202222846FE
:10E7A000F6F7E6FA014630B93846F7F783F86FF026
:10E7B0004C00BDE8F0872046BDE8F0876FF00B0005
:10E7C000BDE8F0870000FFFF2DE9F0470F46054642
:10E7D00010B90020BDE8F0870029FAD010220021EE
:10E7E00001F0BAF93B783A2B04D00024A146264622
:10E7F000A04619E07A783A2A07F10103E9D11F46C9
:10E80000F3E751462B4801F0BFFB98B951462A481F
:10E8100001F0BAFB80B1284BC01A40EA0616B6F5E3
:10E82000803FD6D24FF0010917F801ABBAF1000FC3
:10E83000E7D119E01F4BEFE7BAF13A0FC9D1B9F1AF
:10E84000000F05D1B8F1000FC3D105EB0408EBE7C9
:10E85000A21C102ABDD8631CDBB2310A295581469F
:10E86000EE54D4B20646DFE7B9F1000F08D0A21C7F
:10E87000102AAED8631CDBB2310A2955EE54D4B24B
:10E88000B8F1000F10D02C44C8EB040805F11002B9
:10E8900001230021434504F1FF3407DC207802F80E
:10E8A000010D01332170F5E7102C92D12846BDE807
:10E8B000F08700BF0E230108DC5001087FB50C462D
:10E8C000054600B119B90D490320F2F78DF90A4642
:10E8D00001AE232101F040F9304600F04BF900234E
:10E8E000B3FBF4F204FB1232F15CA85C013341404B
:10E8F0000C2BA954F4D104B070BD00BF2519010838
:10E9000010B50446FFF7DAFF034B1A78511C197053
:10E9100023785340237010BD8A020020062938B5A1
:10E9200004460D46104636D006D8032922D029D8F1
:10E93000B1B3022911D09DE017294AD004D8082983
:10E9400051D0152932D095E0252948D0292900F049
:10E950008980192940F08E8035E0012B03D8484981
:10E960000320F2F741F90A4604F12C0100F0F6FF0A
:10E97000284638BD072BF2D9082204F12E0100F0F9
:10E98000EDFF7AE0022BEAD1228F520701D508224F
:10E9900004E003806CE0022BE1D1628D028067E02D
:10E9A000022BDCD194F8373013800AE0012BD6D14A
:10E9B000238F13F0200F02D00123037058E00023AF
:10E9C0000370012038BD012BC9D1238F13F0020F32
:10E9D000F1E7012BC3D194F92820027048E0022B03
:10E9E000BDD10322DAE7072BB9D9238F5B074CBFD0
:10E9F0002B4602234FF000024CBF04F12E0104F11C
:10EA00002C01042B4270027018D0082B03D0022B6B
:10EA100033D1134619E00A7882F0020202704A7874
:10EA200042708A788270CA78C2700A7902714A7913
:10EA300042718A798271CA79C27119E00B7883F0C8
:10EA4000020303704B7843700223FF240022C4703A
:10EA5000FE24827004714271CA5C827119444B7841
:10EA6000C3710AE0042B7FF47AAF04F10C0111604A
:10EA7000184638BD6FF0850038BD082038BD00BF8E
:10EA80002519010870B515461C4619296AD8DFE812
:10EA900001F00D6919293939496969696969696933
:10EAA000696969696969694E69616958022C03D0AD
:10EAB0002F490320F2F798F81388FF2BF8D880F835
:10EAC00037304DE0022CF3D800F12C060222002151
:10EAD000304601F041F822462946304600F03EFF1C
:10EAE000022070BD082CE3D800F12E060822002178
:10EAF000304601F031F822462946304600F02EFF1C
:10EB0000082070BD022CD3D11388022B06D0082B0D
:10EB10002BD1038F43F00403038721E0038F23F0FD
:10EB200004030CE0022CC3D11388438518E012784B
:10EB3000038F12B143F0200301E023F02003038789
:10EB4000CEE71278038F12B143F00203F7E723F008
:10EB50000203F4E7012CABD192F9003080F82830A1
:10EB6000204670BD6FF0850070BD6FF0690070BD0C
:10EB7000251901080C22014900F0F0BE107AFF1F90
:10EB800010B586B006AC04F8093D012301930DF1E0
:10EB9000170300932346F2F737FC9DF8170006B0E1
:10EBA00010BDF0B585B01F4604AB002403F8012D5D
:10EBB000012205460E4601920094F2F725FC3B46E1
:10EBC000224631462846FFF7DBFF05B0F0BD0000C6
:10EBD000D0400B1CD1409C46203AD34018435242AF
:10EBE000634693401843704780F0004002E000BF46
:10EBF00081F0004142001FBF5FEA410392EA030F28
:10EC00007FEA226C7FEA236C6AD04FEA1262D2EB71
:10EC10001363C1BFD218414048404140B8BF5B4276
:10EC2000192B88BF704710F0004F40F4000020F00F
:10EC30007F4018BF404211F0004F41F4000121F025
:10EC40007F4118BF494292EA030F3FD0A2F101026F
:10EC500041FA03FC10EB0C00C3F1200301FA03F1AD
:10EC600000F0004302D5494260EB4000B0F5000FD0
:10EC700013D3B0F1807F06D340084FEA310102F18F
:10EC80000102FE2A51D2B1F1004F40EBC25008BF41
:10EC900020F0010040EA03007047490040EB00000B
:10ECA00010F4000FA2F10102EDD1B0FA80FCACF13A
:10ECB000080CB2EB0C0200FA0CF0AABF00EBC25039
:10ECC00052421843BCBFD0401843704792F0000F27
:10ECD00081F4000106BF80F400000132013BB5E77A
:10ECE0004FEA41037FEA226C18BF7FEA236C21D0F0
:10ECF00092EA030F04D092F0000F08BF0846704755
:10ED000090EA010F1CBF0020704712F07F4F04D122
:10ED1000400028BF40F00040704712F100723CBF35
:10ED200000F50000704700F0004343F0FE4040F45F
:10ED3000000070477FEA226216BF08467FEA23631D
:10ED40000146420206BF5FEA412390EA010F40F408
:10ED5000800070474FF0000304E000BF10F0004354
:10ED600048BF40425FEA000C08BF704743F096433B
:10ED700001464FF000001CE050EA010208BF704756
:10ED80004FF000030AE000BF50EA010208BF7047DD
:10ED900011F0004302D5404261EB41015FEA010CF2
:10EDA00002BF84460146002043F0B64308BFA3F1EA
:10EDB0008053A3F50003BCFA8CF2083AA3EBC253CC
:10EDC00010DB01FA02FC634400FA02FCC2F12002EB
:10EDD000BCF1004F20FA02F243EB020008BF20F022
:10EDE0000100704702F1200201FA02FCC2F1200288
:10EDF00050EA4C0021FA02F243EB020008BF20EA7D
:10EE0000DC7070474FF0FF0C1CEAD0521EBF1CEAAA
:10EE1000D15392EA0C0F93EA0C0F6FD01A4480EA98
:10EE2000010C400218BF5FEA41211ED04FF0006381
:10EE300043EA501043EA5111A0FB01310CF00040AD
:10EE4000B1F5000F3EBF490041EAD3715B0040EAD3
:10EE5000010062F17F02FD2A1DD8B3F1004F40EBA3
:10EE6000C25008BF20F00100704790F0000F0CF076
:10EE7000004C08BF49024CEA502040EA51207F3A3A
:10EE8000C2BFD2F1FF0340EAC250704740F4000015
:10EE90004FF00003013A5DDC12F1190FDCBF00F006
:10EEA00000407047C2F10002410021FA02F1C2F1B4
:10EEB000200200FA02FC5FEA310040F1000053EA50
:10EEC0004C0308BF20EADC70704792F0000F00F09E
:10EED000004C02BF400010F4000F013AF9D040EAA4
:10EEE0000C0093F0000F01F0004C02BF490011F438
:10EEF000000F013BF9D041EA0C018FE70CEAD15336
:10EF000092EA0C0F18BF93EA0C0F0AD030F0004CB5
:10EF100018BF31F0004CD8D180EA010000F0004069
:10EF2000704790F0000F17BF90F0004F084691F027
:10EF3000000F91F0004F14D092EA0C0F01D1420261
:10EF40000FD193EA0C0F03D14B0218BF084608D12A
:10EF500080EA010000F0004040F0FE4040F4000074
:10EF6000704740F0FE4040F4400070474FF0FF0C07
:10EF70001CEAD0521EBF1CEAD15392EA0C0F93EA4E
:10EF80000C0F69D0A2EB030280EA010C49024FEAA0
:10EF9000402037D04FF0805343EA111143EA101359
:10EFA0000CF000408B4238BF5B0042F17D024FF411
:10EFB000000C8B4224BF5B1A40EA0C00B3EB510FEC
:10EFC00024BFA3EB510340EA5C00B3EB910F24BFD5
:10EFD000A3EB910340EA9C00B3EBD10F24BFA3EB5A
:10EFE000D10340EADC001B0118BF5FEA1C1CE0D122
:10EFF000FD2A3FF650AF8B4240EBC25008BF20F0D5
:10F00000010070470CF0004C4CEA50207F32C2BF28
:10F01000D2F1FF0340EAC250704740F400004FF0C5
:10F020000003013A37E792F0000F00F0004C02BFF6
:10F03000400010F4000F013AF9D040EA0C0093F0C0
:10F04000000F01F0004C02BF490011F4000F013B1A
:10F05000F9D041EA0C0195E70CEAD15392EA0C0F82
:10F0600008D142027FF47DAF93EA0C0F7FF470AFBA
:10F07000084676E793EA0C0F04D14B023FF44CAFFD
:10F0800008466EE730F0004C18BF31F0004CCAD192
:10F0900030F000427FF45CAF31F000437FF43CAFCE
:10F0A0005FE700BF4FEA4002B2F1FE4F0FD34FF0CF
:10F0B0009E03B3EB12620DD94FEA002343F00043E5
:10F0C00010F0004F23FA02F018BF404270474FF093
:10F0D0000000704712F1610F01D1420205D110F01A
:10F0E000004008BF6FF0004070474FF000007047CD
:10F0F00053B94AB9002908BF00281CBF4FF0FF319F
:10F100004FF0FF3000F07EB9ADF1080C6DE904CE90
:10F1100000F006F8DDF804E0DDE9022304B07047F2
:10F120002DE9F0478C460E460446089D002B50D131
:10F130008A4217466CD9B2FA82FEBEF1000F0BD09C
:10F14000CEF1200420FA04F401FA0EF644EA060C8B
:10F1500002FA0EF700FA0EF44FEA1749220CBCFB34
:10F16000F9F01FFA87F809FB10C642EA064600FBD1
:10F1700008F3B34209D9F61900F1FF3280F0228179
:10F18000B34240F21F8102383E44F61AA2B2B6FBE7
:10F19000F9F309FB136642EA064403FB08F8A045AD
:10F1A00009D9E41903F1FF3280F00A81A04540F249
:10F1B0000781023B3C44C8EB040443EA00400021C1
:10F1C000002D62D024FA0EF400232C606B60BDE8A1
:10F1D000F0878B4207D9002D55D0002185E84100EA
:10F1E0000846BDE8F087B3FA83F1002940F090802B
:10F1F000B34202D3824200F2F880841A66EB03061F
:10F200000120B446002D40D085E81010BDE8F087FD
:10F2100012B90127B7FBF2F7B7FA87FEBEF1000F6C
:10F2200035D1F31B4FEA17481FFA87FC0121B3FBC6
:10F23000F8F0220C08FB103642EA06460CFB00F3FD
:10F24000B34207D9F61900F1FF3202D2B34200F2FD
:10F25000CE801046F61AA2B2B6FBF8F308FB13668E
:10F2600042EA06440CFB03FCA44507D9E41903F168
:10F27000FF3202D2A44500F2B5801346CCEB040461
:10F2800043EA00409CE729462846BDE8F087CEF1D6
:10F29000200106FA0EF307FA0EF720FA01F94FEAF9
:10F2A0001748CE4049EA0309B6FBF8FA4FEA194479
:10F2B00008FB1A661FFA87FC44EA06430AFB0CF2B5
:10F2C0009A4200FA0EF40AD9DB190AF1FF3180F0F4
:10F2D00087809A4240F28480AAF1020A3B449B1A3A
:10F2E0001FFA89F9B3FBF8F108FB113349EA03432C
:10F2F00001FB0CF69E4207D9DB1901F1FF326BD2FC
:10F300009E4269D902393B449B1B41EA0A418EE780
:10F31000C1F1200E22FA0EF48B40234320FA0EF79F
:10F3200006FA01F44FEA134C26FA0EF63C43B6FBFC
:10F33000FCF9270C0CFB19661FFA83F847EA06460E
:10F3400009FB08F7B74202FA01F200FA01FA08D9FC
:10F35000F61809F1FF3041D2B7423FD9A9F10209AD
:10F360001E44F61BA0B2B6FBFCF40CFB146640EA8C
:10F37000064704FB08F8B84507D9FF1804F1FF3029
:10F3800028D2B84526D9023C1F4444EA0940C8EBBC
:10F390000707A0FB02894F4544464E4614D329D0A7
:10F3A00065B3BAEB040367EB060707FA0EFECB4022
:10F3B000CF404EEA030385E888000021BDE8F087CE
:10F3C0001346F8E61046E0E6B8EB020469EB0306E4
:10F3D0000138E5E70446D8E7114695E78146C0E7DE
:10F3E0008A467CE7023B3C4448E708460AE7023885
:10F3F0003E442FE7C245E7D33E46D1E72946BDE864
:10F40000F08700BF704700BF0A22002101F04AB90F
:10F410000A23002201F0B2B8014B1868704700BF00
:10F420008C0200208B891A072DE9F0410D46804699
:10F4300035D44A68002A6BDDEC6A002C47D003F40F
:10F440008052002192B2D8F80060C8F80010002A5B
:10F4500062D06A6D5F0705D569686B6B521A0BB194
:10F460002B6CD21A0023296A4046A047441C39D08D
:10F47000AB892A692A60DB044FF000026A6045D438
:10F48000696BC8F8006011B305F14403994202D0DA
:10F49000404600F0AFFB00206863BDE8F0810E69D4
:10F4A000AEB10C680E6098070CBF4B690023A41B1B
:10F4B0008B600AE023463246AF6A296A4046B84765
:10F4C0000028A4EB0004064404DD002CF2DC00203C
:10F4D000BDE8F081AB8943F04003AB814FF0FF30D2
:10F4E000BDE8F081D8F800201D2AF3D8184BD3408E
:10F4F00003F0010383F00101002BEBD0AB892C69F1
:10F500006960D9042C60BBD5002AB9D16865B7E71A
:10F510000A6C002A90DCDAE70123296A4046A047FA
:10F52000431C024602D0AB89EC6A93E7D8F800305E
:10F53000002BF8D01D2B01D0162B02D1C8F800608B
:10F54000C5E7AB8943F04003AB81BDE8F08100BF64
:10F55000010040200B6933B310B5044682B008B1F6
:10F560008369ABB1114B994219D0114B994218D014
:10F57000104B994208BFE168B1F90C3013B9002073
:10F5800002B010BD204602B0BDE81040FFF74ABFF0
:10F59000019100F019F90199044B9942E5D1616894
:10F5A000EAE7A168E8E70020704700BF3051010892
:10F5B00010510108F050010820B1054B01461868B0
:10F5C000FFF7C8BF034B0449186800F043B900BFF8
:10F5D0008C0200205051010855F5000800207047AA
:10F5E000014900F037B900BF55F500080020704709
:10F5F00070B568234D1E03FB05F50E4605F1740139
:10F6000000F03EFB044640B100210C30666005F17D
:10F6100068022160A06000F09FFA204670BD00BF24
:10F620001F4B70B51D68AB69064613B9284600F03C
:10F6300039F848356B68AC68013B05D521E0013BE2
:10F640005A1C04F168041CD0B4F90C20002AF6D12D
:10F65000002501234FF6FF72E281A38165662560D4
:10F66000A560656025616561A5612946082204F1F0
:10F670005C0000F071FA6563A563A564E56420464B
:10F6800070BD2B680BB11D46D4E704213046FFF74F
:10F69000AFFF286008B10546CCE70C23336070BD8E
:10F6A000505101083D4B3E491A682DE9F04F9042F8
:10F6B0004FF000038364C364036508BF012383B074
:10F6C00008BF836181620746FFF7AAFF786038466A
:10F6D000FFF7A6FFB8603846FFF7A2FF7D68F86025
:10F6E00000240423AB812C606C60AC606C66EC8100
:10F6F0002C616C61AC61214605F15C00082200F0D0
:10F700002BFABE68DFF89CB0DFF89CA0DFF89C9075
:10F71000DFF89C80C5F824B001230922C5F828A091
:10F72000C5F82C90C5F830802D622146F381B28156
:10F7300034607460B460746634617461B46106F1FD
:10F740005C000822019300F007FAFD68366212207F
:10F750000222C6F824B0C6F828A0C6F82C90C6F835
:10F7600030802146A881EA812C606C60AC606C66B8
:10F770002C616C61AC6105F15C00082200F0ECF9D1
:10F78000019B2D62C5F824B0C5F828A0C5F82C90BF
:10F79000C5F83080BB6103B0BDE8F08F505101085F
:10F7A000E1F50008FDFE000825FF000861FF0008E4
:10F7B00081FF0008024B0349186800F04BB800BFF6
:10F7C0005051010855F50008836903B96AE770478D
:10F7D000704700BF704700BF704700BF704700BF51
:10F7E000024B0349186800F00FB800BF8C020020DC
:10F7F000EDF50008024B0349186800F005B800BF9A
:10F800008C020020DDF500082DE9F04110F14807D9
:10F810001BD0884600267D68BC68013D0FD4A389B3
:10F82000012B05F1FF3506D9B4F90E30013320461E
:10F8300001D0C04706436B1C04F16804EFD13F6858
:10F84000002FE8D13046BDE8F0813E463046BDE8A5
:10F85000F08100BF2DE9F84310F148071FD088461A
:10F8600006464FF000097D68BC68013D11D4A389AC
:10F87000012B05F1FF3508D9B4F90E3001332146CB
:10F88000304602D0C04749EA00096B1C04F1680405
:10F89000EDD13F68002FE6D14846BDE8F883B94670
:10F8A0004846BDE8F88300BF70B50F4E0F4D761B7C
:10F8B000B61018BF002405D0013455F8043B984712
:10F8C000A642F9D10A4E0B4D761BF0F75FFCB6103D
:10F8D00018BF002406D0013455F8043B9847A642CF
:10F8E000F9D170BD70BD00BF98520108985201084F
:10F8F0009852010898520108032A70B426D940EAA8
:10F9000001039B0711D004780D78AC4222D1024448
:10F91000431C05E013F8014B11F8015FAC4219D10B
:10F920009342F7D1002070BC70470C4603461E6816
:10F930002568AE421846214603F1040304F104048D
:10F94000E1D1043A032A18462146F0D8002ADAD138
:10F950001046E8E7601B70BC704700BF844641EA70
:10F96000000313F003036DD1403A41D351F8043B37
:10F9700040F8043B51F8043B40F8043B51F8043B89
:10F9800040F8043B51F8043B40F8043B51F8043B79
:10F9900040F8043B51F8043B40F8043B51F8043B69
:10F9A00040F8043B51F8043B40F8043B51F8043B59
:10F9B00040F8043B51F8043B40F8043B51F8043B49
:10F9C00040F8043B51F8043B40F8043B51F8043B39
:10F9D00040F8043B51F8043B40F8043B51F8043B29
:10F9E00040F8043B51F8043B40F8043B403ABDD298
:10F9F000303211D351F8043B40F8043B51F8043B3A
:10FA000040F8043B51F8043B40F8043B51F8043BF8
:10FA100040F8043B103AEDD20C3205D351F8043BC8
:10FA200040F8043B043AF9D2043208D0D2071CBF94
:10FA300011F8013B00F8013B01D30B8803806046BD
:10FA4000704700BF082A13D38B078DD010F0030333
:10FA50008AD0C3F10403D21ADB071CBF11F8013BA3
:10FA600000F8013B80D331F8023B20F8023B7BE7F2
:10FA7000043AD9D3013A11F8013B00F8013BF9D21D
:10FA80000B7803704B7843708B78837060467047B7
:10FA90008842F0B50DD98B1898420AD28118002AF5
:10FAA00051D09A1A13F8014D01F8014D9342F9D142
:10FAB000F0BD0F2A48D941EA00039B0746D100F167
:10FAC000100401F11003154653F8106C44F8106C43
:10FAD00053F80C6C44F80C6C53F8086C44F8086C40
:10FAE000103D53F8046C44F8046C0F2D03F110031F
:10FAF00004F11004E8D8A2F1100323F00F0302F080
:10FB00000F0E1033BEF1030F1944034421D91E1FF9
:10FB10000D467446043C55F8047B46F8047F032CDC
:10FB2000F8D8AEF1040424F003040434234421443F
:10FB300002F0030262B1013B0A4411F8014B03F8E1
:10FB4000014F8A42F9D1F0BD0346F3E70346F2E7DD
:10FB5000F0BD7246EEE700BF70B4840746D0541E75
:10FB6000002A41D0CDB2034602E0621EE4B314463F
:10FB700003F8015B9A07F8D1032C2ED9CDB245EAE0
:10FB800005250F2C45EA054519D903F11002264633
:10FB9000103E0F2E42F8105C42F80C5C42F8085CF4
:10FBA00042F8045C02F11002F2D8A4F1100222F033
:10FBB0000F0204F00F041032032C13440DD91E461B
:10FBC0002246043A032A46F8045BFAD8221F22F0A0
:10FBD00003020432134404F003042CB1C9B21C44E0
:10FBE00003F8011BA342FBD170BC704714460346C7
:10FBF000C2E700BF30B481B151F8043C0439002B96
:10FC0000B8BFC9181D4B1A682AB18A420AD90868B8
:10FC10000C18A24225D04A60196030BC70478B4254
:10FC200003D81A465368002BF9D1146815198D4270
:10FC30000CD007D808680C189C4218D04B6030BC18
:10FC4000516070470C23036030BC704709680C4456
:10FC5000111999421460E0D10ACB0C44536014602E
:10FC6000DBE7146852684A6020440860D4E71C68E7
:10FC70005B684B60204408605160CEE7D864002088
:10FC800070B5CD1C25F0030508350C2D38BF0C25AB
:10FC9000002D06463BDBA94239D827490A6852B1F4
:10FCA00013685B1B04D436E023685B1B1AD522461D
:10FCB0005468002CF8D149681F4C002936D02946D9
:10FCC0003046F0F767FA431C21D0C41C24F003042B
:10FCD000A04205D0211A3046F0F75CFA013016D068
:10FCE000256004E00B2B0DD923601C44256004F132
:10FCF0000B0020F00700231DC31A02D05A42E25025
:10FD000070BD70BD94420ED063685360EFE70C2362
:10FD10003360002070BD0B2B03D8536814460B6072
:10FD2000E5E71446E0E713461446F8E73046F0F7F7
:10FD300031FA6060C3E700BFD86400200EB410B58C
:10FD4000044683B018B183690BB9FFF73DFD06A8DF
:10FD500003460190059AA168204600F0EBFE03B02F
:10FD6000BDE8104003B070470FB410B50A4B1C68D3
:10FD700082B024B1A36913B92046FFF725FD05A879
:10FD800003460190049AA168204600F0D3FE02B019
:10FD9000BDE8104004B070478C0200202DE9F0410E
:10FDA0000E46804600283ED08369002B39D08468F7
:10FDB0002F4B9C4243D02F4B9C4256D02E4B9C4203
:10FDC00008BFD8F80C40A3891B073DD52369002B39
:10FDD0003AD0013EA36816F8015F013BA360B5B1BC
:10FDE000002B04DB23685A1C22601D70F2E7A76910
:10FDF000BB4222462946404601DB0A2DF2D100F0E3
:10FE00000FFD0130E6D14FF0FF30BDE8F081002B4F
:10FE100021DB23680A22591C21601A701046BDE8B4
:10FE2000F081FFF7D1FCD8F81830D8F80840002B43
:10FE3000BED14046FFF7C8FC0D4B9C42BBD1D8F861
:10FE40000440A3891B07C1D42146404600F04AFD67
:10FE50000028BED0D7E7224640460A2100F0E0FC49
:10FE60000130D0D00A20BDE8F081D8F80840AAE7D8
:10FE70003051010810510108F0500108024B0146B1
:10FE80001868FFF78BBF00BF8C02002038B50C4606
:10FE9000054608B18369B3B1114B9C4218D0114B90
:10FEA0009C4217D0104B9C4208BFEC682846214664
:10FEB00001F076F980B994E80C00013B511C84E80C
:10FEC0000A00107838BDFFF77FFC054B9C42E6D155
:10FED0006C68EBE7AC68E9E74FF0FF3038BD00BF76
:10FEE0003051010810510108F0500108024B014641
:10FEF0001868FFF7CBBF00BF8C02002010B50C467E
:10FF0000B1F90E10F0F764F9002803DB636D0344C8
:10FF1000636510BDA38923F48053A38110BD00BF86
:10FF2000002070472DE9F0411646B1F90C201F461C
:10FF3000D3050C46054607D500220223B1F90E1061
:10FF4000F0F753F9B4F90C20B4F90E1022F48052F2
:10FF5000A2813B4632462846BDE8F041F0F73CB965
:10FF600010B50C46B1F90E10F0F73FF9A389421C09
:10FF70000EBF23F4805343F480536065A38110BD0A
:10FF8000B1F90E10F0F72CB970B411F0FF0434D0B1
:10FF900085070FD00378002B5AD09C422BD0431CEE
:10FFA00005E013F8012B002A4FD0944223D09A0782
:10FFB0001846F6D10E0206F47F462643036846EA49
:10FFC000064601E050F8043F86EA0305A5F1013238
:10FFD000A3F1013122EA050221EA0303134313F0DE
:10FFE000803FEFD0037823B932E010F8013F002BB7
:10FFF0002ED09C42F9D170BC704784070BD0037897
:020000040801F1
:10000000002BF8D0431C03E002780133002AF2D021
:1000100099071846F8D10268A2F1013323EA0203D6
:1000200013F0803F08D150F8042FA2F1013323EAE6
:10003000020313F0803FF6D00378002BDBD010F8DA
:10004000013F002BFBD170BC7047104670BC70475D
:10005000184670BC704700BF0000000000000000A0
:10006000A2EB0300704700BF02780B78012A28BF7B
:100070009A42F5D16DE9044540EA0104CDE90267F1
:100080006FF0000C4FEA447212B380EA010414F0DE
:10009000070F6AD100F0070420F0070004F0030501
:1000A00021F007014FEAC505F0E8042314F0040F1E
:1000B000F1E804670CFA05F462EA040266EA040651
:1000C0000AD063EA0403624667EA0407664603E06F
:1000D000F0E80423F1E8046782FA4CF582EA0604AA
:1000E000A4FA8CF46CBB83FA4CF583EA0705A5FAF5
:1000F0008CF595B950E9022351E9026782FA4CF573
:1001000082EA0604A4FA8CF483FA4CF583EA070524
:10011000A5FA8CF52543DBD09CB92DBAB5FA85F448
:1001200024F0070427FA04F1DDE9026723FA04F357
:1001300003F0FF0001F0FF01FDE80445A0EB010022
:10014000704724BAB4FA84F424F0070426FA04F1C0
:10015000DDE9026722FA04F202F0FF0001F0FF017C
:10016000FDE80445A0EB0100704714F0030F3CD1FB
:1001700010F0030428D150F8082B51F8083B82FAFC
:100180004CF582EA0305A5FA8CF55DB950F8042C0C
:1001900051F8043C82FA4CF582EA0305A5FA8CF585
:1001A000002DE8D02DBAB5FA85F424F0070423FA1F
:1001B00004F122FA04F202F0FF0001F0FF01FDE871
:1001C0000445A0EB010070474FEAC40420F003008F
:1001D00050F8082B21F0030151F8083B0CFA04F405
:1001E00062EA040263EA0403C9E710F003041AD0C8
:1001F000A1EB040120F00300E40750F8042B06D023
:100200000FD28B785FFAA2F4E41A06D12BB1CB7827
:100210005FFAB2F4E41A00D11BB920465DF8104B26
:10022000704701F1040150F8042BCC0721F00301C1
:1002300051F8043B48D824D222F07F4482FA4CF58E
:1002400094EA1325A5FA8CF50AD165B951F8043B57
:1002500084EA0204B4EB036F0ED150F8042BEBE7F1
:100260004FEA132355E035F07F454DD10878FDE87E
:100270000445C0F1000070474FEA126203F0FF032B
:1002800047E002EA1C4482FA4CF594EA1345A5FAC9
:100290008CF50AD165B951F8043B84EA0204B4EB49
:1002A000034F0CD150F8042BEBE74FEA134330E037
:1002B00015EA1C4528D10B884FEA124229E04FEA83
:1002C000124203EA1C4324E002F0FF0482FA4CF5D8
:1002D00094EA1365A5FA8CF50AD165B951F8043B87
:1002E00084EA0204B4EB032F09D150F8042BEBE7A6
:1002F0004FEA13630DE015F0FF0F05D10B684FEACD
:10030000122223F07F4304E04FF00000FDE8044593
:10031000704712BA1BBA82FA4CF482EA0304A4FAB8
:100320008CF5B5FA85F402FA04F203FA04F34FEA05
:100330001260FDE80445A0EB1360704780EA0102FB
:10034000844612F0030F4FD111F0030F32D14DF854
:10035000044D11F0040F51F8043B0BD0A3F101320E
:100360009A4312F0803F04BF4CF8043B51F8043B21
:1003700016D100BF51F8044BA3F101329A4312F099
:10038000803FA4F101320BD14CF8043BA24312F0A0
:10039000803F04BF51F8043B4CF8044BEAD023469D
:1003A0000CF8013B13F0FF0F4FEA3323F8D15DF84F
:1003B000044B704711F0010F06D011F8012B0CF817
:1003C000012B002A08BF704711F0020FBFD031F88F
:1003D000022B12F0FF0F16BF2CF8022B8CF8002016
:1003E00012F47F4FB3D1704711F8012B0CF8012B99
:1003F000002AF9D1704700BF000000000000000093
:1004000090F800F06DE9024520F007016FF0000C54
:1004100010F0070491F820F040F049804FF00004FC
:100420006FF00700D1E9002391F840F000F10800D7
:1004300082FA4CF2A4FA8CF283FA4CF3A2FA8CF30F
:100440004BBBD1E9022382FA4CF200F10800A4FA76
:100450008CF283FA4CF3A2FA8CF3E3B9D1E90423CA
:1004600082FA4CF200F10800A4FA8CF283FA4CF301
:10047000A2FA8CF37BB9D1E9062301F1200182FABB
:100480004CF200F10800A4FA8CF283FA4CF3A2FAC1
:100490008CF3002BC6D0002A04BF04301A4612BACF
:1004A000B2FA82F2FDE8024500EBD2007047D1E9D2
:1004B000002304F00305C4F100004FEAC50514F061
:1004C000040F91F840F00CFA05F562EA05021CBF32
:1004D00063EA050362464FF00004A9E7002A41D011
:1004E00040EA010313F00303F0B425D1032A23D912
:1004F00004680D68AC421FD1043A35D0A4F101352F
:1005000025EA040414F0803F31D1071D0D1D0DE0D4
:1005100057F8043B0E68A3F10134B34224EA030404
:100520000AD1043A20D014F0803F23D1032A29466F
:10053000384605F10405EBD803780C789C4202F1AB
:10054000FF320CD182B114B916E06AB17BB110F858
:10055000013F11F8014FA34202F1FF32F5D0181B01
:10056000F0BC7047104670471046F0BC7047184604
:10057000F0BC70470020F3E72046F1E72DE9F04F8B
:10058000474C83460E46D4F800E000E02646344649
:1005900014F8015B0EEB0500407800F0080000F055
:1005A000FF080028F2D12D2D5CD02B2D04BF7578CB
:1005B000B41C002B3ED0102B60D09A46B8F1000F2F
:1005C0000CBF6FF000404FF000400027B0FBFAF97D
:1005D000BC460AFB19000CE0303DAB4219DD7E1C25
:1005E00005D0CC4523D820D00AFB0C5C012714F899
:1005F000015B0EEB0506767816F0040FECD116F0D1
:10060000030606D0012E14BF57263726AD1BAB427A
:10061000E5DC7B1C16D0B8F1000F10D16046002A33
:1006200039D0DFB91160BDE8F08F8542DCDD4FF0D5
:10063000FF37DCE7302D1AD00A239A46BEE7CCF10B
:10064000000CEBE7B8F1000F4FF022030CBF6FF086
:1006500000404FF00040CBF80030F2B1611E116055
:10066000BDE8F08FB41C75784FF00108A1E723783E
:1006700003F0DF03582B08D008239EE7302D9CD1D0
:10068000207800F0DF00582897D14FF0100A6578E5
:100690005346023492E7BDE8F08FBDE8F08F00BF0B
:1006A000F002002010B4044C13460A4601462068AC
:1006B00010BCFFF763BF00BF8C0200202DE9F04F94
:1006C000494C82460E46D4F800E000E02646344607
:1006D00014F8015B0EEB0500407800F0080000F014
:1006E000FF0C0028F2D12D2D54D02B2D04BF75788E
:1006F000B41C5BB1102B5ED04FF0FF38B8FBF3F8A1
:1007000003FB08FB6FEA0B0B994607E0302D46D040
:100710000A23DFF8D88099464FF0050B00273846AA
:100720000CE0303DAB4219DD7E1C05D0404522D89F
:100730001FD009FB0050012714F8015B0EEB0506E2
:10074000767816F0040FECD116F0030606D0012ED1
:1007500014BF57263726AD1BAB42E5DC002F0FDB5D
:10076000BCF1000F00D0404242B17FB91160BDE83A
:10077000F08F5D45DDDD4FF0FF37DDE7BDE8F08F41
:100780002223CAF800304FF0FF305AB3611E1160C7
:10079000BDE8F08FB41C75784FF0010CA9E7237801
:1007A00003F0DF03582B0DD0082399464FF0070BB9
:1007B0006FF06048B2E7302D0ED1207800F0DF00F6
:1007C000582809D14FF0100965784B464FF00F0BB0
:1007D00002346FF07048A1E74FF00F0B6FF07048D4
:1007E00099469BE7BDE8F08FF0020020999999198E
:1007F00010B4044C13460A460146206810BCFFF7AB
:100800005DBF00BF8C02002010B4044C13460A46A2
:100810000146206810BCEFF7DFBC00BF8C0200204F
:10082000F8B50E461446054610B18369002B41D039
:10083000254B9C4243D0254B9C4242D0244B9C42AA
:1008400008BFEC68A389A269A2601A0721D52369B1
:10085000FBB122686169D31A8B42F7B221DA013306
:10086000A168501C0139A1602060167062699A422B
:1008700006D0A389DB0701D50A2F01D03846F8BD81
:1008800021462846FEF766FE0028F7D04FF0FF37D6
:10089000F4E72146284600F025F80028F6D1236920
:1008A000D7E721462846FEF755FE0028EED12268FC
:1008B0000123D5E7FEF788FF034B9C42BBD16C6850
:1008C000C0E7AC68BEE700BF305101081051010815
:1008D000F0500108024B0A4601461868FFF7A0BF16
:1008E0008C020020384B70B51D6806460C4615B1C9
:1008F000AB69002B42D0354B9C4245D0344B9C42D7
:1009000058D0344B9C4208BFEC68B4F90C2093B229
:1009100019070CD52069A8B113F001021ED0636934
:1009200000225B42A361A260F0B1002070BDDD0631
:1009300042D558072AD4206942F00803A3819BB20C
:100940000028E9D103F42072B2F5007FE4D03046EC
:10095000214600F06FF8A3892069DDE7990758BFA9
:100960006269A2600028E0D1B4F90C301A06DDD526
:1009700043F04003A3814FF0FF3070BD2846FEF7DF
:1009800023FF124B9C42B9D16C68BEE7616B51B139
:1009900004F14403994204D03046FFF72BF9B4F92F
:1009A0000C200023636300232069636022F024028B
:1009B0002060C1E7AC68A8E742F040020923336039
:1009C0004FF0FF30A28170BD8C0200203051010831
:1009D00010510108F050010870B50C46B1F90E1025
:1009E000002990B015461E4613DB01AAEFF702FC62
:1009F00000280EDB029A02F47042A2F50052B2FA0D
:100A000082F252094FF48063002032602B6010B0F4
:100A100070BDA38900221B06326004D5402300204C
:100A20002B6010B070BD4FF4806300202B6010B0BD
:100A300070BD00BF8A8992070B4606D501F14702B7
:100A400001211A601A6159617047F0B583B001AB9A
:100A50006A460C460546FFF7BFFF00990646284642
:100A6000FFF70EF9B4F90C30D0B1019A124F00998A
:100A7000AF6243F08003A3812060206161611AB9F5
:100A80003343A38103B0F0BD2846B4F90E10EFF74D
:100A9000B6FBB4F90C300028F2D043F00103EFE7C5
:100AA0009A05EFD404F1470243F002030121A38128
:100AB000226022616161E5E7E1F500089368013B8E
:100AC000002B10B4936007DBCCB21368581C106085
:100AD0001970204610BC70479469A34202DBCCB267
:100AE0000A2CF2D110BCFFF79BBE00BF93B1F8B542
:100AF00014460F460646D51801E0AC4208D03A46E7
:100B000014F8011B3046FFF7D9FF431CF5D1F8BD9F
:100B10000020F8BD00207047936810B5144613B943
:100B20005360184610BD00F0D1FB0023A360636042
:100B300010BD00BF2DE9F04F9DB0884614460393C9
:100B4000814618B18369002B00F00B818B4B9845CF
:100B500000F00D818A4B984500F00C81894B984537
:100B600008BFD9F80C80B8F80C301D0740F1EF80B1
:100B7000D8F81030002B00F0EA8030238DF82A30AE
:100B80002378814DDFF804A20021202209918DF8FD
:100B90002920002B00F08580252B264603D117E065
:100BA000252B00F0868016F8013F002BF8D1B6EB1C
:100BB000040B76D022465B4641464846FFF796FF37
:100BC00001306ED0099B32785B440993002A68D0CB
:100BD00000234FF0FF31721C0493079306938DF8A6
:100BE00053301A930591012604E0049906FA03F3A1
:100BF0000B430493144664482178052200F0E8FC76
:100C0000621C431B0028F0D1049BD80644BF20225D
:100C10008DF853201907217844BF2B228DF85320DB
:100C20002A2968D0A1F13002092A0BD8079B14F8B1
:100C3000011F03EB830302EB4303A1F13002092AF6
:100C4000F5D907932E293FD00322504800F0C0FC6D
:100C500048B10499CAEB0000402202FA00F041EAD0
:100C6000000301340493217849488DF828100622A6
:100C7000013400F0ADFC00285FD0464BEBB103AB74
:100C800000934246444B04A94846AFF30080074610
:100C90007A1C06D0099B3B4409932378002B7FF4F0
:100CA0007BAFB8F80C305B0658D409981DB0BDE88E
:100CB000F08FB6EB040B8BD07CE7039B073323F05C
:100CC000070308330393E5E761782A291DD0A1F1D2
:100CD00030020023092A04F101040593B4D814F862
:100CE000011F03EB830302EB4303A1F13002092A46
:100CF000F5D90593A8E7039A1168043200290392F5
:100D000015DB0791617801349CE7039B1A68059213
:100D1000002A03F104030393B8BF4FF0FF3204F13C
:100D20000203AEBFA178A17805921C468CE7494228
:100D300043F0020307910493E4E703AB00934246B8
:100D4000154B04A9484600F0CDF80746A0E74146F8
:100D50004846FFF7C7FD00283FF40FAF4FF0FF30C4
:100D6000A4E7FEF731FD054B98457FF4F3AED9F8C3
:100D70000480F8E6D9F80880F5E600BF3051010894
:100D800010510108F05001085C520108645201083A
:100D90006852010800000000ED0A010810B4044C7C
:100DA00013460A460146206810BCFFF7C3BE00BFC9
:100DB0008C0200202DE9F0470C4691460969A26893
:100DC000DDF820808A42B8BF0A46C9F8002094F8AE
:100DD000431006461F4611B10132C9F800202368AE
:100DE00099065DD5D9F800200232C9F800202368A1
:100DF00013F0060F19461DD1E1688A1A002AD8BFE0
:100E0000194617DD04F1190A002505E0E368D9F851
:100E100000209B1AAB420CDD012352463946304676
:100E2000C047013005F10105F0D14FF0FF30BDE8BA
:100E3000F087216894F84330003318BF01238A06F5
:100E40000AD5E1185A1C302081F84300224494F856
:100E5000451082F84310023304F14302394630460C
:100E6000C0470130E1D0236803F00603042B29D0EA
:100E7000A36822699342C8BF4FF000092FDD9B1A77
:100E800099441A34002501E04D4528D0012322461B
:100E900039463046C047013005F10105F4D1C4E7B9
:100EA00013F0060F08D1E168D9F800208A1A002A49
:100EB000D8BF1946A6DCBDE794F84330003318BF0D
:100EC0000123C9E7D9F80000E168A3682269091A7B
:100ED000934221EAE179D2DCB9F1000FD1D10020AF
:100EE000BDE8F0872DE9F0430C46097E85B06E29F8
:100EF000064617460C98984604F1430C5AD01AD867
:100F0000632900F0128100F2D68000295CD05829B4
:100F100040F0F58084F8451022680368DFF864E249
:100F2000150603F104011ED4550653BF1B6801606A
:100F30001B88016019E0732900F0CF807ED86F29EB
:100F400000F0E480702940F0DA80226842F020024C
:100F50002260782384F845300368DFF82CE2150618
:100F600003F10401E0D51B680160D00744BF42F0E3
:100F700020022260002B40F09080226822F02002A4
:100F800022601021002284F843206068A0600028BD
:100F9000C0F28880226822F004022260002B62D115
:100FA000002840F08180654608296AD0C5EB0C0313
:100FB00023610CE023681A0640F1D580036862695A
:100FC000191D01601B681A60002365462361CDF876
:100FD00000803B4603AA21463046FFF7EBFE013076
:100FE00021D02A46236939463046C04701301AD0FD
:100FF0002368039813F0020FE36819D01A1A002A25
:1010000016DD04F11909002504E0E36803981A1AB3
:10101000AA420DDD01234A4639463046C047013019
:1010200005F10105F1D14FF0FF3005B0BDE8F083C7
:101030009842B8BF184605B0BDE8F083752965D061
:1010400078295CD1226884E76168A1602D2000299D
:10105000C3F1000384F8430021DB22F00402DFF82F
:1010600024E122600A216546B3FBF1F201FB123054
:1010700013461EF8002005F8012D002BF4D1082995
:1010800094D12368D90791D5626823699A428DDC8F
:10109000302305F8013C013D88E7102172E7DFF8B5
:1010A000E4E00A21002BDED19EF8003084F84230C3
:1010B00004F1420578E7642901D069291FD122682B
:1010C0000368150603F104013AD51B680160002B83
:1010D000BADBDFF8B0E00A2157E703686268191D40
:1010E00001601D680021284600F072FA002846D0F1
:1010F000401B60602061002384F8433067E70123D0
:1011000084F84210236104F14205F4E723681A06CB
:101110001ED503681A1D1B680260227EDFF864E09A
:101120006F2A14BF0A2108212CE703681A68191DC9
:101130000123016004F1420584F842202361DAE7CB
:10114000550653BF1B680160B3F900300160BEE76C
:1011500013F0400F036803F1040215BF02601B681F
:101160001B880260D9E713F0400F0368626903F13E
:10117000040101601B6814BF1A801A6024E76068CC
:10118000B8E700BF7052010884520108838903F058
:101190000903092B01D000207047FEF70DBA00BFEC
:1011A000F8B50C46054610B18369002B45D0424B7B
:1011B0009C4247D0414B9C426FD0414B9C4208BF60
:1011C000EC68B4F90C2093B200219F06616031D421
:1011D0005E0722D5616B61B104F14403994202D0EC
:1011E0002846FEF707FD236C636000206063002B38
:1011F00043D12369002B52D0B4F90C70BEB2B307AF
:1012000022D12269226028466369656A216AA8475B
:101210000028606009DD0020F8BDD80644D5190714
:101220002ED442F00402A281E3E7A3891DD143F04A
:101230002003A3814FF0FF30F8BDFEF7C5FA1E4B27
:101240009C42B7D16C68BCE71E4B1F49186801234C
:10125000A38106F00906FEF7D7FA092EA781D0D19F
:1012600021462846FEF7DEF8CBE7002243F0400394
:10127000A38162604FF0FF30F8BDE36B2360F8BDDF
:1012800021462846FEF766F90028D3D1B4F90C2090
:10129000A060A06122F00802C3E7AC6891E7214694
:1012A0002846FFF7C7FBA7E742F0400209232B605F
:1012B0004FF0FF30A281F8BD3051010810510108F4
:1012C000F0500108505101088D1101089368002B5E
:1012D00076D02DE9F04F8B8985B00C461907019027
:1012E000164629D522693AB303F002081FFA88F09E
:1012F000356800282FD04FF00009B44FC846B246D9
:10130000B84543464A4628BF3B460198B8F1000F0E
:1013100050D0216AA66AB047002871DDDAF808309B
:101320001B1A8144C0EB0808CAF80830002BE7D12B
:10133000002005B0BDE8F08F21460198FFF7D2FAF2
:10134000002840F03A81A389356803F002081FFAAB
:1013500088F00028CFD113F001095BD14F460296E7
:101360001FB39A05D4F808802CD54745C246C0F073
:10137000A48013F4906F40F0B18020685246494633
:10138000FEF786FBA0682368C8EB00005344A0600A
:1013900023603846029A93681B1A81443F1A93606F
:1013A000002BC5D0A389002FDBD1D5F800906F6842
:1013B0000835D5E7D5F80090D5F8048008359FE7C3
:1013C0000020704720682369984203D861698F42E2
:1013D00080F0B780B84528BFB84642464946FEF778
:1013E00057FBA3682268C8EB03034244A360226052
:1013F000002B49D121460198FEF7ACF8002843D0D4
:10140000B4F90C3043F040034FF0FF30A38105B036
:10141000BDE8F08F8046029082468146B9F1000F08
:101420002AD0029B002B4CD0206823696269C845F2
:10143000C34628BFCB4698425F4604D9A3681344ED
:101440009B4500F39080934520DB1346A76A216AF1
:1014500001985246B847071ED2DDB8EB070823D0E3
:10146000B368DB1BBA44C7EB0909B360002B3FF438
:101470005FAFB9F1000FD4D10023D5F800A0D5F8A3
:10148000049002930835C9E7404683E75A4651461F
:10149000FEF7FEFAA2682368CBEB02025B44B8EBCE
:1014A0000708A2602360DBD121460198FEF752F8BD
:1014B0000028A5D1CDF80880D2E72068B846BA4602
:1014C0005CE74A460A21504600F082F800286FD0B7
:1014D00001300123CAEB00080293A5E76269206886
:1014E000216902EB4208C1EB000A08EBD8780AF147
:1014F00001004FEA680838444045424684BF8046B0
:1015000042465B0542D511460198FEF7B9FB83467A
:10151000002855D052462169FEF720FAA38923F40A
:10152000906343F08003A381CAEB08030BEB0A002E
:10153000C4F81480C4F810B02060A360B846BA465E
:101540001CE76FF00043BB4228BF3B464A4693FB73
:10155000F1F30198A66A01FB03F3216AB047002862
:101560003FF718AF4CE71A4651460393FEF790FA3F
:101570002268039B01981A4422602146FDF7EAFF86
:10158000039B00287FF43CAF1F4666E7019800F0FC
:101590006FF883460028C7D1019D21692846FEF7D0
:1015A00029FBB4F90C300C2223F080032A6029E7D0
:1015B000012309F10108029336E74FF0FF30B8E646
:1015C000019A0C231360B4F90C301BE700FCFF7F79
:1015D00001F0FF01102A2BDB10F0070F08D010F8E4
:1015E000013B013A8B422DD010F0070F42B3F6D1E8
:1015F000F0B441EA012141EA014122F007047FF001
:1016000000070023F0E80256083C85EA010586EA57
:10161000010685FA47F5A3FA87F586FA47F6A5FA93
:1016200087F68EB9EED1F0BC01F0FF0102F007029F
:1016300032B110F8013B013A83EA010313B1F8D14A
:101640000020704701387047002D06BF354603382B
:10165000073815F0010F07D1013015F4807F02BF64
:10166000013015F4C03F0130F0BC0138704700BFB5
:10167000F9B1F8B506461546B2B10C4600F01CF8B3
:10168000854201D82046F8BD29463046FEF7F8FAD3
:10169000074668B12A462146FEF760F930462146E2
:1016A000FEF7A8FA3846F8BDFEF7A4FA2846F8BDBA
:1016B000F8BD1146FEF7E4BA51F8040C0028BEBF8D
:1016C000091851F8043CC018043870474E4D4920A1
:1016D00048414E444C4552004D454D204D414E41F0
:1016E00047452048414E444C455200425553204600
:1016F00041554C542048414E444C455200555341AD
:101700004745204641554C542048414E444C455293
:10171000004445425547204D4F4E2048414E444CD1
:1017200045520044554D4D592048414E444C455278
:10173000000A49535220737461636B206F7665729F
:10174000666C6F77656400537461636B20706F69BA
:101750006E74657220636F727275707465642C208C
:10176000726573657420746F20746F70206F6620CB
:10177000737461636B000A436F6E746578742062E2
:1017800065666F726520686172646661756C743A33
:101790000020202072303A2030782530386C780ACA
:1017A00020202072313A2030782530386C780A2099
:1017B000202072323A2030782530386C780A202088
:1017C0002072333A2030782530386C780A00202097
:1017D0007231323A2030782530386C780A20202057
:1017E0006C723A2030782530386C780A20202070CE
:1017F000633A2030782530386C780A202070737274
:101800003A2030782530386C780A0A004653522F37
:101810004641523A0020434653523A203078253010
:10182000386C780A0020484653523A2030782530E8
:10183000386C780A0020444653523A2030782530DC
:10184000386C780A0020414653523A2030782530CF
:10185000386C780A0020424641523A2030782530D0
:10186000386C780A004D4D4641523A203078253088
:10187000386C780A004D697363004558435F5245E0
:10188000543A2030782530386C780A0041747465F9
:101890006D7074696E6720746F207265636F6E730C
:1018A000747275637420737461746520666F72203E
:1018B000646562756767696E672E2E2E00496E201B
:1018C0004744423A0A2020736574202470633D30F7
:1018D00078256C780A20206672616D6520300A20B8
:1018E0002062740A000A49535220737461636B20AA
:1018F0006F766572666C6F776564206279206174BB
:10190000206C656173742025642062797465732E80
:101910000A0048415244204641554C542048414E0B
:10192000444C4552004641494C454420415353459F
:101930005254494F4E2E0025700A002A2A2A20525E
:10194000494F54206B65726E656C2070616E6963DF
:101950003A0A25730A0A002A2A2A2068616C7465EB
:10196000642E0A0A006D61696E28293A205468695C
:10197000732069732052494F542120285665727391
:10198000696F6E3A20554E4B4E4F574E2028627568
:10199000696C646469723A202F686F6D652F656C9D
:1019A0006F7065732F50464531352F52494F54297A
:1019B000290A0069646C65006D61696E005F510001
:1019C000E91A0108F11A0108FA1A0108031B0108B3
:1019D000091B0108111B01081A1B0108231B010820
:1019E0002C1B0108341B01083C1B01087374617433
:1019F00065006E616D650009706964207C20252D8D
:101A00003231737C20252D397351207C207072690E
:101A1000207C20737461636B2020282075736564BB
:101A200029207C2062617365206164647220207CBF
:101A30002063757272656E7420202020200A0009D0
:101A400020202D207C206973725F737461636B208A
:101A500020202020202020202020207C202D20201D
:101A60002020202020202D207C2020202D207C20A4
:101A7000253669202825356929207C2025313070BC
:101A8000207C20253130700A000925336869207CCC
:101A900020252D323073207C20252D387320252ED3
:101AA0003173207C20253369207C2025366920284D
:101AB00025356929207C2025313070207C20253176
:101AC0003070200A007C0053554D000925357320E5
:101AD000252D3231737C253133732536732025361D
:101AE000692028253569290A0073746F7070656450
:101AF00000736C656570696E6700626C206D75744B
:101B0000657800626C20727800626C2073656E6488
:101B100000626C207265706C7900626C20616E7975
:101B2000666C00626C20616C6C666C00626C206D8F
:101B3000626F780072756E6E696E670070656E64B4
:101B4000696E67000044004000000200030002408C
:101B50000200024007070026004800400000040081
:101B6000090C0240080C0240070700270706040280
:101B70000107070503020000003001400700024092
:101B8000060002400500024004000240050000007B
:101B90000010000001000000003800400F04024067
:101BA0000E0402400D0402400C0402400500000037
:101BB000004000000000000000000040FFFFFFFFA9
:101BC00001000000001C0000000C0040FFFFFFFFB0
:101BD000080000000032000002020000FC1C0108A6
:101BE000021D0108891B0008000000000000000021
:101BF000000000004572726F722073656E64696E3A
